 lcdc

 Timestamp is 4da2a521 (Mon Apr 11 18:52:17 2011)

 Preferred load address is 10000000

 Start         Length     Name                   Class
 0001:00000000 00000004H .CRT$XCA                CODE
 0001:00000004 00000018H .CRT$XCU                CODE
 0001:0000001c 00000004H .CRT$XCZ                CODE
 0001:00000020 00000004H .CRT$XIA                CODE
 0001:00000024 00000004H .CRT$XIZ                CODE
 0001:00000028 00000004H .CRT$XPA                CODE
 0001:0000002c 00000004H .CRT$XPZ                CODE
 0001:00000030 00000004H .CRT$XTA                CODE
 0001:00000034 00000004H .CRT$XTZ                CODE
 0001:00000040 000114c6H .rdata                  CODE
 0001:00011508 00000021H .rdata$debug            CODE
 0001:0001152c 0004a174H .text                   CODE
 0001:0005b6a0 000000b0H .text$yc                CODE
 0001:0005b750 00000094H .xdata                  CODE
 0001:0005b7e4 0000003cH .idata$2                CODE
 0001:0005b820 00000014H .idata$3                CODE
 0001:0005b834 00000160H .idata$4                CODE
 0001:0005b994 000000a2H .idata$6                CODE
 0001:0005ba40 0000005cH .edata                  CODE
 0002:00000000 00000160H .idata$5                DATA
 0002:00000160 00003360H .data                   DATA
 0002:000034c0 00004010H .bss                    DATA
 0003:00000000 00001040H .pdata                  DATA

  Address         Publics by Value              Rva+Base       Lib:Object

 0000:00000000       ___safe_se_handler_count   00000000     <absolute>
 0000:00000000       ___safe_se_handler_table   00000000     <absolute>
 0001:00000000       __xc_a                     10001000     corelib0:crt0init.obj
 0001:0000001c       __xc_z                     1000101c     corelib0:crt0init.obj
 0001:00000020       __xi_a                     10001020     corelib0:crt0init.obj
 0001:00000024       __xi_z                     10001024     corelib0:crt0init.obj
 0001:00000028       __xp_a                     10001028     corelib0:crt0init.obj
 0001:0000002c       __xp_z                     1000102c     corelib0:crt0init.obj
 0001:00000030       __xt_a                     10001030     corelib0:crt0init.obj
 0001:00000034       __xt_z                     10001034     corelib0:crt0init.obj
 0001:00000060       ??_C@_1FO@OPBNOLOL@?$AA?5?$AAB?$AAS?$AAP?$AAG?$AAe?$AAt?$AAM?$AAo?$AAd?$AAe?$AAD?$AAe?$AAs?$AAc?$AAr?$AAi?$AAp?$AAt?$AAo?$AAr?$AA?3?$AA?5?$AAN?$AAo?$AA?5?$AAm?$AAo?$AAd?$AAe?$AA?5?$AAm@ 10001060     bsplcdc.obj
 0001:000000c0       ??_C@_19OBGHODPD@?$AAM?$AAo?$AAd?$AAe?$AA?$AA@ 100010c0     bsplcdc.obj
 0001:000000cc       ??_C@_1CK@ENPFCICM@?$AAD?$AAr?$AAi?$AAv?$AAe?$AAr?$AAs?$AA?2?$AAD?$AAi?$AAs?$AAp?$AAl?$AAa?$AAy?$AA?2?$AAL?$AAC?$AAD?$AAC?$AA?$AA@ 100010cc     bsplcdc.obj
 0001:000000f8       ??_C@_1CM@JBPFNDBJ@?$AAD?$AAr?$AAi?$AAv?$AAe?$AAr?$AAs?$AA?2?$AAB?$AAu?$AAi?$AAl?$AAt?$AAI?$AAn?$AA?2?$AAL?$AAC?$AAD?$AAA?$AAD?$AA?$AA@ 100010f8     bsplcdc.obj
 0001:00000128       ??_C@_1FG@DLFCFGFO@?$AAG?$AAe?$AAt?$AAV?$AAM?$AAe?$AAm?$AAS?$AAi?$AAz?$AAe?$AAF?$AAr?$AAo?$AAm?$AAR?$AAe?$AAg?$AAi?$AAs?$AAt?$AAr?$AAy?$AA?3?$AA?5?$AA?$CF?$AAs?$AA?0?$AA?5?$AAs?$AAi?$AAz@ 10001128     bsplcdc.obj
 0001:00000180       ??_C@_1M@LEHIOEPF@?$AAf?$AAa?$AAi?$AAl?$AAs?$AA?$AA@ 10001180     bsplcdc.obj
 0001:0000018c       ??_C@_1BC@PEGPCAEI@?$AAs?$AAu?$AAc?$AAc?$AAe?$AAe?$AAd?$AAs?$AA?$AA@ 1000118c     bsplcdc.obj
 0001:000001a0       ??_C@_1MK@GCOIBOAM@?$AAD?$AAD?$AAI?$AAP?$AAU?$AA?5?$AAG?$AAe?$AAt?$AAV?$AAM?$AAe?$AAm?$AAS?$AAi?$AAz?$AAe?$AAF?$AAr?$AAo?$AAm?$AAR?$AAe?$AAg?$AAi?$AAs?$AAt?$AAr?$AAy?$AA?3?$AA?5?$AAF@ 100011a0     bsplcdc.obj
 0001:0000026c       ??_C@_1BK@CDFMAEAD@?$AAV?$AAi?$AAd?$AAe?$AAo?$AAM?$AAe?$AAm?$AAS?$AAi?$AAz?$AAe?$AA?$AA@ 1000126c     bsplcdc.obj
 0001:00000288       ??_C@_1FM@BKDNCKAH@?$AA?$CF?$AAs?$AA?3?$AA?5?$AAF?$AAa?$AAi?$AAl?$AAe?$AAd?$AA?5?$AAt?$AAo?$AA?5?$AAo?$AAp?$AAe?$AAn?$AA?5?$AAr?$AAe?$AAg?$AA?5?$AAp?$AAa?$AAt?$AAh?$AA?3?$AA?$CF?$AAs?$AA?5?$AA?$FL@ 10001288     bsplcdc.obj
 0001:000002e4       ??_C@_1CM@DOEOHNFH@?$AAB?$AAS?$AAP?$AAG?$AAe?$AAt?$AAV?$AAi?$AAd?$AAe?$AAo?$AAM?$AAe?$AAm?$AAo?$AAr?$AAy?$AAS?$AAi?$AAz?$AAe?$AA?$AA@ 100012e4     bsplcdc.obj
 0001:00000310       ??_C@_1CE@JDIIGOKD@?$AA?9?$AAS?$AAe?$AAt?$AAW?$AAa?$AAl?$AAl?$AAp?$AAa?$AAp?$AAe?$AAr?$AA?$CI?$AA?$CJ?$AA?$AN?$AA?6?$AA?$AA@ 10001310     bsplcdc.obj
 0001:00000338       ??_C@_1FC@JEMHBHLB@?$AA?5?$AAS?$AAe?$AAt?$AAW?$AAa?$AAl?$AAl?$AAp?$AAa?$AAp?$AAe?$AAr?$AA?3?$AA?5?$AAC?$AAa?$AAn?$AA?8?$AAt?$AA?5?$AAo?$AAp?$AAe?$AAn?$AA?5?$AAr?$AAe?$AAg?$AAi?$AAs?$AAt@ 10001338     bsplcdc.obj
 0001:00000390       ??_C@_1EM@GDBJLPMO@?$AA?5?$AAS?$AAe?$AAt?$AAW?$AAa?$AAl?$AAl?$AAp?$AAa?$AAp?$AAe?$AAr?$AA?3?$AA?5?$AAS?$AAe?$AAt?$AA?5?$AAw?$AAa?$AAl?$AAl?$AAp?$AAa?$AAp?$AAe?$AAr?$AA?5?$AAf?$AAa?$AAi@ 10001390     bsplcdc.obj
 0001:000003dc       ??_C@_1BE@NLLCHOPM@?$AAW?$AAa?$AAl?$AAl?$AAp?$AAa?$AAp?$AAe?$AAr?$AA?$AA@ 100013dc     bsplcdc.obj
 0001:000003f0       ??_C@_1CK@NGGJLNDN@?$AAC?$AAo?$AAn?$AAt?$AAr?$AAo?$AAl?$AAP?$AAa?$AAn?$AAe?$AAl?$AA?2?$AAD?$AAe?$AAs?$AAk?$AAt?$AAo?$AAp?$AA?$AA@ 100013f0     bsplcdc.obj
 0001:0000041c       ??_C@_1CE@FKEIJJFP@?$AA?$CL?$AAS?$AAe?$AAt?$AAW?$AAa?$AAl?$AAl?$AAp?$AAa?$AAp?$AAe?$AAr?$AA?$CI?$AA?$CJ?$AA?$AN?$AA?6?$AA?$AA@ 1000141c     bsplcdc.obj
 0001:000004f4       ??_C@_1DG@OLIIDDGP@?$AAM?$AAX?$AAD?$AAD?$AAL?$AAc?$AAd?$AAc?$AA?3?$AA?5?$AAG?$AAe?$AAt?$AAG?$AAP?$AAE?$AA?$CI?$AA0?$AAx?$AA?$CF?$AA0?$AA8?$AAx?$AA?$CJ?$AA?$AN?$AA?6?$AA?$AA@ 100014f4     lcdc_common_topaz_v1:DDLcdc.obj
 0001:00000530       ??_C@_1FA@KINKKOGP@?$AAM?$AAX?$AAD?$AAD?$AAL?$AAc?$AAd?$AAc?$AA?3?$AA?5?$AAF?$AAa?$AAi?$AAl?$AAe?$AAd?$AA?5?$AAt?$AAo?$AA?5?$AAg?$AAe?$AAt?$AA?5?$AAG?$AAP?$AAE?$AA?5?$AAi?$AAn?$AAs?$AAt@ 10001530     lcdc_common_topaz_v1:DDLcdc.obj
 0001:00000580       ??_C@_1EI@ECHABLAD@?$AAM?$AAX?$AAD?$AAD?$AAL?$AAc?$AAd?$AAc?$AA?3?$AA?5?$AAc?$AAl?$AAa?$AAs?$AAs?$AA?5?$AAc?$AAo?$AAn?$AAs?$AAt?$AAr?$AAu?$AAc?$AAt?$AAi?$AAo?$AAn?$AA?5?$AA?$CF?$AAs?$AA?$CB@ 10001580     lcdc_common_topaz_v1:DDLcdc.obj
 0001:000005c8       ??_C@_1KI@CAACDMHF@?$AAM?$AAX?$AAD?$AAD?$AAL?$AAc?$AAd?$AAc?$AA?5?$AAI?$AAn?$AAi?$AAt?$AA?3?$AA?5?$AAf?$AAa?$AAi?$AAl?$AAe?$AAd?$AA?5?$AAt?$AAo?$AA?5?$AAa?$AAl?$AAl?$AAo?$AAc?$AAa?$AAt@ 100015c8     lcdc_common_topaz_v1:DDLcdc.obj
 0001:00000670       ??_7MXDDLcdc@@6B@          10001670     lcdc_common_topaz_v1:DDLcdc.obj
 0001:00000758       ??_C@_1GC@GACOFDCB@?$AAM?$AAX?$AAD?$AAD?$AAL?$AAc?$AAd?$AAc?$AA?5?$AAS?$AAe?$AAt?$AAM?$AAo?$AAd?$AAe?$AA?3?$AA?5?$AAf?$AAa?$AAi?$AAl?$AA?5?$AAt?$AAo?$AA?5?$AAi?$AAn?$AAi?$AAt?$AAi?$AAa@ 10001758     lcdc_common_topaz_v1:DDLcdc.obj
 0001:000007c0       ??_C@_1GM@DNNNOGED@?$AAM?$AAX?$AAD?$AAD?$AAL?$AAc?$AAd?$AAc?$AA?5?$AAS?$AAe?$AAt?$AAM?$AAo?$AAd?$AAe?$AA?3?$AA?5?$AAC?$AAo?$AAu?$AAl?$AAd?$AAn?$AA?8?$AAt?$AA?5?$AAa?$AAl?$AAl?$AAo?$AAc@ 100017c0     lcdc_common_topaz_v1:DDLcdc.obj
 0001:0000082c       ??_C@_1DA@JMJKEBFM@?$AA?7?$AA?7?$AAm?$AA_?$AAn?$AAS?$AAc?$AAr?$AAe?$AAe?$AAn?$AAB?$AAp?$AAp?$AA?3?$AA?5?$AA?5?$AA?5?$AA?5?$AA?$CF?$AAd?$AA?$AN?$AA?6?$AA?$AA@ 1000182c     lcdc_common_topaz_v1:DDLcdc.obj
 0001:0000085c       ??_C@_1DA@LNJDMHOI@?$AA?7?$AA?7?$AAm?$AA_?$AAn?$AAS?$AAc?$AAr?$AAe?$AAe?$AAn?$AAS?$AAt?$AAr?$AAi?$AAd?$AAe?$AA?3?$AA?5?$AA?$CF?$AAd?$AA?$AN?$AA?6?$AA?$AA@ 1000185c     lcdc_common_topaz_v1:DDLcdc.obj
 0001:0000088c       ??_C@_1DA@CKHDBKKN@?$AA?7?$AA?7?$AAm?$AA_?$AAn?$AAS?$AAc?$AAr?$AAe?$AAe?$AAn?$AAH?$AAe?$AAi?$AAg?$AAh?$AAt?$AA?3?$AA?5?$AA?$CF?$AAd?$AA?$AN?$AA?6?$AA?$AA@ 1000188c     lcdc_common_topaz_v1:DDLcdc.obj
 0001:000008bc       ??_C@_1DA@LBBMGECH@?$AA?7?$AA?7?$AAm?$AA_?$AAn?$AAS?$AAc?$AAr?$AAe?$AAe?$AAn?$AAW?$AAi?$AAd?$AAt?$AAh?$AA?3?$AA?5?$AA?5?$AA?$CF?$AAd?$AA?$AN?$AA?6?$AA?$AA@ 100018bc     lcdc_common_topaz_v1:DDLcdc.obj
 0001:000008f0       ??_C@_1EO@EIJCBDNL@?$AAM?$AAX?$AAD?$AAD?$AAL?$AAc?$AAd?$AAc?$AA?5?$AAI?$AAn?$AAi?$AAt?$AA?3?$AA?5?$AAC?$AAu?$AAr?$AAr?$AAe?$AAn?$AAt?$AA?5?$AAd?$AAi?$AAs?$AAp?$AAl?$AAa?$AAy?$AA?5?$AAm@ 100018f0     lcdc_common_topaz_v1:DDLcdc.obj
 0001:00000940       ??_C@_1HO@CBJCNPND@?$AAM?$AAX?$AAD?$AAD?$AAL?$AAc?$AAd?$AAc?$AA?5?$AAI?$AAn?$AAi?$AAt?$AA?3?$AA?5?$AAI?$AAn?$AAv?$AAa?$AAl?$AAi?$AAd?$AA?5?$AAB?$AAP?$AAP?$AA?5?$AAv?$AAa?$AAl?$AAu?$AAe@ 10001940     lcdc_common_topaz_v1:DDLcdc.obj
 0001:000009c0       ??_C@_1IA@FOIDIIMC@?$AAM?$AAX?$AAD?$AAD?$AAL?$AAc?$AAd?$AAc?$AA?5?$AAI?$AAn?$AAi?$AAt?$AA?3?$AA?5?$AAS?$AAc?$AAr?$AAe?$AAe?$AAn?$AA?5?$AAw?$AAi?$AAd?$AAt?$AAh?$AA?5?$AA?$CI?$AA?$CF?$AAd?$AA?$CJ@ 100019c0     lcdc_common_topaz_v1:DDLcdc.obj
 0001:00000a40       ??_C@_1HE@MEHKPNBG@?$AAF?$AAa?$AAi?$AAl?$AAe?$AAd?$AA?5?$AAt?$AAo?$AA?5?$AAg?$AAe?$AAt?$AA?5?$AAt?$AAh?$AAe?$AA?5?$AAm?$AAo?$AAd?$AAe?$AA?5?$AAd?$AAe?$AAs?$AAc?$AAr?$AAi?$AAp?$AAt?$AAo@ 10001a40     lcdc_common_topaz_v1:DDLcdc.obj
 0001:00000ab4       ??_C@_1DM@MMNPAEOA@?$AAF?$AAa?$AAi?$AAl?$AAe?$AAd?$AA?5?$AAt?$AAo?$AA?5?$AAA?$AAl?$AAl?$AAo?$AAc?$AAa?$AAt?$AAe?$AAV?$AAi?$AAd?$AAe?$AAo?$AAM?$AAe?$AAm?$AAo?$AAr?$AAy?$AA?$AA@ 10001ab4     lcdc_common_topaz_v1:DDLcdc.obj
 0001:00000af0       ??_C@_1DE@PMDJFIKK@?$AAF?$AAa?$AAi?$AAl?$AAe?$AAd?$AA?5?$AAt?$AAo?$AA?5?$AAF?$AAr?$AAe?$AAe?$AAV?$AAi?$AAd?$AAe?$AAo?$AAM?$AAe?$AAm?$AAo?$AAr?$AAy?$AA?$AA@ 10001af0     lcdc_common_topaz_v1:DDLcdc.obj
 0001:00000b24       ??_C@_1CI@OHCJFJPM@?$AAE?$AAR?$AAR?$AAO?$AAR?$AA?3?$AA?5?$AA?$CF?$AAs?$AA?5?$AAl?$AAi?$AAn?$AAe?$AA?5?$AA?$CF?$AAd?$AA?3?$AA?5?$AA?$AA@ 10001b24     lcdc_common_topaz_v1:DDLcdc.obj
 0001:00000b50       ??_C@_1KK@OPMOFFPA@?$AAc?$AA?3?$AA?2?$AAw?$AAi?$AAn?$AAc?$AAe?$AAr?$AAo?$AAo?$AAt?$AAs?$AA?2?$AAt?$AAo?$AAp?$AAa?$AAz?$AA?2?$AAw?$AAi?$AAn?$AAc?$AAe?$AA7?$AA0?$AA0?$AA?2?$AAp?$AAl?$AAa@ 10001b50     lcdc_common_topaz_v1:DDLcdc.obj
 0001:00000c00       ??_C@_1FE@KGKMFBBJ@?$AAM?$AAX?$AAD?$AAD?$AAL?$AAc?$AAd?$AAc?$AA?5?$AAG?$AAe?$AAt?$AAM?$AAo?$AAd?$AAe?$AAI?$AAn?$AAf?$AAo?$AA?3?$AA?5?$AAw?$AAr?$AAo?$AAn?$AAg?$AA?5?$AAm?$AAo?$AAd?$AAe@ 10001c00     lcdc_common_topaz_v1:DDLcdc.obj
 0001:00000c58       ??_C@_1FI@DPPBMLME@?$AAM?$AAX?$AAD?$AAD?$AAL?$AAc?$AAd?$AAc?$AA?5?$AAG?$AAe?$AAt?$AAM?$AAo?$AAd?$AAe?$AAI?$AAn?$AAf?$AAo?$AAE?$AAx?$AA?3?$AA?5?$AAw?$AAr?$AAo?$AAn?$AAg?$AA?5?$AAm?$AAo@ 10001c58     lcdc_common_topaz_v1:DDLcdc.obj
 0001:00000cb0       ??_C@_1BI@NJMEJEKJ@?$AAm?$AAo?$AAd?$AAe?$AA?5?$AA0?$AAx?$AA?$CF?$AAx?$AA?$AN?$AA?6?$AA?$AA@ 10001cb0     lcdc_common_topaz_v1:DDLcdc.obj
 0001:00000cc8       ??_C@_1FO@ELJEEDAG@?$AAM?$AAX?$AAD?$AAD?$AAL?$AAc?$AAd?$AAc?$AA?5?$AAI?$AAn?$AAi?$AAt?$AA?3?$AA?5?$AAD?$AAe?$AAf?$AAa?$AAu?$AAl?$AAt?$AA?5?$AAd?$AAi?$AAs?$AAp?$AAl?$AAa?$AAy?$AA?5?$AAm@ 10001cc8     lcdc_common_topaz_v1:DDLcdc.obj
 0001:00000d28       ??_C@_1JG@GCGDCFPB@?$AAM?$AAX?$AAD?$AAD?$AAL?$AAc?$AAd?$AAc?$AA?5?$AAI?$AAn?$AAi?$AAt?$AAH?$AAa?$AAr?$AAd?$AAw?$AAa?$AAr?$AAe?$AA?3?$AA?5?$AAf?$AAa?$AAi?$AAl?$AA?5?$AAt?$AAo?$AA?5?$AAi@ 10001d28     lcdc_common_topaz_v1:DDLcdc.obj
 0001:00000dc0       ??_C@_1IM@OFBBKFIF@?$AAM?$AAX?$AAD?$AAD?$AAL?$AAc?$AAd?$AAc?$AA?5?$AAI?$AAn?$AAi?$AAt?$AAH?$AAa?$AAr?$AAd?$AAw?$AAa?$AAr?$AAe?$AA?3?$AA?5?$AAf?$AAa?$AAi?$AAl?$AA?5?$AAt?$AAo?$AA?5?$AAi@ 10001dc0     lcdc_common_topaz_v1:DDLcdc.obj
 0001:00000e50       ??_C@_1EE@FNCPOFJK@?$AAF?$AAa?$AAi?$AAl?$AAe?$AAd?$AA?5?$AAt?$AAo?$AA?5?$AAo?$AAb?$AAt?$AAa?$AAi?$AAn?$AA?5?$AAs?$AAy?$AAs?$AAi?$AAn?$AAt?$AAr?$AA?5?$AAv?$AAa?$AAl?$AAu?$AAe?$AA?$CB?$AA?$AN@ 10001e50     lcdc_common_topaz_v1:DDLcdc.obj
 0001:00000e98       ??_C@_1KE@PMDBHBFH@?$AAM?$AAX?$AAD?$AAD?$AAL?$AAc?$AAd?$AAc?$AA?5?$AAI?$AAn?$AAi?$AAt?$AAH?$AAa?$AAr?$AAd?$AAw?$AAa?$AAr?$AAe?$AA?3?$AA?5?$AAf?$AAa?$AAi?$AAl?$AAe?$AAd?$AA?5?$AAt?$AAo@ 10001e98     lcdc_common_topaz_v1:DDLcdc.obj
 0001:00000f40       ??_C@_1IK@LNPNMHKJ@?$AAM?$AAX?$AAD?$AAD?$AAL?$AAc?$AAd?$AAc?$AA?5?$AAI?$AAn?$AAi?$AAt?$AAH?$AAa?$AAr?$AAd?$AAw?$AAa?$AAr?$AAe?$AA?3?$AA?5?$AAf?$AAa?$AAi?$AAl?$AAe?$AAd?$AA?5?$AAt?$AAo@ 10001f40     lcdc_common_topaz_v1:DDLcdc.obj
 0001:00000fd0       ??_C@_1EE@MGBMNNCD@?$AAL?$AAc?$AAd?$AAc?$AAC?$AAl?$AAa?$AAs?$AAs?$AA?3?$AA?5?$AAV?$AAi?$AAr?$AAt?$AAu?$AAa?$AAl?$AAA?$AAl?$AAl?$AAo?$AAc?$AA?5?$AAf?$AAa?$AAi?$AAl?$AAe?$AAd?$AA?$CB?$AA?$AN@ 10001fd0     lcdc_common_topaz_v1:DDLcdc.obj
 0001:00001018       ??_C@_1GA@ECJIMKOK@?$AA?7?$AAS?$AAi?$AAz?$AAe?$AA?3?$AA?5?$AA?5?$AA?5?$AA?5?$AA?5?$AA?5?$AA?5?$AA?5?$AA?5?$AA?5?$AA?5?$AA?5?$AA?5?$AA?5?$AA?5?$AA?5?$AA?5?$AA?5?$AA?5?$AA?5?$AA?5?$AA?5?$AA?5?$AA?5?$AA?5?$AA?5@ 10002018     lcdc_common_topaz_v1:DDLcdc.obj
 0001:00001078       ??_C@_1GA@NNFKDLNG@?$AA?7?$AAP?$AAh?$AAy?$AAs?$AAi?$AAc?$AAa?$AAl?$AA?5?$AAa?$AAd?$AAd?$AAr?$AAe?$AAs?$AAs?$AA?5?$AAo?$AAf?$AA?5?$AAv?$AAi?$AAd?$AAe?$AAo?$AA?5?$AAm?$AAe?$AAm?$AAo?$AAr@ 10002078     lcdc_common_topaz_v1:DDLcdc.obj
 0001:000010d8       ??_C@_1GA@OKLECHH@?$AA?7?$AAV?$AAi?$AAr?$AAt?$AAu?$AAa?$AAl?$AA?5?$AAa?$AAd?$AAd?$AAr?$AAe?$AAs?$AAs?$AA?5?$AAo?$AAf?$AA?5?$AAv?$AAi?$AAd?$AAe?$AAo?$AA?5?$AAm?$AAe?$AAm?$AAo?$AAr?$AAy@ 100020d8     lcdc_common_topaz_v1:DDLcdc.obj
 0001:00001138       ??_C@_1GA@EKNPOFEF@?$AA?7?$AAV?$AAi?$AAr?$AAt?$AAu?$AAa?$AAl?$AA?5?$AAa?$AAd?$AAd?$AAr?$AAe?$AAs?$AAs?$AA?5?$AAm?$AAa?$AAp?$AAp?$AAe?$AAd?$AA?5?$AAa?$AAc?$AAc?$AAe?$AAs?$AAs?$AA?5?$AAw@ 10002138     lcdc_common_topaz_v1:DDLcdc.obj
 0001:00001198       ??_C@_1DM@LFJKIAPB@?$AAM?$AAX?$AAD?$AAD?$AAL?$AAc?$AAd?$AAc?$AA?5?$AAA?$AAl?$AAl?$AAo?$AAc?$AAV?$AAi?$AAd?$AAe?$AAo?$AAM?$AAe?$AAm?$AAo?$AAr?$AAy?$AA?3?$AA?5?$AA?$AN?$AA?6?$AA?$AA@ 10002198     lcdc_common_topaz_v1:DDLcdc.obj
 0001:000011d8       ??_C@_1IE@DBADCNLN@?$AAM?$AAX?$AAD?$AAD?$AAL?$AAc?$AAd?$AAc?$AA?5?$AAA?$AAl?$AAl?$AAo?$AAc?$AAV?$AAi?$AAd?$AAe?$AAo?$AAM?$AAe?$AAm?$AAo?$AAr?$AAy?$AA?3?$AA?5?$AAf?$AAa?$AAi?$AAl?$AAe@ 100021d8     lcdc_common_topaz_v1:DDLcdc.obj
 0001:0000125c       ??_C@_1DK@JJAIFIFI@?$AA?$CF?$AAs?$AA?$CI?$AA?$CJ?$AA?3?$AA?5?$AAM?$AAm?$AAM?$AAa?$AAp?$AAI?$AAo?$AAS?$AAp?$AAa?$AAc?$AAe?$AA?5?$AAf?$AAa?$AAi?$AAl?$AAe?$AAd?$AA?$CB?$AA?$AN?$AA?6?$AA?$AA@ 1000225c     lcdc_common_topaz_v1:DDLcdc.obj
 0001:00001298       ??_C@_1DG@NCKPPAEH@?$AAM?$AAX?$AAD?$AAD?$AAL?$AAc?$AAd?$AAc?$AA?3?$AA?3?$AAA?$AAl?$AAl?$AAo?$AAc?$AAV?$AAi?$AAd?$AAe?$AAo?$AAM?$AAe?$AAm?$AAo?$AAr?$AAy?$AA?$AA@ 10002298     lcdc_common_topaz_v1:DDLcdc.obj
 0001:000012d0       ??_C@_1DA@GKJLOJNH@?$AAW?$AAa?$AAi?$AAt?$AA?5?$AAf?$AAo?$AAr?$AA?5?$AAS?$AAy?$AAn?$AAc?$AAT?$AAh?$AAr?$AAe?$AAa?$AAd?$AA?5?$AAe?$AAn?$AAd?$AA?$AA@ 100022d0     lcdc_common_topaz_v1:DDLcdc.obj
 0001:00001300       ??_C@_1FE@MCMAOJFB@?$AAM?$AAX?$AAD?$AAD?$AAL?$AAc?$AAd?$AAc?$AA?5?$AAI?$AAn?$AAt?$AAr?$AAP?$AAr?$AAo?$AAc?$AA?3?$AA?5?$AAi?$AAn?$AAt?$AAe?$AAr?$AAr?$AAu?$AAp?$AAt?$AA?5?$AAe?$AAr?$AAr@ 10002300     lcdc_common_topaz_v1:DDLcdc.obj
 0001:0000140c       ??_C@_1CE@LGAKADBG@?$AAD?$AAi?$AAs?$AAp?$AAl?$AAa?$AAy?$AAP?$AAo?$AAw?$AAe?$AAr?$AAC?$AAl?$AAa?$AAs?$AAs?$AA?$AA@ 1000240c     lcdc_common_topaz_v1:DDLcdcPower.obj
 0001:00001430       ??_C@_1CG@BEPCNIEH@?$AAS?$AAy?$AAs?$AAt?$AAe?$AAm?$AA?2?$AAG?$AAD?$AAI?$AA?2?$AAD?$AAr?$AAi?$AAv?$AAe?$AAr?$AAs?$AA?$AA@ 10002430     lcdc_common_topaz_v1:DDLcdcPower.obj
 0001:00001458       ??_C@_1FK@FNONLNGN@?$AA?$CF?$AAs?$AA?3?$AA?5?$AAD?$AAE?$AAB?$AAU?$AAG?$AAC?$AAH?$AAK?$AA?5?$AAf?$AAa?$AAi?$AAl?$AAe?$AAd?$AA?5?$AAi?$AAn?$AA?5?$AAf?$AAi?$AAl?$AAe?$AA?5?$AA?$CF?$AAs?$AA?5?$AAa@ 10002458     lcdc_common_topaz_v1:DDLcdcPower.obj
 0001:000014b8       ??_C@_1LE@NKAGLOHM@?$AAc?$AA?3?$AA?2?$AAw?$AAi?$AAn?$AAc?$AAe?$AAr?$AAo?$AAo?$AAt?$AAs?$AA?2?$AAt?$AAo?$AAp?$AAa?$AAz?$AA?2?$AAw?$AAi?$AAn?$AAc?$AAe?$AA7?$AA0?$AA0?$AA?2?$AAp?$AAl?$AAa@ 100024b8     lcdc_common_topaz_v1:DDLcdcPower.obj
 0001:00001570       ??_C@_1EO@BHDHHEGO@?$AA?$HL?$AAE?$AAB?$AA9?$AA1?$AAC?$AA7?$AAC?$AA9?$AA?9?$AA8?$AAB?$AAF?$AA6?$AA?9?$AA4?$AAa?$AA2?$AAd?$AA?9?$AA9?$AAA?$AAB?$AA8?$AA?9?$AA6?$AA9?$AA7?$AA2?$AA4?$AAE?$AAE@ 10002570     lcdc_common_topaz_v1:DDLcdcPower.obj
 0001:000015c0       ??_C@_1JI@FOBCENMN@?$AAM?$AAX?$AAD?$AAD?$AAL?$AAc?$AAd?$AAc?$AA?5?$AAP?$AAm?$AAT?$AAo?$AAV?$AAi?$AAd?$AAe?$AAo?$AAP?$AAo?$AAw?$AAe?$AAr?$AAS?$AAt?$AAa?$AAt?$AAe?$AA?3?$AA?5?$AAm?$AAa@ 100025c0     lcdc_common_topaz_v1:DDLcdcPower.obj
 0001:00001658       ??_C@_1JM@PACHABC@?$AAM?$AAX?$AAD?$AAD?$AAL?$AAc?$AAd?$AAc?$AA?5?$AAV?$AAi?$AAd?$AAe?$AAo?$AAT?$AAo?$AAP?$AAm?$AAP?$AAo?$AAw?$AAe?$AAr?$AAS?$AAt?$AAa?$AAt?$AAe?$AA?3?$AA?5?$AAm?$AAa@ 10002658     lcdc_common_topaz_v1:DDLcdcPower.obj
 0001:000016f8       ??_C@_1IA@INLOHPGM@?$AAM?$AAX?$AAD?$AAD?$AAL?$AAc?$AAd?$AAc?$AA?5?$AAC?$AAo?$AAn?$AAv?$AAe?$AAr?$AAt?$AAS?$AAt?$AAr?$AAi?$AAn?$AAg?$AAT?$AAo?$AAG?$AAu?$AAi?$AAd?$AA?3?$AA?5?$AAE?$AAX@ 100026f8     lcdc_common_topaz_v1:DDLcdcPower.obj
 0001:00001778       ??_C@_1GI@LBPPMOKF@?$AA?$HL?$AA?$CF?$AA0?$AA8?$AAl?$AAX?$AA?9?$AA?$CF?$AA0?$AA4?$AAX?$AA?9?$AA?$CF?$AA0?$AA4?$AAX?$AA?9?$AA?$CF?$AA0?$AA2?$AAX?$AA?$CF?$AA0?$AA2?$AAX?$AA?9?$AA?$CF?$AA0?$AA2?$AAX?$AA?$CF?$AA0@ 10002778     lcdc_common_topaz_v1:DDLcdcPower.obj
 0001:0000194c       ??_C@_1DA@CLIHLKHC@?$AAI?$AAn?$AAv?$AAa?$AAl?$AAi?$AAd?$AA?5?$AAd?$AAi?$AAr?$AAe?$AAc?$AAt?$AAi?$AAo?$AAn?$AA?3?$AA?5?$AA?$CF?$AAd?$AA?$AN?$AA?6?$AA?$AA@ 1000294c     lcdc_common_topaz_v1:DDLcdcLine.obj
 0001:00001a38       ??_C@_1JI@HONGKBPO@?$AAC?$AAr?$AAe?$AAa?$AAt?$AAi?$AAn?$AAg?$AA?5?$AAa?$AA?5?$AAD?$AAD?$AAG?$AAP?$AAE?$AAS?$AAu?$AAr?$AAf?$AA?5?$AAi?$AAn?$AA?5?$AAs?$AAy?$AAs?$AAt?$AAe?$AAm?$AA?5?$AAm@ 10002a38     lcdc_common_topaz_v1:DDLcdcSurf.obj
 0001:00001ad0       ??_C@_1GI@MHDEJMFC@?$AAV?$AAi?$AAd?$AAe?$AAo?$AA?5?$AAm?$AAe?$AAm?$AAo?$AAr?$AAy?$AA?5?$AAr?$AAe?$AAm?$AAa?$AAi?$AAn?$AAi?$AAn?$AAg?$AA?5?$AAa?$AAf?$AAt?$AAe?$AAr?$AA?5?$AAs?$AAu?$AAr@ 10002ad0     lcdc_common_topaz_v1:DDLcdcSurf.obj
 0001:00001b38       ??_C@_1GC@BIJMGCND@?$AAV?$AAi?$AAd?$AAe?$AAo?$AA?5?$AAm?$AAe?$AAm?$AAo?$AAr?$AAy?$AA?5?$AAb?$AAe?$AAf?$AAo?$AAr?$AAe?$AA?5?$AAa?$AAf?$AAt?$AAe?$AAr?$AA?5?$AAs?$AAu?$AAr?$AAf?$AAa?$AAc@ 10002b38     lcdc_common_topaz_v1:DDLcdcSurf.obj
 0001:00001b9c       ??_C@_1CO@DPICPPM@?$AAG?$AAr?$AAa?$AAp?$AAh?$AAi?$AAc?$AAs?$AA?5?$AAe?$AAn?$AAg?$AAi?$AAn?$AAe?$AA?5?$AAb?$AAu?$AAs?$AAy?$AA?$AN?$AA?6?$AA?$AA@ 10002b9c     lcdc_common_topaz_v1:DDLcdcSurf.obj
 0001:00001bd0       ??_7MXDDLcdcSurf@@6B@      10002bd0     lcdc_common_topaz_v1:DDLcdcSurf.obj
 0001:00001ccc       ??_C@_1CG@JHDABJCF@?$AAM?$AAo?$AAu?$AAs?$AAe?$AAD?$AAe?$AAt?$AAa?$AAc?$AAh?$AAe?$AAd?$AAE?$AAv?$AAe?$AAn?$AAt?$AA?$AA@ 10002ccc     lcdc_common_topaz_v1:DDLcdcCursor.obj
 0001:00001cf4       ??_C@_1CG@NNBNONKD@?$AAM?$AAo?$AAu?$AAs?$AAe?$AAA?$AAt?$AAt?$AAa?$AAc?$AAh?$AAe?$AAd?$AAE?$AAv?$AAe?$AAn?$AAt?$AA?$AA@ 10002cf4     lcdc_common_topaz_v1:DDLcdcCursor.obj
 0001:00001dd8       ??_C@_1IA@JOAPHLGH@?$AAM?$AAX?$AAD?$AAD?$AAL?$AAc?$AAd?$AAc?$AA?5?$AAD?$AAr?$AAv?$AAE?$AAs?$AAc?$AAa?$AAp?$AAe?$AA?3?$AA?5?$AAI?$AAO?$AAC?$AAT?$AAL?$AA_?$AAP?$AAO?$AAW?$AAE?$AAR?$AA_@ 10002dd8     lcdc_common_topaz_v1:DDLcdcMisc.obj
 0001:00001e58       ??_C@_1HK@DHDJPOHA@?$AAM?$AAX?$AAD?$AAD?$AAL?$AAc?$AAd?$AAc?$AA?5?$AAD?$AAr?$AAv?$AAE?$AAs?$AAc?$AAa?$AAp?$AAe?$AA?3?$AA?5?$AA?$CF?$AAs?$AA?5?$AAI?$AAO?$AAC?$AAT?$AAL?$AA_?$AAP?$AAO?$AAW@ 10002e58     lcdc_common_topaz_v1:DDLcdcMisc.obj
 0001:00001ed8       ??_C@_1HE@LGFLNCAL@?$AAM?$AAX?$AAD?$AAD?$AAL?$AAc?$AAd?$AAc?$AA?5?$AAD?$AAr?$AAv?$AAE?$AAs?$AAc?$AAa?$AAp?$AAe?$AA?3?$AA?5?$AA?$CF?$AAs?$AA?5?$AAI?$AAO?$AAC?$AAT?$AAL?$AA_?$AAP?$AAO?$AAW@ 10002ed8     lcdc_common_topaz_v1:DDLcdcMisc.obj
 0001:00001f50       ??_C@_1FM@JPBPDABM@?$AAM?$AAX?$AAD?$AAD?$AAL?$AAc?$AAd?$AAc?$AA?5?$AAD?$AAr?$AAv?$AAE?$AAs?$AAc?$AAa?$AAp?$AAe?$AA?3?$AA?5?$AAI?$AAO?$AAC?$AAT?$AAL?$AA_?$AAP?$AAO?$AAW?$AAE?$AAR?$AA_@ 10002f50     lcdc_common_topaz_v1:DDLcdcMisc.obj
 0001:00001fac       ??_C@_1O@KPGHAGDD@?$AAf?$AAa?$AAi?$AAl?$AAe?$AAd?$AA?$AA@ 10002fac     lcdc_common_topaz_v1:DDLcdcMisc.obj
 0001:00001fbc       ??_C@_1BE@GCAFJAHI@?$AAs?$AAu?$AAc?$AAc?$AAe?$AAe?$AAd?$AAe?$AAd?$AA?$AA@ 10002fbc     lcdc_common_topaz_v1:DDLcdcMisc.obj
 0001:00001fd0       ??_C@_1JK@JEPAFNFO@?$AAM?$AAX?$AAD?$AAD?$AAL?$AAc?$AAd?$AAc?$AA?5?$AAD?$AAr?$AAv?$AAE?$AAs?$AAc?$AAa?$AAp?$AAe?$AA?3?$AA?5?$AAS?$AAe?$AAt?$AAP?$AAo?$AAw?$AAe?$AAr?$AAM?$AAa?$AAn?$AAa@ 10002fd0     lcdc_common_topaz_v1:DDLcdcMisc.obj
 0001:00002070       ??_C@_1GK@LJPBAHKJ@?$AAM?$AAX?$AAD?$AAD?$AAL?$AAc?$AAd?$AAc?$AA?5?$AAD?$AAr?$AAv?$AAE?$AAs?$AAc?$AAa?$AAp?$AAe?$AA?3?$AA?5?$AAB?$AAa?$AAc?$AAk?$AAL?$AAi?$AAg?$AAh?$AAt?$AA?5?$AAO?$AAN@ 10003070     lcdc_common_topaz_v1:DDLcdcMisc.obj
 0001:000020e0       ??_C@_1GA@LCMKHHMP@?$AAM?$AAX?$AAD?$AAD?$AAL?$AAc?$AAd?$AAc?$AA?5?$AAD?$AAr?$AAv?$AAE?$AAs?$AAc?$AAa?$AAp?$AAe?$AA?3?$AA?5?$AAR?$AAe?$AAq?$AAu?$AAe?$AAs?$AAt?$AAi?$AAn?$AAg?$AA?5?$AAP@ 100030e0     lcdc_common_topaz_v1:DDLcdcMisc.obj
 0001:00002140       ??_C@_1GM@OENAJDHD@?$AAM?$AAX?$AAD?$AAD?$AAL?$AAc?$AAd?$AAc?$AA?5?$AAD?$AAr?$AAv?$AAE?$AAs?$AAc?$AAa?$AAp?$AAe?$AA?3?$AA?5?$AAB?$AAa?$AAc?$AAk?$AAL?$AAi?$AAg?$AAh?$AAt?$AA?5?$AAO?$AAf@ 10003140     lcdc_common_topaz_v1:DDLcdcMisc.obj
 0001:000021b0       ??_C@_1GE@CLPJIBFD@?$AAM?$AAX?$AAD?$AAD?$AAL?$AAc?$AAd?$AAc?$AA?5?$AAD?$AAr?$AAv?$AAE?$AAs?$AAc?$AAa?$AAp?$AAe?$AA?3?$AA?5?$AAR?$AAe?$AAq?$AAu?$AAe?$AAs?$AAt?$AAi?$AAn?$AAg?$AA?5?$AAP@ 100031b0     lcdc_common_topaz_v1:DDLcdcMisc.obj
 0001:000022cc       ??_C@_1M@FIJHFMPA@?$AAA?$AAN?$AAG?$AAL?$AAE?$AA?$AA@ 100032cc     lcdc_common_topaz_v1:DDLcdcRotate.obj
 0001:000022d8       ??_C@_1CI@PNCEGBJC@?$AAS?$AAY?$AAS?$AAT?$AAE?$AAM?$AA?2?$AAG?$AAD?$AAI?$AA?2?$AAR?$AAO?$AAT?$AAA?$AAT?$AAI?$AAO?$AAN?$AA?$AA@ 100032d8     lcdc_common_topaz_v1:DDLcdcRotate.obj
 0001:000023b4       ??_C@_1DM@JKLIOIB@?$AAM?$AAX?$AAD?$AAD?$AAL?$AAc?$AAd?$AAc?$AA?5?$AAU?$AAp?$AAd?$AAa?$AAt?$AAe?$AAO?$AAv?$AAe?$AAr?$AAl?$AAa?$AAy?$AA?3?$AA?5?$AA?$CF?$AAs?$AA?$CB?$AA?$AN?$AA?6?$AA?$AA@ 100033b4     lcdc_common_topaz_v1:DDLcdcOverlay.obj
 0001:000023f0       ??_C@_1BG@GELEOFE@?$AAs?$AAu?$AAc?$AAc?$AAe?$AAs?$AAs?$AAf?$AAu?$AAl?$AA?$AA@ 100033f0     lcdc_common_topaz_v1:DDLcdcOverlay.obj
 0001:00002408       ??_C@_1EE@MPOCKEPP@?$AAE?$AAr?$AAr?$AAo?$AAr?$AA?3?$AA?5?$AAc?$AAa?$AAn?$AA?8?$AAt?$AA?5?$AAh?$AAa?$AAn?$AAd?$AAl?$AAe?$AA?5?$AAd?$AAe?$AAs?$AAt?$AA?5?$AAa?$AAl?$AAp?$AAh?$AAa?$AA?$CB?$AA?$AN@ 10003408     lcdc_common_topaz_v1:DDLcdcOverlay.obj
 0001:00002450       ??_C@_1FC@HAKFHIGF@?$AAE?$AAr?$AAr?$AAo?$AAr?$AA?3?$AA?5?$AAc?$AAa?$AAn?$AA?8?$AAt?$AA?5?$AAh?$AAa?$AAn?$AAd?$AAl?$AAe?$AA?5?$AAd?$AAe?$AAs?$AAt?$AA?5?$AAc?$AAo?$AAl?$AAo?$AAr?$AA?5?$AAk@ 10003450     lcdc_common_topaz_v1:DDLcdcOverlay.obj
 0001:000024a8       ??_C@_1HI@EBGEMEGB@?$AAM?$AAX?$AAD?$AAD?$AAL?$AAc?$AAd?$AAc?$AA?5?$AAU?$AAp?$AAd?$AAa?$AAt?$AAe?$AAO?$AAv?$AAe?$AAr?$AAl?$AAa?$AAy?$AA?3?$AA?5?$AAu?$AAp?$AAs?$AAi?$AAd?$AAe?$AA?9?$AAd@ 100034a8     lcdc_common_topaz_v1:DDLcdcOverlay.obj
 0001:00002520       ??_C@_1FO@OGPJNIA@?$AAO?$AAv?$AAe?$AAr?$AAl?$AAa?$AAy?$AA?5?$AAO?$AAP?$AA?3?$AA?5?$AAO?$AAv?$AAe?$AAr?$AAl?$AAa?$AAy?$AA?9?$AA?$DO?$AAC?$AAo?$AAl?$AAo?$AAr?$AAK?$AAe?$AAy?$AAM?$AAa?$AAs@ 10003520     lcdc_common_topaz_v1:DDLcdcOverlay.obj
 0001:00002580       ??_C@_1FG@GLADNDHJ@?$AAO?$AAv?$AAe?$AAr?$AAl?$AAa?$AAy?$AA?5?$AAO?$AAP?$AA?3?$AA?5?$AAO?$AAv?$AAe?$AAr?$AAl?$AAa?$AAy?$AA?9?$AA?$DO?$AAi?$AAs?$AAU?$AAp?$AAs?$AAi?$AAd?$AAe?$AAD?$AAo?$AAw@ 10003580     lcdc_common_topaz_v1:DDLcdcOverlay.obj
 0001:000025d8       ??_C@_1FG@PLIIEE@?$AAO?$AAv?$AAe?$AAr?$AAl?$AAa?$AAy?$AA?5?$AAO?$AAP?$AA?3?$AA?5?$AAO?$AAv?$AAe?$AAr?$AAl?$AAa?$AAy?$AA?9?$AA?$DO?$AAT?$AAr?$AAa?$AAn?$AAs?$AAp?$AAa?$AAr?$AAe?$AAn?$AAc@ 100035d8     lcdc_common_topaz_v1:DDLcdcOverlay.obj
 0001:00002630       ??_C@_1FG@FIGKFPAN@?$AAO?$AAv?$AAe?$AAr?$AAl?$AAa?$AAy?$AA?5?$AAO?$AAP?$AA?3?$AA?5?$AAO?$AAv?$AAe?$AAr?$AAl?$AAa?$AAy?$AA?9?$AA?$DO?$AAY?$AAO?$AAf?$AAf?$AAs?$AAe?$AAt?$AA?5?$AA?5?$AA?5?$AA?5@ 10003630     lcdc_common_topaz_v1:DDLcdcOverlay.obj
 0001:00002688       ??_C@_1FG@HCECGHGP@?$AAO?$AAv?$AAe?$AAr?$AAl?$AAa?$AAy?$AA?5?$AAO?$AAP?$AA?3?$AA?5?$AAO?$AAv?$AAe?$AAr?$AAl?$AAa?$AAy?$AA?9?$AA?$DO?$AAX?$AAO?$AAf?$AAf?$AAs?$AAe?$AAt?$AA?5?$AA?5?$AA?5?$AA?5@ 10003688     lcdc_common_topaz_v1:DDLcdcOverlay.obj
 0001:000026e0       ??_C@_1FG@FLNGDNOL@?$AAO?$AAv?$AAe?$AAr?$AAl?$AAa?$AAy?$AA?5?$AAO?$AAP?$AA?3?$AA?5?$AAO?$AAv?$AAe?$AAr?$AAl?$AAa?$AAy?$AA?9?$AA?$DO?$AAL?$AAi?$AAn?$AAe?$AAS?$AAt?$AAr?$AAi?$AAd?$AAe?$AA?5@ 100036e0     lcdc_common_topaz_v1:DDLcdcOverlay.obj
 0001:00002738       ??_C@_1FG@JKCOJDBP@?$AAO?$AAv?$AAe?$AAr?$AAl?$AAa?$AAy?$AA?5?$AAO?$AAP?$AA?3?$AA?5?$AAO?$AAv?$AAe?$AAr?$AAl?$AAa?$AAy?$AA?9?$AA?$DO?$AAH?$AAe?$AAi?$AAg?$AAh?$AAt?$AAH?$AAw?$AA?5?$AA?5?$AA?5@ 10003738     lcdc_common_topaz_v1:DDLcdcOverlay.obj
 0001:00002790       ??_C@_1FG@LGABOKGH@?$AAO?$AAv?$AAe?$AAr?$AAl?$AAa?$AAy?$AA?5?$AAO?$AAP?$AA?3?$AA?5?$AAO?$AAv?$AAe?$AAr?$AAl?$AAa?$AAy?$AA?9?$AA?$DO?$AAW?$AAi?$AAd?$AAt?$AAh?$AAH?$AAw?$AA?5?$AA?5?$AA?5?$AA?5@ 10003790     lcdc_common_topaz_v1:DDLcdcOverlay.obj
 0001:000027e8       ??_C@_1FG@OLOCKCEO@?$AAO?$AAv?$AAe?$AAr?$AAl?$AAa?$AAy?$AA?5?$AAO?$AAP?$AA?3?$AA?5?$AAO?$AAv?$AAe?$AAr?$AAl?$AAa?$AAy?$AA?9?$AA?$DO?$AAH?$AAe?$AAi?$AAg?$AAh?$AAt?$AA?5?$AA?5?$AA?5?$AA?5?$AA?5@ 100037e8     lcdc_common_topaz_v1:DDLcdcOverlay.obj
 0001:00002840       ??_C@_1FG@EEHPPHIE@?$AAO?$AAv?$AAe?$AAr?$AAl?$AAa?$AAy?$AA?5?$AAO?$AAP?$AA?3?$AA?5?$AAO?$AAv?$AAe?$AAr?$AAl?$AAa?$AAy?$AA?9?$AA?$DO?$AAW?$AAi?$AAd?$AAt?$AAh?$AA?5?$AA?5?$AA?5?$AA?5?$AA?5?$AA?5@ 10003840     lcdc_common_topaz_v1:DDLcdcOverlay.obj
 0001:00002898       ??_C@_1FO@NBIGCGMH@?$AAO?$AAv?$AAe?$AAr?$AAl?$AAa?$AAy?$AA?5?$AAO?$AAP?$AA?3?$AA?5?$AAO?$AAv?$AAe?$AAr?$AAl?$AAa?$AAy?$AA?9?$AA?$DO?$AAn?$AAB?$AAu?$AAf?$AAP?$AAh?$AAy?$AAs?$AAi?$AAc?$AAa@ 10003898     lcdc_common_topaz_v1:DDLcdcOverlay.obj
 0001:000028f8       ??_C@_1GC@HCJIPCIC@?$AAO?$AAv?$AAe?$AAr?$AAl?$AAa?$AAy?$AA?5?$AAO?$AAP?$AA?3?$AA?5?$AAO?$AAv?$AAe?$AAr?$AAl?$AAa?$AAy?$AA?9?$AA?$DO?$AAi?$AAs?$AAG?$AAr?$AAa?$AAp?$AAh?$AAi?$AAc?$AAW?$AAi@ 100038f8     lcdc_common_topaz_v1:DDLcdcOverlay.obj
 0001:0000295c       ??_C@_1M@HCOOECOK@?$AAF?$AAA?$AAL?$AAS?$AAE?$AA?$AA@ 1000395c     lcdc_common_topaz_v1:DDLcdcOverlay.obj
 0001:00002968       ??_C@_19ELAAHEEL@?$AAT?$AAR?$AAU?$AAE?$AA?$AA@ 10003968     lcdc_common_topaz_v1:DDLcdcOverlay.obj
 0001:00002978       ??_C@_1KG@OJHGOKIK@?$AAM?$AAX?$AAD?$AAD?$AAL?$AAc?$AAd?$AAc?$AA?5?$AAU?$AAp?$AAd?$AAa?$AAt?$AAe?$AAO?$AAv?$AAe?$AAr?$AAl?$AAa?$AAy?$AA?3?$AA?5?$AAw?$AAr?$AAo?$AAn?$AAg?$AA?5?$AAp?$AAa@ 10003978     lcdc_common_topaz_v1:DDLcdcOverlay.obj
 0001:00002a20       ??_C@_1DC@EMHGNEAI@?$AAM?$AAX?$AAD?$AAD?$AAL?$AAc?$AAd?$AAc?$AA?3?$AA?3?$AAO?$AAV?$AAE?$AAR?$AAL?$AAA?$AAY?$AA?5?$AAS?$AAH?$AAO?$AAW?$AA?$AN?$AA?6?$AA?$AA@ 10003a20     lcdc_common_topaz_v1:DDLcdcOverlay.obj
 0001:00002a58       ??_C@_1FA@PKOCDHGG@?$AAE?$AAr?$AAr?$AAo?$AAr?$AA?3?$AA?5?$AAO?$AAt?$AAh?$AAe?$AAr?$AA?5?$AAo?$AAv?$AAe?$AAr?$AAl?$AAa?$AAy?$AA?5?$AAa?$AAl?$AAr?$AAe?$AAa?$AAd?$AAy?$AA?5?$AAv?$AAi?$AAs@ 10003a58     lcdc_common_topaz_v1:DDLcdcOverlay.obj
 0001:00002aa8       ??_C@_1EC@FNBJLOCL@?$AAM?$AAX?$AAD?$AAD?$AAL?$AAc?$AAd?$AAc?$AA?3?$AA?3?$AAO?$AAV?$AAE?$AAR?$AAL?$AAA?$AAY?$AA?5?$AAS?$AAH?$AAO?$AAW?$AA?5?$AAR?$AAE?$AAQ?$AAU?$AAE?$AAS?$AAT?$AA?$AN?$AA?6@ 10003aa8     lcdc_common_topaz_v1:DDLcdcOverlay.obj
 0001:00002aec       ??_C@_1DE@OGDMHGPI@?$AAM?$AAX?$AAD?$AAD?$AAL?$AAc?$AAd?$AAc?$AA?3?$AA?3?$AAO?$AAV?$AAE?$AAR?$AAL?$AAA?$AAY?$AA?5?$AAH?$AAI?$AAD?$AAE?$AA?$CB?$AA?$AN?$AA?6?$AA?$AA@ 10003aec     lcdc_common_topaz_v1:DDLcdcOverlay.obj
 0001:00002b20       ??_C@_1EC@FBLJDHFL@?$AAM?$AAX?$AAD?$AAD?$AAL?$AAc?$AAd?$AAc?$AA?3?$AA?3?$AAO?$AAV?$AAE?$AAR?$AAL?$AAA?$AAY?$AA?5?$AAH?$AAI?$AAD?$AAE?$AA?5?$AAR?$AAE?$AAQ?$AAU?$AAE?$AAS?$AAT?$AA?$AN?$AA?6@ 10003b20     lcdc_common_topaz_v1:DDLcdcOverlay.obj
 0001:00002b68       ??_C@_1IG@GNENBGG@?$AAM?$AAX?$AAD?$AAD?$AAL?$AAc?$AAd?$AAc?$AA?5?$AAS?$AAe?$AAt?$AAO?$AAv?$AAe?$AAr?$AAl?$AAa?$AAy?$AAP?$AAo?$AAs?$AAi?$AAt?$AAi?$AAo?$AAn?$AA?3?$AA?5?$AAe?$AAr?$AAr@ 10003b68     lcdc_common_topaz_v1:DDLcdcOverlay.obj
 0001:00002bf0       ??_C@_1FA@OHNDIOK@?$AAM?$AAX?$AAD?$AAD?$AAL?$AAc?$AAd?$AAc?$AA?5?$AAE?$AAn?$AAa?$AAb?$AAl?$AAe?$AAO?$AAv?$AAe?$AAr?$AAl?$AAa?$AAy?$AA?3?$AA?5?$AAr?$AAe?$AAs?$AAu?$AAl?$AAt?$AA?5?$AA0@ 10003bf0     lcdc_common_topaz_v1:DDLcdcOverlay.obj
 0001:00002c40       ??_C@_1GO@KPMPDPLL@?$AAM?$AAX?$AAD?$AAD?$AAL?$AAc?$AAd?$AAc?$AA?5?$AAE?$AAn?$AAa?$AAb?$AAl?$AAe?$AAO?$AAv?$AAe?$AAr?$AAl?$AAa?$AAy?$AA?3?$AA?5?$AAL?$AAC?$AAD?$AAC?$AA?5?$AAh?$AAw?$AA?5@ 10003c40     lcdc_common_topaz_v1:DDLcdcOverlay.obj
 0001:00002cb0       ??_C@_1II@NIOCPCAN@?$AAM?$AAX?$AAD?$AAD?$AAL?$AAc?$AAd?$AAc?$AA?5?$AAS?$AAe?$AAt?$AAM?$AAo?$AAd?$AAe?$AAH?$AAa?$AAr?$AAd?$AAw?$AAa?$AAr?$AAe?$AA?3?$AA?5?$AAc?$AAa?$AAn?$AA?5?$AAn?$AAo@ 10003cb0     lcdc_common_topaz_v1:DDLcdcOverlay.obj
 0001:00002d38       ??_C@_1DI@NPPPJHHK@?$AAS?$AAe?$AAt?$AAA?$AAt?$AAt?$AAr?$AAi?$AAb?$AAu?$AAt?$AAe?$AAE?$AAx?$AA?$CI?$AA?$CJ?$AA?5?$AAf?$AAa?$AAi?$AAl?$AAe?$AAd?$AA?$CB?$AA?5?$AA?$AN?$AA?6?$AA?$AA@ 10003d38     lcdc_common_topaz_v1:DDLcdcEscape.obj
 0001:00002d70       ??_C@_1LG@NNDHFDLG@?$AAc?$AA?3?$AA?2?$AAw?$AAi?$AAn?$AAc?$AAe?$AAr?$AAo?$AAo?$AAt?$AAs?$AA?2?$AAt?$AAo?$AAp?$AAa?$AAz?$AA?2?$AAw?$AAi?$AAn?$AAc?$AAe?$AA7?$AA0?$AA0?$AA?2?$AAp?$AAl?$AAa@ 10003d70     lcdc_common_topaz_v1:DDLcdcEscape.obj
 0001:00002e28       ??_C@_1GI@ONMNDGBB@?$AAS?$AAe?$AAt?$AAA?$AAt?$AAt?$AAr?$AAi?$AAb?$AAu?$AAt?$AAe?$AAE?$AAx?$AA?3?$AA?5?$AAA?$AAD?$AAD?$AA?$DN?$AA0?$AAx?$AA?$CF?$AAx?$AA?0?$AA?5?$AAS?$AAI?$AAZ?$AAE?$AA?$DN?$AA0@ 10003e28     lcdc_common_topaz_v1:DDLcdcEscape.obj
 0001:00002f44       ??_C@_1CM@JGLFDINH@?$AAL?$AAe?$AAa?$AAv?$AAi?$AAn?$AAg?$AA?5?$AAf?$AAu?$AAn?$AAc?$AAt?$AAi?$AAo?$AAn?$AA?5?$AA?$CF?$AAs?$AA?$AN?$AA?6?$AA?$AA@ 10003f44     ddgpe:ddhinit.obj
 0001:00002f70       ??_C@_1CO@ENKLBDPK@?$AAE?$AAn?$AAt?$AAe?$AAr?$AAi?$AAn?$AAg?$AA?5?$AAf?$AAu?$AAn?$AAc?$AAt?$AAi?$AAo?$AAn?$AA?5?$AA?$CF?$AAs?$AA?$AN?$AA?6?$AA?$AA@ 10003f70     ddgpe:ddhinit.obj
 0001:00002fa0       ??_C@_1BA@MLJOMGFD@?$AAH?$AAA?$AAL?$AAI?$AAn?$AAi?$AAt?$AA?$AA@ 10003fa0     ddgpe:ddhinit.obj
 0001:00002fb0       ??_C@_1BM@FBKBLPHO@?$AAU?$AAp?$AAd?$AAa?$AAt?$AAe?$AAH?$AAA?$AAL?$AAI?$AAn?$AAi?$AAt?$AA?$AA@ 10003fb0     ddgpe:ddhinit.obj
 0001:00003088       ?EDDGPEPixelFormatToEGPEFormat@@3QBW4EGPEFormat@@B 10004088     ddgpe:ddgpe.obj
 0001:000030d4       ?EGPEFormatToEDDGPEPixelFormat@@3QBW4EDDGPEPixelFormat@@B 100040d4     ddgpe:ddgpe.obj
 0001:00003100       ??_7DDGPE@@6B@             10004100     ddgpe:ddgpe.obj
 0001:000031e8       ??_C@_1HC@FBEEEDMN@?$AAA?$AAl?$AAl?$AAo?$AAc?$AAS?$AAu?$AAr?$AAf?$AAa?$AAc?$AAe?$AA?$CI?$AAE?$AAD?$AAD?$AAG?$AAP?$AAE?$AAP?$AAi?$AAx?$AAe?$AAl?$AAF?$AAo?$AAr?$AAm?$AAa?$AAt?$AA?$CJ?$AA?5@ 100041e8     ddgpe:ddgpe.obj
 0001:00003260       ??_C@_1HK@KEGJHKLC@?$AAA?$AAl?$AAl?$AAo?$AAc?$AAS?$AAu?$AAr?$AAf?$AAa?$AAc?$AAe?$AA?$CI?$AAD?$AAD?$AAG?$AAP?$AAE?$AAA?$AAl?$AAl?$AAo?$AAc?$AAS?$AAu?$AAr?$AAf?$AAa?$AAc?$AAe?$AAD?$AAa@ 10004260     ddgpe:ddgpe.obj
 0001:000032e0       ??_C@_1GM@GIKALOGL@?$AAG?$AAP?$AAE?$AA_?$AAA?$AAl?$AAl?$AAo?$AAc?$AAV?$AAi?$AAd?$AAe?$AAo?$AAS?$AAu?$AAr?$AAf?$AAa?$AAc?$AAe?$AA?3?$AA?5?$AAo?$AAf?$AAf?$AAs?$AAe?$AAt?$AA?5?$AAi?$AAn@ 100042e0     ddgpe:ddgpe.obj
 0001:00003350       ??_C@_1GI@DDHLBIAG@?$AAD?$AAD?$AAG?$AAP?$AAE?$AA?3?$AA?5?$AAO?$AAu?$AAt?$AA?5?$AAo?$AAf?$AA?5?$AAm?$AAe?$AAm?$AAo?$AAr?$AAy?$AA?5?$AAw?$AAh?$AAe?$AAn?$AA?5?$AAc?$AAr?$AAe?$AAa?$AAt?$AAi@ 10004350     ddgpe:ddgpe.obj
 0001:000033b8       ??_C@_1GA@GJFBJMED@?$AAD?$AAe?$AAt?$AAe?$AAc?$AAt?$AAe?$AAd?$AA?5?$AAs?$AAu?$AAr?$AAf?$AAa?$AAc?$AAe?$AA?5?$AAp?$AAi?$AAx?$AAe?$AAl?$AAF?$AAo?$AAr?$AAm?$AAa?$AAt?$AA?0?$AA?5?$AAf?$AAo@ 100043b8     ddgpe:ddgpe.obj
 0001:00003418       ??_C@_1DA@MIPLHNFE@?$AA1?$AA5?$AA5?$AA5?$AA?5?$AAs?$AAu?$AAr?$AAf?$AAa?$AAc?$AAe?$AA?5?$AAd?$AAe?$AAt?$AAe?$AAc?$AAt?$AAe?$AAd?$AA?$AN?$AA?6?$AA?$AA@ 10004418     ddgpe:ddgpe.obj
 0001:00003448       ??_C@_1CO@MMMACBJG@?$AA5?$AA6?$AA5?$AA?5?$AAs?$AAu?$AAr?$AAf?$AAa?$AAc?$AAe?$AA?5?$AAd?$AAe?$AAt?$AAe?$AAc?$AAt?$AAe?$AAd?$AA?$AN?$AA?6?$AA?$AA@ 10004448     ddgpe:ddgpe.obj
 0001:00003478       ??_C@_1FI@FCNOILPG@?$AAD?$AAe?$AAt?$AAe?$AAc?$AAt?$AAM?$AAo?$AAd?$AAe?$AA?3?$AA?5?$AAI?$AAn?$AAf?$AAo?$AA?5?$AAo?$AAn?$AA?5?$AAm?$AAo?$AAd?$AAe?$AA?5?$AA?$CF?$AAd?$AA?5?$AAF?$AAA?$AAI?$AAL@ 10004478     ddgpe:ddgpe.obj
 0001:000034d0       ??_C@_1DA@NGJFBDPF@?$AAD?$AAe?$AAt?$AAe?$AAc?$AAt?$AAM?$AAo?$AAd?$AAe?$AA?3?$AA?5?$AAR?$AAe?$AAq?$AAu?$AAe?$AAs?$AAt?$AAe?$AAd?$AA?$AN?$AA?6?$AA?$AA@ 100044d0     ddgpe:ddgpe.obj
 0001:00003500       ??_C@_1DG@HPLEAAFB@?$AA?5?$AA?5?$AAm?$AAo?$AAd?$AAe?$AA?5?$AAp?$AAi?$AAx?$AAe?$AAl?$AA?5?$AAf?$AAo?$AAr?$AAm?$AAa?$AAt?$AA?5?$AA?$DN?$AA?5?$AA?$CF?$AAd?$AA?$AN?$AA?6?$AA?$AA@ 10004500     ddgpe:ddgpe.obj
 0001:00003538       ??_C@_1DG@JHKBDNGD@?$AA?5?$AA?5?$AAm?$AAo?$AAd?$AAe?$AA?5?$AAf?$AAo?$AAr?$AAm?$AAa?$AAt?$AA?5?$AA?5?$AA?5?$AA?5?$AA?5?$AA?5?$AA?5?$AA?$DN?$AA?5?$AA?$CF?$AAd?$AA?$AN?$AA?6?$AA?$AA@ 10004538     ddgpe:ddgpe.obj
 0001:00003570       ??_C@_1DG@JOACGOHA@?$AA?5?$AA?5?$AAm?$AAo?$AAd?$AAe?$AA?5?$AAh?$AAe?$AAi?$AAg?$AAh?$AAt?$AA?5?$AA?5?$AA?5?$AA?5?$AA?5?$AA?5?$AA?5?$AA?$DN?$AA?5?$AA?$CF?$AAd?$AA?$AN?$AA?6?$AA?$AA@ 10004570     ddgpe:ddgpe.obj
 0001:000035a8       ??_C@_1DG@KGEIJEF@?$AA?5?$AA?5?$AAm?$AAo?$AAd?$AAe?$AA?5?$AAw?$AAi?$AAd?$AAt?$AAh?$AA?5?$AA?5?$AA?5?$AA?5?$AA?5?$AA?5?$AA?5?$AA?5?$AA?$DN?$AA?5?$AA?$CF?$AAd?$AA?$AN?$AA?6?$AA?$AA@ 100045a8     ddgpe:ddgpe.obj
 0001:000035e0       ??_C@_1DA@EFKDLIKI@?$AAD?$AAe?$AAt?$AAe?$AAc?$AAt?$AAM?$AAo?$AAd?$AAe?$AA?3?$AA?5?$AAM?$AAo?$AAd?$AAe?$AA?5?$AAI?$AAn?$AAf?$AAo?$AA?$AN?$AA?6?$AA?$AA@ 100045e0     ddgpe:ddgpe.obj
 0001:00003610       ??_C@_1EO@MBMICCC@?$AAD?$AAe?$AAt?$AAe?$AAc?$AAt?$AAM?$AAo?$AAd?$AAe?$AA?3?$AA?5?$AAG?$AAe?$AAt?$AAt?$AAi?$AAn?$AAg?$AA?5?$AAi?$AAn?$AAf?$AAo?$AA?5?$AAo?$AAn?$AA?5?$AAm?$AAo?$AAd?$AAe@ 10004610     ddgpe:ddgpe.obj
 0001:00003660       ??_C@_1EG@JNDAGKAC@?$AAD?$AAe?$AAt?$AAe?$AAc?$AAt?$AAM?$AAo?$AAd?$AAe?$AA?3?$AA?5?$AAT?$AAh?$AAe?$AAr?$AAe?$AA?5?$AAa?$AAr?$AAe?$AA?5?$AA0?$AAx?$AA?$CF?$AAd?$AA?5?$AAm?$AAo?$AAd?$AAe?$AAs@ 10004660     ddgpe:ddgpe.obj
 0001:000036a8       ??_C@_1EG@HJHLFGIJ@?$AAD?$AAD?$AAG?$AAP?$AAE?$AA?3?$AA?3?$AAG?$AAe?$AAt?$AAM?$AAo?$AAd?$AAe?$AAI?$AAn?$AAf?$AAo?$AAE?$AAx?$AA?5?$AAU?$AAn?$AAs?$AAu?$AAp?$AAp?$AAo?$AAr?$AAt?$AAe?$AAd@ 100046a8     ddgpe:ddgpe.obj
 0001:000036f0       ??_C@_1FK@OHOGDCHC@?$AAD?$AAD?$AAG?$AAP?$AAE?$AA?3?$AA?3?$AAS?$AAe?$AAt?$AAM?$AAo?$AAd?$AAe?$AA?$CI?$AA?$CJ?$AA?5?$AAi?$AAs?$AA?5?$AAN?$AAo?$AAt?$AA?5?$AAI?$AAm?$AAp?$AAl?$AAe?$AAm?$AAe?$AAn@ 100046f0     ddgpe:ddgpe.obj
 0001:00003808       ??_C@_1KE@OJAJEPGI@?$AAS?$AAu?$AAr?$AAf?$AAa?$AAc?$AAe?$AAH?$AAe?$AAa?$AAp?$AA?3?$AA?3?$AAS?$AAu?$AAr?$AAf?$AAa?$AAc?$AAe?$AAH?$AAe?$AAa?$AAp?$AA?5?$AAs?$AAi?$AAz?$AAe?$AA?5?$AA?$CF?$AAd@ 10004808     ddgpe:surfheap.obj
 0001:000038ac       ??_C@_1CK@LIOJGCDK@?$AAD?$AAe?$AAl?$AAe?$AAt?$AAi?$AAn?$AAg?$AA?5?$AAn?$AAo?$AAd?$AAe?$AA?5?$AAo?$AAn?$AAl?$AAy?$AA?$AN?$AA?6?$AA?$AA@ 100048ac     ddgpe:surfheap.obj
 0001:000038d8       ??_C@_1CC@KCHFJKML@?$AAD?$AAe?$AAl?$AAe?$AAt?$AAi?$AAn?$AAg?$AA?5?$AAh?$AAe?$AAa?$AAp?$AA?$CB?$AA?$AN?$AA?6?$AA?$AA@ 100048d8     ddgpe:surfheap.obj
 0001:00003900       ??_C@_1FK@KIBLCHKL@?$AAS?$AAu?$AAr?$AAf?$AAa?$AAc?$AAe?$AAH?$AAe?$AAa?$AAp?$AA?3?$AA?3?$AA?$HO?$AAS?$AAu?$AAr?$AAf?$AAa?$AAc?$AAe?$AAH?$AAe?$AAa?$AAp?$AA?5?$AA0?$AAx?$AA?$CF?$AA0?$AA8?$AAx@ 10004900     ddgpe:surfheap.obj
 0001:00003960       ??_C@_1GE@CINLEPBF@?$AAM?$AAa?$AAr?$AAk?$AAi?$AAn?$AAg?$AA?5?$AAn?$AAo?$AAd?$AAe?$AA?5?$AAa?$AAt?$AA?5?$AA0?$AAx?$AA?$CF?$AA0?$AA8?$AAx?$AA?5?$AAa?$AAs?$AA?5?$AAu?$AAs?$AAe?$AAd?$AA?5?$AA?$CI@ 10004960     ddgpe:surfheap.obj
 0001:000039c4       ??_C@_1DM@NHHILNKE@?$AAF?$AAa?$AAi?$AAl?$AAe?$AAd?$AA?5?$AAt?$AAo?$AA?5?$AAa?$AAl?$AAl?$AAo?$AAc?$AAa?$AAt?$AAe?$AA?5?$AAn?$AAe?$AAw?$AA?5?$AAn?$AAo?$AAd?$AAe?$AA?$AN?$AA?6?$AA?$AA@ 100049c4     ddgpe:surfheap.obj
 0001:00003a00       ??_C@_1EG@GAMEKDIE@?$AAS?$AAp?$AAl?$AAi?$AAt?$AAt?$AAi?$AAn?$AAg?$AA?5?$AA?$CF?$AAd?$AA?5?$AAb?$AAy?$AAt?$AAe?$AA?5?$AAn?$AAo?$AAd?$AAe?$AA?5?$AAa?$AAt?$AA?5?$AA0?$AAx?$AA?$CF?$AA0?$AA8?$AAx@ 10004a00     ddgpe:surfheap.obj
 0001:00003a48       ??_C@_1DC@OAGNOIOB@?$AAS?$AAu?$AAr?$AAf?$AAa?$AAc?$AAe?$AAH?$AAe?$AAa?$AAp?$AA?3?$AA?3?$AAA?$AAl?$AAl?$AAo?$AAc?$AA?$CI?$AA?$CF?$AAd?$AA?$CJ?$AA?$AN?$AA?6?$AA?$AA@ 10004a48     ddgpe:surfheap.obj
 0001:00003a80       ??_C@_1HO@BKIBPFEO@?$AAS?$AAu?$AAr?$AAf?$AAa?$AAc?$AAe?$AAH?$AAe?$AAa?$AAp?$AA?3?$AA?3?$AAF?$AAr?$AAe?$AAe?$AA?5?$AA?9?$AA?5?$AAm?$AAe?$AAr?$AAg?$AAi?$AAn?$AAg?$AA?5?$AA?$CF?$AA0?$AA8?$AAx@ 10004a80     ddgpe:surfheap.obj
 0001:00003b00       ??_C@_1HO@OHDFKGKH@?$AAS?$AAu?$AAr?$AAf?$AAa?$AAc?$AAe?$AAH?$AAe?$AAa?$AAp?$AA?3?$AA?3?$AAF?$AAr?$AAe?$AAe?$AA?5?$AA?9?$AA?5?$AAm?$AAe?$AAr?$AAg?$AAi?$AAn?$AAg?$AA?5?$AAn?$AAo?$AAd?$AAe@ 10004b00     ddgpe:surfheap.obj
 0001:00003b80       ??_C@_1EK@NENKGICN@?$AAS?$AAu?$AAr?$AAf?$AAa?$AAc?$AAe?$AAH?$AAe?$AAa?$AAp?$AA?3?$AA?3?$AAF?$AAr?$AAe?$AAe?$AA?5?$AA0?$AAx?$AA?$CF?$AA0?$AA8?$AAx?$AA?5?$AA?$CI?$AAs?$AAi?$AAz?$AAe?$AA?$DN?$AA?$CF@ 10004b80     ddgpe:surfheap.obj
 0001:00003c88       ??_7DDGPESurf@@6B@         10004c88     ddgpe:ddgpesurf.obj
 0001:00003cd0       ??_7GPESurf@@6B@           10004cd0     ddgpe:ddgpesurf.obj
 0001:00003cd8       ??_C@_1IA@EDILFOMD@?$AAD?$AAD?$AAG?$AAP?$AAE?$AA?3?$AA?5?$AAI?$AA?5?$AAh?$AAa?$AAv?$AAe?$AA?5?$AAa?$AAl?$AAl?$AAo?$AAc?$AAa?$AAt?$AAe?$AAd?$AA?5?$AAs?$AAy?$AAs?$AAt?$AAe?$AAm?$AA?5?$AAm@ 10004cd8     ddgpe:ddgpesurf.obj
 0001:00003d58       ??_C@_1GO@CMFDBJB@?$AAD?$AAD?$AAG?$AAP?$AAE?$AA?3?$AA?5?$AAF?$AAr?$AAe?$AAe?$AAi?$AAn?$AAg?$AA?5?$AAs?$AAy?$AAs?$AAt?$AAe?$AAm?$AA?5?$AAm?$AAe?$AAm?$AAo?$AAr?$AAy?$AA?5?$AAs?$AAu?$AAr@ 10004d58     ddgpe:ddgpesurf.obj
 0001:00003dc8       g_NullBlendFunction        10004dc8     gpe:ddi_if.obj
 0001:00003e4c       ??_C@_1DE@FAMIGPCK@?$AAL?$AAe?$AAa?$AAv?$AAi?$AAn?$AAg?$AA?5?$AAD?$AAr?$AAv?$AAE?$AAn?$AAa?$AAb?$AAl?$AAe?$AAD?$AAr?$AAi?$AAv?$AAe?$AAr?$AA?$AN?$AA?6?$AA?$AA@ 10004e4c     gpe:ddi_if.obj
 0001:00003e80       ??_C@_1DG@DIPIFIGI@?$AAE?$AAn?$AAt?$AAe?$AAr?$AAi?$AAn?$AAg?$AA?5?$AAD?$AAr?$AAv?$AAE?$AAn?$AAa?$AAb?$AAl?$AAe?$AAD?$AAr?$AAi?$AAv?$AAe?$AAr?$AA?$AN?$AA?6?$AA?$AA@ 10004e80     gpe:ddi_if.obj
 0001:00003eb8       ??_C@_1DG@OHECPOKD@?$AAL?$AAe?$AAa?$AAv?$AAi?$AAn?$AAg?$AA?5?$AAD?$AAr?$AAv?$AAD?$AAi?$AAs?$AAa?$AAb?$AAl?$AAe?$AAD?$AAr?$AAi?$AAv?$AAe?$AAr?$AA?$AN?$AA?6?$AA?$AA@ 10004eb8     gpe:ddi_if.obj
 0001:00003ef0       ??_C@_1DI@JNLABOBL@?$AAE?$AAn?$AAt?$AAe?$AAr?$AAi?$AAn?$AAg?$AA?5?$AAD?$AAr?$AAv?$AAD?$AAi?$AAs?$AAa?$AAb?$AAl?$AAe?$AAD?$AAr?$AAi?$AAv?$AAe?$AAr?$AA?$AN?$AA?6?$AA?$AA@ 10004ef0     gpe:ddi_if.obj
 0001:00003f28       ??_C@_1DC@GILMKGDL@?$AAL?$AAe?$AAa?$AAv?$AAi?$AAn?$AAg?$AA?5?$AAD?$AAr?$AAv?$AAD?$AAi?$AAs?$AAa?$AAb?$AAl?$AAe?$AAP?$AAD?$AAE?$AAV?$AA?$AN?$AA?6?$AA?$AA@ 10004f28     gpe:ddi_if.obj
 0001:00003f5c       ??_C@_1BA@LEPJIIOK@?$AAU?$AAn?$AAk?$AAn?$AAo?$AAw?$AAn?$AA?$AA@ 10004f5c     gpe:ddi_if.obj
 0001:00003f70       ??_C@_1HO@MDFFNBNO@?$AAd?$AA?3?$AA?2?$AAc?$AAh?$AAe?$AAl?$AAa?$AAn?$AAr?$AAt?$AAm?$AA2?$AA?2?$AAp?$AAu?$AAb?$AAl?$AAi?$AAc?$AA?2?$AAc?$AAo?$AAm?$AAm?$AAo?$AAn?$AA?2?$AAo?$AAa?$AAk?$AA?2@ 10004f70     gpe:ddi_if.obj
 0001:00003ff0       ??_C@_1DE@FEIFFELL@?$AAE?$AAn?$AAt?$AAe?$AAr?$AAi?$AAn?$AAg?$AA?5?$AAD?$AAr?$AAv?$AAD?$AAi?$AAs?$AAa?$AAb?$AAl?$AAe?$AAP?$AAD?$AAE?$AAV?$AA?$AN?$AA?6?$AA?$AA@ 10004ff0     gpe:ddi_if.obj
 0001:00004024       ??_C@_1DI@FPBBEDJF@?$AAL?$AAe?$AAa?$AAv?$AAi?$AAn?$AAg?$AA?5?$AAD?$AAr?$AAv?$AAD?$AAi?$AAs?$AAa?$AAb?$AAl?$AAe?$AAS?$AAu?$AAr?$AAf?$AAa?$AAc?$AAe?$AA?$AN?$AA?6?$AA?$AA@ 10005024     gpe:ddi_if.obj
 0001:0000405c       ??_C@_1DK@NDAHPPKP@?$AAE?$AAn?$AAt?$AAe?$AAr?$AAi?$AAn?$AAg?$AA?5?$AAD?$AAr?$AAv?$AAD?$AAi?$AAs?$AAa?$AAb?$AAl?$AAe?$AAS?$AAu?$AAr?$AAf?$AAa?$AAc?$AAe?$AA?$AN?$AA?6?$AA?$AA@ 1000505c     gpe:ddi_if.obj
 0001:00004098       ??_C@_1DG@DCFIHEMP@?$AAL?$AAe?$AAa?$AAv?$AAi?$AAn?$AAg?$AA?5?$AAD?$AAr?$AAv?$AAE?$AAn?$AAa?$AAb?$AAl?$AAe?$AAS?$AAu?$AAr?$AAf?$AAa?$AAc?$AAe?$AA?$AN?$AA?6?$AA?$AA@ 10005098     gpe:ddi_if.obj
 0001:000040d0       ??_C@_1EE@IPIBAOIA@?$AAF?$AAo?$AAr?$AAm?$AAa?$AAt?$AA?5?$AAo?$AAf?$AA?5?$AAp?$AAr?$AAi?$AAm?$AAa?$AAr?$AAy?$AA?5?$AAs?$AAu?$AAr?$AAf?$AAa?$AAc?$AAe?$AA?5?$AAi?$AAs?$AA?5?$AA?$CF?$AAd?$AA?$AN@ 100050d0     gpe:ddi_if.obj
 0001:00004114       ??_C@_1DO@FOHDIFLJ@?$AAP?$AAr?$AAi?$AAm?$AAa?$AAr?$AAy?$AA?5?$AAs?$AAu?$AAr?$AAf?$AAa?$AAc?$AAe?$AA?5?$AAi?$AAs?$AA?5?$AAa?$AAt?$AA?5?$AA0?$AAx?$AA?$CF?$AA0?$AA8?$AAx?$AA?$AN?$AA?6?$AA?$AA@ 10005114     gpe:ddi_if.obj
 0001:00004154       ??_C@_1DI@EIKKJEHH@?$AAE?$AAn?$AAt?$AAe?$AAr?$AAi?$AAn?$AAg?$AA?5?$AAD?$AAr?$AAv?$AAE?$AAn?$AAa?$AAb?$AAl?$AAe?$AAS?$AAu?$AAr?$AAf?$AAa?$AAc?$AAe?$AA?$AN?$AA?6?$AA?$AA@ 10005154     gpe:ddi_if.obj
 0001:00004190       ??_C@_1EC@DOEGPCON@?$AAE?$AAn?$AAt?$AAe?$AAr?$AAi?$AAn?$AAg?$AA?5?$AAD?$AAr?$AAv?$AAC?$AAr?$AAe?$AAa?$AAt?$AAe?$AAD?$AAe?$AAv?$AAi?$AAc?$AAe?$AAB?$AAi?$AAt?$AAm?$AAa?$AAp?$AA?$AN?$AA?6@ 10005190     gpe:ddi_if.obj
 0001:000041d8       ??_C@_1EA@LBCKBJNL@?$AAL?$AAe?$AAa?$AAv?$AAi?$AAn?$AAg?$AA?5?$AAD?$AAr?$AAv?$AAD?$AAe?$AAl?$AAe?$AAt?$AAe?$AAD?$AAe?$AAv?$AAi?$AAc?$AAe?$AAB?$AAi?$AAt?$AAm?$AAa?$AAp?$AA?$AN?$AA?6?$AA?$AA@ 100051d8     gpe:ddi_if.obj
 0001:00004218       ??_C@_1EC@ODGLMPKP@?$AAE?$AAn?$AAt?$AAe?$AAr?$AAi?$AAn?$AAg?$AA?5?$AAD?$AAr?$AAv?$AAD?$AAe?$AAl?$AAe?$AAt?$AAe?$AAD?$AAe?$AAv?$AAi?$AAc?$AAe?$AAB?$AAi?$AAt?$AAm?$AAa?$AAp?$AA?$AN?$AA?6@ 10005218     gpe:ddi_if.obj
 0001:0000425c       ??_C@_1DC@NEKPMNED@?$AAL?$AAe?$AAa?$AAv?$AAi?$AAn?$AAg?$AA?5?$AAD?$AAr?$AAv?$AAM?$AAo?$AAv?$AAe?$AAP?$AAo?$AAi?$AAn?$AAt?$AAe?$AAr?$AA?$AN?$AA?6?$AA?$AA@ 1000525c     gpe:ddi_if.obj
 0001:00004290       ??_C@_1DE@OIJGDPMD@?$AAE?$AAn?$AAt?$AAe?$AAr?$AAi?$AAn?$AAg?$AA?5?$AAD?$AAr?$AAv?$AAM?$AAo?$AAv?$AAe?$AAP?$AAo?$AAi?$AAn?$AAt?$AAe?$AAr?$AA?$AN?$AA?6?$AA?$AA@ 10005290     gpe:ddi_if.obj
 0001:000042c4       ??_C@_1DK@BPHDJFEP@?$AAL?$AAe?$AAa?$AAv?$AAi?$AAn?$AAg?$AA?5?$AAD?$AAr?$AAv?$AAS?$AAe?$AAt?$AAP?$AAo?$AAi?$AAn?$AAt?$AAe?$AAr?$AAS?$AAh?$AAa?$AAp?$AAe?$AA?$AN?$AA?6?$AA?$AA@ 100052c4     gpe:ddi_if.obj
 0001:00004300       ??_C@_1DM@PIANDIIH@?$AAE?$AAn?$AAt?$AAe?$AAr?$AAi?$AAn?$AAg?$AA?5?$AAD?$AAr?$AAv?$AAS?$AAe?$AAt?$AAP?$AAo?$AAi?$AAn?$AAt?$AAe?$AAr?$AAS?$AAh?$AAa?$AAp?$AAe?$AA?$AN?$AA?6?$AA?$AA@ 10005300     gpe:ddi_if.obj
 0001:0000433c       ??_C@_1DA@CMGHIIMF@?$AAL?$AAe?$AAa?$AAv?$AAi?$AAn?$AAg?$AA?5?$AAD?$AAr?$AAv?$AAS?$AAe?$AAt?$AAP?$AAa?$AAl?$AAe?$AAt?$AAt?$AAe?$AA?$AN?$AA?6?$AA?$AA@ 1000533c     gpe:ddi_if.obj
 0001:0000436c       ??_C@_1DC@IPGHGCKE@?$AAE?$AAn?$AAt?$AAe?$AAr?$AAi?$AAn?$AAg?$AA?5?$AAD?$AAr?$AAv?$AAS?$AAe?$AAt?$AAP?$AAa?$AAl?$AAe?$AAt?$AAt?$AAe?$AA?$AN?$AA?6?$AA?$AA@ 1000536c     gpe:ddi_if.obj
 0001:000043a0       ??_C@_1GI@FGCHMFAF@?$AAC?$AAa?$AAl?$AAl?$AAi?$AAn?$AAg?$AA?5?$AAP?$AAo?$AAl?$AAy?$AAg?$AAo?$AAn?$AAL?$AAi?$AAs?$AAt?$AA?3?$AA?3?$AAF?$AAi?$AAl?$AAl?$AA?$CI?$AA?$CJ?$AA?5?$AAw?$AAi?$AAt?$AAh@ 100053a0     gpe:ddi_if.obj
 0001:00004408       ??_C@_1DA@HMEEEAF@?$AAC?$AAa?$AAl?$AAl?$AAi?$AAn?$AAg?$AA?5?$AAC?$AAL?$AAI?$AAP?$AAO?$AAB?$AAJ?$AA_?$AAb?$AAE?$AAn?$AAu?$AAm?$AA?$AN?$AA?6?$AA?$AA@ 10005408     gpe:ddi_if.obj
 0001:00004438       ??_C@_1GE@CKEJAAIC@?$AAI?$AAt?$AAe?$AAr?$AAa?$AAt?$AAi?$AAn?$AAg?$AA?5?$AAt?$AAh?$AAr?$AAo?$AAu?$AAg?$AAh?$AA?5?$AAc?$AAo?$AAm?$AAp?$AAl?$AAe?$AAx?$AA?5?$AAc?$AAl?$AAi?$AAp?$AAp?$AAi@ 10005438     gpe:ddi_if.obj
 0001:000044a0       ??_C@_1GG@CBKOLKEC@?$AAC?$AAa?$AAl?$AAl?$AAi?$AAn?$AAg?$AA?5?$AAP?$AAo?$AAl?$AAy?$AAg?$AAo?$AAn?$AAL?$AAi?$AAs?$AAt?$AA?3?$AA?3?$AAF?$AAi?$AAl?$AAl?$AA?$CI?$AA?$CJ?$AA?5?$AAw?$AAi?$AAt?$AAh@ 100054a0     gpe:ddi_if.obj
 0001:00004508       ??_C@_1FO@KBLIELFA@?$AAC?$AAa?$AAl?$AAl?$AAi?$AAn?$AAg?$AA?5?$AAP?$AAo?$AAl?$AAy?$AAg?$AAo?$AAn?$AAL?$AAi?$AAs?$AAt?$AA?3?$AA?3?$AAF?$AAi?$AAl?$AAl?$AA?$CI?$AA?$CJ?$AA?5?$AAw?$AAi?$AAt?$AAh@ 10005508     gpe:ddi_if.obj
 0001:00004568       ??_C@_1GA@MGPBKDJD@?$AAF?$AAa?$AAi?$AAl?$AAe?$AAd?$AA?5?$AAt?$AAo?$AA?5?$AAp?$AAr?$AAe?$AAp?$AAa?$AAr?$AAe?$AA?5?$AAb?$AAl?$AAt?$AA?5?$AAf?$AAo?$AAr?$AA?5?$AAf?$AAi?$AAl?$AAl?$AAp?$AAo@ 10005568     gpe:ddi_if.obj
 0001:000045c8       ??_C@_1CM@DCPLGONG@?$AAL?$AAe?$AAa?$AAv?$AAi?$AAn?$AAg?$AA?5?$AAD?$AAr?$AAv?$AAF?$AAi?$AAl?$AAl?$AAP?$AAa?$AAt?$AAh?$AA?$AN?$AA?6?$AA?$AA@ 100055c8     gpe:ddi_if.obj
 0001:000045f4       ??_C@_1DG@FIDENMKJ@?$AAF?$AAa?$AAi?$AAl?$AAe?$AAd?$AA?5?$AAt?$AAo?$AA?5?$AAa?$AAl?$AAl?$AAo?$AAc?$AAa?$AAt?$AAe?$AA?5?$AAb?$AAr?$AAu?$AAs?$AAh?$AA?$AN?$AA?6?$AA?$AA@ 100055f4     gpe:ddi_if.obj
 0001:0000462c       ??_C@_1CO@OJOFEFPL@?$AAE?$AAn?$AAt?$AAe?$AAr?$AAi?$AAn?$AAg?$AA?5?$AAD?$AAr?$AAv?$AAF?$AAi?$AAl?$AAl?$AAP?$AAa?$AAt?$AAh?$AA?$AN?$AA?6?$AA?$AA@ 1000562c     gpe:ddi_if.obj
 0001:0000465c       ??_C@_1DE@PFEEBFPK@?$AAL?$AAe?$AAa?$AAv?$AAi?$AAn?$AAg?$AA?5?$AAD?$AAr?$AAv?$AAR?$AAe?$AAa?$AAl?$AAi?$AAz?$AAe?$AAB?$AAr?$AAu?$AAs?$AAh?$AA?$AN?$AA?6?$AA?$AA@ 1000565c     gpe:ddi_if.obj
 0001:00004690       ??_C@_1DG@JNHECCLI@?$AAE?$AAn?$AAt?$AAe?$AAr?$AAi?$AAn?$AAg?$AA?5?$AAD?$AAr?$AAv?$AAR?$AAe?$AAa?$AAl?$AAi?$AAz?$AAe?$AAB?$AAr?$AAu?$AAs?$AAh?$AA?$AN?$AA?6?$AA?$AA@ 10005690     gpe:ddi_if.obj
 0001:000046c8       ??_C@_17BJMBELJK@?$AAG?$AAP?$AAE?$AA?$AA@ 100056c8     gpe:ddi_if.obj
 0001:000046d0       ??_C@_1CM@PKBMGPPM@?$AAL?$AAe?$AAa?$AAv?$AAi?$AAn?$AAg?$AA?5?$AAD?$AAr?$AAv?$AAG?$AAe?$AAt?$AAM?$AAo?$AAd?$AAe?$AAs?$AA?$AN?$AA?6?$AA?$AA@ 100056d0     gpe:ddi_if.obj
 0001:000046fc       ??_C@_1CO@CBACEENB@?$AAE?$AAn?$AAt?$AAe?$AAr?$AAi?$AAn?$AAg?$AA?5?$AAD?$AAr?$AAv?$AAG?$AAe?$AAt?$AAM?$AAo?$AAd?$AAe?$AAs?$AA?$AN?$AA?6?$AA?$AA@ 100056fc     gpe:ddi_if.obj
 0001:0000472c       ??_C@_1CK@PNIBBLCM@?$AAB?$AAi?$AAt?$AAs?$AA?9?$AAp?$AAe?$AAr?$AA?9?$AAp?$AAi?$AAx?$AAe?$AAl?$AA?3?$AA?5?$AA?$CF?$AAd?$AA?$AN?$AA?6?$AA?$AA@ 1000572c     gpe:ddi_if.obj
 0001:00004758       ??_C@_1FI@FEOICDNP@?$AAF?$AAa?$AAi?$AAl?$AAe?$AAd?$AA?5?$AAt?$AAo?$AA?5?$AAs?$AAe?$AAt?$AA?5?$AAm?$AAo?$AAd?$AAe?$AA?$CB?$AA?5?$AAL?$AAe?$AAa?$AAv?$AAi?$AAn?$AAg?$AA?5?$AAD?$AAr?$AAv?$AAE@ 10005758     gpe:ddi_if.obj
 0001:000047b0       ??_C@_1HE@NKFIKAEA@?$AAF?$AAa?$AAi?$AAl?$AAe?$AAd?$AA?5?$AAA?$AAl?$AAl?$AAo?$AAc?$AAa?$AAt?$AAe?$AA?5?$AAc?$AAo?$AAl?$AAo?$AAr?$AA?5?$AAc?$AAo?$AAn?$AAv?$AAe?$AAr?$AAt?$AAe?$AAr?$AAs@ 100057b0     gpe:ddi_if.obj
 0001:00004824       ??_C@_1DA@HIINMLMJ@?$AAL?$AAe?$AAa?$AAv?$AAi?$AAn?$AAg?$AA?5?$AAD?$AAr?$AAv?$AAE?$AAn?$AAa?$AAb?$AAl?$AAe?$AAP?$AAD?$AAE?$AAV?$AA?$AN?$AA?6?$AA?$AA@ 10005824     gpe:ddi_if.obj
 0001:00004858       ??_C@_1FE@ENEIHIHG@?$AAE?$AAR?$AAR?$AAO?$AAR?$AA?3?$AA?5?$AAF?$AAa?$AAi?$AAl?$AAe?$AAd?$AA?5?$AAt?$AAo?$AA?5?$AAi?$AAn?$AAs?$AAt?$AAa?$AAn?$AAt?$AAi?$AAa?$AAt?$AAe?$AA?5?$AAG?$AAP?$AAE@ 10005858     gpe:ddi_if.obj
 0001:000048ac       ??_C@_1DC@NLINCBKI@?$AAE?$AAn?$AAt?$AAe?$AAr?$AAi?$AAn?$AAg?$AA?5?$AAD?$AAr?$AAv?$AAE?$AAn?$AAa?$AAb?$AAl?$AAe?$AAP?$AAD?$AAE?$AAV?$AA?$AN?$AA?6?$AA?$AA@ 100058ac     gpe:ddi_if.obj
 0001:000048e0       ??_C@_1CG@JKBKEKHA@?$AAL?$AAe?$AAa?$AAv?$AAi?$AAn?$AAg?$AA?5?$AAD?$AAr?$AAv?$AAP?$AAa?$AAi?$AAn?$AAt?$AA?$AN?$AA?6?$AA?$AA@ 100058e0     gpe:ddi_if.obj
 0001:00004908       ??_C@_1DA@HDIPCCJP@?$AAD?$AAr?$AAv?$AAP?$AAa?$AAi?$AAn?$AAt?$AA?5?$AA?$CI?$AAm?$AAi?$AAx?$AA?$DN?$AA0?$AAx?$AA?$CF?$AA0?$AA4?$AAx?$AA?$CJ?$AA?$AN?$AA?6?$AA?$AA@ 10005908     gpe:ddi_if.obj
 0001:00004938       ??_C@_1CI@BGHCMLLF@?$AAE?$AAn?$AAt?$AAe?$AAr?$AAi?$AAn?$AAg?$AA?5?$AAD?$AAr?$AAv?$AAP?$AAa?$AAi?$AAn?$AAt?$AA?$AN?$AA?6?$AA?$AA@ 10005938     gpe:ddi_if.obj
 0001:00004960       ??_C@_1IC@LKLBHCP@?$AAE?$AAn?$AAt?$AAe?$AAr?$AAi?$AAn?$AAg?$AA?5?$AAD?$AAr?$AAv?$AAC?$AAo?$AAp?$AAy?$AAB?$AAi?$AAt?$AAs?$AA?$CB?$AA?5?$AA?9?$AA?5?$AAS?$AAH?$AAO?$AAU?$AAL?$AAD?$AA?5?$AAO@ 10005960     gpe:ddi_if.obj
 0001:000049e4       ??_C@_1CK@FEEIOLBK@?$AAE?$AAn?$AAt?$AAe?$AAr?$AAi?$AAn?$AAg?$AA?5?$AAD?$AAr?$AAv?$AAA?$AAn?$AAy?$AAB?$AAl?$AAt?$AA?$AN?$AA?6?$AA?$AA@ 100059e4     gpe:ddi_if.obj
 0001:00004a10       ??_C@_1DK@KMLCKHGG@?$AAE?$AAn?$AAt?$AAe?$AAr?$AAi?$AAn?$AAg?$AA?5?$AAD?$AAr?$AAv?$AAT?$AAr?$AAa?$AAn?$AAs?$AAp?$AAa?$AAr?$AAe?$AAn?$AAt?$AAB?$AAl?$AAt?$AA?$AN?$AA?6?$AA?$AA@ 10005a10     gpe:ddi_if.obj
 0001:00004a4c       ??_C@_1CK@PEMNLOFG@?$AAE?$AAn?$AAt?$AAe?$AAr?$AAi?$AAn?$AAg?$AA?5?$AAD?$AAr?$AAv?$AAB?$AAi?$AAt?$AAB?$AAl?$AAt?$AA?$AN?$AA?6?$AA?$AA@ 10005a4c     gpe:ddi_if.obj
 0001:00004a78       ??_C@_1FC@KFANHFOM@?$AAC?$AAa?$AAl?$AAl?$AAi?$AAn?$AAg?$AA?5?$AAG?$AAP?$AAE?$AA?3?$AA?3?$AAB?$AAl?$AAt?$AA?5?$AAw?$AAi?$AAt?$AAh?$AA?5?$AAc?$AAo?$AAm?$AAp?$AAl?$AAe?$AAx?$AA?5?$AAc?$AAl@ 10005a78     gpe:ddi_if.obj
 0001:00004acc       ??_C@_1CI@NIPPKCID@?$AAL?$AAe?$AAa?$AAv?$AAi?$AAn?$AAg?$AA?5?$AAD?$AAr?$AAv?$AAB?$AAi?$AAt?$AAB?$AAl?$AAt?$AA?$AN?$AA?6?$AA?$AA@ 10005acc     gpe:ddi_if.obj
 0001:00004af4       ??_C@_1DA@BBNMBMPA@?$AAf?$AAa?$AAi?$AAl?$AAe?$AAd?$AA?5?$AAt?$AAo?$AA?5?$AAp?$AAr?$AAe?$AAp?$AAa?$AAr?$AAe?$AA?5?$AAb?$AAl?$AAt?$AA?$AN?$AA?6?$AA?$AA@ 10005af4     gpe:ddi_if.obj
 0001:00004b28       ??_C@_1EK@IIPEPFHJ@?$AAB?$AAl?$AAt?$AA?5?$AAw?$AA?1?$AA?5?$AAr?$AAo?$AAp?$AA4?$AA?$DN?$AA0?$AAx?$AA?$CF?$AA0?$AA4?$AAx?$AA?5?$AAa?$AAn?$AAd?$AA?5?$AAp?$AAb?$AAo?$AA?$DN?$AA?$DN?$AAN?$AAU?$AAL?$AAL@ 10005b28     gpe:ddi_if.obj
 0001:00004b78       ??_C@_1FM@GOEMNJPF@?$AAB?$AAl?$AAt?$AA?5?$AAw?$AA?1?$AA?5?$AAr?$AAo?$AAp?$AA4?$AA?$DN?$AA0?$AAx?$AA?$CF?$AA0?$AA4?$AAx?$AA?5?$AAa?$AAn?$AAd?$AA?5?$AAp?$AAa?$AAr?$AAm?$AAs?$AA?4?$AAp?$AAB?$AAr@ 10005b78     gpe:ddi_if.obj
 0001:00004bd8       ??_C@_1GI@MNGANCMC@?$AAA?$AAn?$AAy?$AAB?$AAl?$AAt?$AA?5?$AA?$CI?$AAr?$AAo?$AAp?$AA4?$AA?5?$AA?$DN?$AA?5?$AA0?$AAx?$AA?$CF?$AA0?$AA4?$AAx?$AA?$CJ?$AA?5?$AAr?$AAc?$AAl?$AAT?$AAr?$AAg?$AA?$DN?$AAt?$AA?3@ 10005bd8     gpe:ddi_if.obj
 0001:00004c40       ??_C@_1DC@NPHDKAFM@?$AAC?$AAl?$AAi?$AAp?$AAB?$AAl?$AAt?$AA?5?$AAc?$AAo?$AAn?$AAt?$AAi?$AAn?$AAu?$AAe?$AA?5?$AAp?$AAh?$AAa?$AAs?$AAe?$AA?$AN?$AA?6?$AA?$AA@ 10005c40     gpe:ddi_if.obj
 0001:00004c74       EGPEFormatToBpp            10005c74     gpe:gpe.obj
 0001:00004c98       EGPEFormatToIFormat        10005c98     gpe:gpe.obj
 0001:00004cbc       IFormatToEGPEFormat        10005cbc     gpe:gpe.obj
 0001:00004ce8       ??_7GPE@@6B@               10005ce8     gpe:gpe.obj
 0001:00004d68       ??_C@_1CA@BGCHCNGF@?$AAT?$AAo?$AAu?$AAc?$AAh?$AAT?$AAa?$AAr?$AAg?$AAe?$AAt?$AAS?$AAi?$AAz?$AAe?$AA?$AA@ 10005d68     gpe:gpe.obj
 0001:00004d88       ??_C@_1BM@OHJNPODK@?$AAA?$AAs?$AAp?$AAe?$AAc?$AAt?$AAR?$AAa?$AAt?$AAi?$AAo?$AAX?$AAY?$AA?$AA@ 10005d88     gpe:gpe.obj
 0001:00004da4       ??_C@_1BK@GPCKCPMK@?$AAA?$AAs?$AAp?$AAe?$AAc?$AAt?$AAR?$AAa?$AAt?$AAi?$AAo?$AAY?$AA?$AA@ 10005da4     gpe:gpe.obj
 0001:00004dc0       ??_C@_1BK@NHJGEIKP@?$AAA?$AAs?$AAp?$AAe?$AAc?$AAt?$AAR?$AAa?$AAt?$AAi?$AAo?$AAX?$AA?$AA@ 10005dc0     gpe:gpe.obj
 0001:00004ddc       ??_C@_1BO@ONBCMHFO@?$AAL?$AAo?$AAg?$AAi?$AAc?$AAa?$AAl?$AAP?$AAi?$AAx?$AAe?$AAl?$AAs?$AAY?$AA?$AA@ 10005ddc     gpe:gpe.obj
 0001:00004dfc       ??_C@_1BO@FFKOKADL@?$AAL?$AAo?$AAg?$AAi?$AAc?$AAa?$AAl?$AAP?$AAi?$AAx?$AAe?$AAl?$AAs?$AAX?$AA?$AA@ 10005dfc     gpe:gpe.obj
 0001:00004e1c       ??_C@_1BK@HNDINEGH@?$AAV?$AAe?$AAr?$AAt?$AAi?$AAc?$AAa?$AAl?$AAS?$AAi?$AAz?$AAe?$AA?$AA@ 10005e1c     gpe:gpe.obj
 0001:00004e38       ??_C@_1BO@CPEMBNKP@?$AAH?$AAo?$AAr?$AAi?$AAz?$AAo?$AAn?$AAt?$AAa?$AAl?$AAS?$AAi?$AAz?$AAe?$AA?$AA@ 10005e38     gpe:gpe.obj
 0001:00004e58       ??_C@_1KA@GGIGJJEF@?$AAI?$AAn?$AAt?$AAe?$AAg?$AAe?$AAr?$AA?9?$AAo?$AAv?$AAe?$AAr?$AAf?$AAl?$AAo?$AAw?$AA?5?$AAd?$AAe?$AAt?$AAe?$AAc?$AAt?$AAe?$AAd?$AA?5?$AAw?$AAh?$AAi?$AAl?$AAe?$AA?5@ 10005e58     gpe:gpe.obj
 0001:00004ef8       ??_C@_1HI@FBPHGCDA@?$AAd?$AA?3?$AA?2?$AAc?$AAh?$AAe?$AAl?$AAa?$AAn?$AAr?$AAt?$AAm?$AA2?$AA?2?$AAp?$AAu?$AAb?$AAl?$AAi?$AAc?$AA?2?$AAc?$AAo?$AAm?$AAm?$AAo?$AAn?$AA?2?$AAo?$AAa?$AAk?$AA?2@ 10005ef8     gpe:gpe.obj
 0001:00004f70       ??_C@_1GA@NKEECKM@?$AAy?$AAS?$AAt?$AAr?$AAe?$AAt?$AAc?$AAh?$AA?5?$AA?9?$AA?5?$AAS?$AAw?$AAi?$AAt?$AAc?$AAh?$AA?5?$AAt?$AAo?$AA?5?$AAn?$AAe?$AAx?$AAt?$AA?5?$AAa?$AAf?$AAt?$AAe?$AAr?$AA?5@ 10005f70     gpe:swblt.obj
 0001:00004fd0       ??_C@_1DM@KJNPBLPC@?$AAy?$AAS?$AAt?$AAr?$AAe?$AAt?$AAc?$AAh?$AA?5?$AA?9?$AA?5?$AAR?$AAe?$AAp?$AAe?$AAa?$AAt?$AA?4?$AA?5?$AAA?$AAc?$AAc?$AAu?$AAm?$AA?$DN?$AA?$CF?$AAd?$AA?$AN?$AA?6?$AA?$AA@ 10005fd0     gpe:swblt.obj
 0001:0000500c       ??_C@_1CM@EKMJNAGM@?$AAy?$AAS?$AAh?$AAr?$AAi?$AAn?$AAk?$AA?5?$AA?9?$AA?5?$AAs?$AAk?$AAi?$AAp?$AA?5?$AAl?$AAi?$AAn?$AAe?$AA?$AN?$AA?6?$AA?$AA@ 1000600c     gpe:swblt.obj
 0001:00005038       ??_C@_1IG@BICGLEAL@?$AAt?$AAr?$AAa?$AAn?$AAs?$AAp?$AAa?$AAr?$AAe?$AAn?$AAt?$AA?3?$AA?$CF?$AAd?$AA?0?$AAm?$AAa?$AAs?$AAk?$AAe?$AAd?$AA?3?$AA?$CF?$AA2?$AAx?$AA?0?$AAu?$AAn?$AAm?$AAa?$AAs?$AAk@ 10006038     gpe:swblt.obj
 0001:000050c0       ??_C@_1BO@HLFKJPKP@?$AAC?$AAo?$AAm?$AAp?$AAl?$AAe?$AAx?$AA?5?$AAB?$AAl?$AAt?$AA?$CB?$AA?$AN?$AA?6?$AA?$AA@ 100060c0     gpe:swblt.obj
 0001:000050e0       ??_C@_1HA@IKNKPGOM@?$AAy?$AAS?$AAt?$AAr?$AAe?$AAt?$AAc?$AAh?$AA?3?$AA?$CF?$AAd?$AA?5?$AAy?$AAS?$AAh?$AAr?$AAi?$AAn?$AAk?$AA?3?$AA?$CF?$AAd?$AA?5?$AAy?$AAD?$AAM?$AAi?$AAn?$AAo?$AAr?$AA?3?$AA?$CF@ 100060e0     gpe:swblt.obj
 0001:00005150       ??_C@_1CO@FHBFEHPE@?$AAp?$AAB?$AAr?$AAu?$AAs?$AAh?$AA?5?$AAd?$AAe?$AAp?$AAt?$AAh?$AA?3?$AA?5?$AA?$CF?$AAd?$AA?5?$AAB?$AAp?$AAp?$AA?$AN?$AA?6?$AA?$AA@ 10006150     gpe:swblt.obj
 0001:00005180       ??_C@_1DA@PPGABIAI@?$AAP?$AAa?$AAt?$AAt?$AAe?$AAr?$AAn?$AA?5?$AAd?$AAe?$AAp?$AAt?$AAh?$AA?3?$AA?5?$AA?$CF?$AAd?$AA?5?$AAB?$AAp?$AAp?$AA?$AN?$AA?6?$AA?$AA@ 10006180     gpe:swblt.obj
 0001:000051b0       ??_C@_1CK@HHCIFAFM@?$AAp?$AAD?$AAs?$AAt?$AA?5?$AAd?$AAe?$AAp?$AAt?$AAh?$AA?3?$AA?5?$AA?$CF?$AAd?$AA?5?$AAB?$AAp?$AAp?$AA?$AN?$AA?6?$AA?$AA@ 100061b0     gpe:swblt.obj
 0001:000051dc       ??_C@_1CK@EJILBMCC@?$AAp?$AAS?$AAr?$AAc?$AA?5?$AAd?$AAe?$AAp?$AAt?$AAh?$AA?3?$AA?5?$AA?$CF?$AAd?$AA?5?$AAB?$AAp?$AAp?$AA?$AN?$AA?6?$AA?$AA@ 100061dc     gpe:swblt.obj
 0001:00005208       ??_C@_1GI@BPNEJCEA@?$AAp?$AAS?$AAr?$AAc?$AA?$DN?$AA0?$AAx?$AA?$CF?$AA0?$AA8?$AAx?$AA?0?$AA?5?$AAp?$AAD?$AAs?$AAt?$AA?$DN?$AA0?$AAx?$AA?$CF?$AA0?$AA8?$AAx?$AA?0?$AA?5?$AAp?$AAB?$AAr?$AAu?$AAs?$AAh@ 10006208     gpe:swblt.obj
 0001:00005270       ??_C@_1HM@KDLGFJNL@?$AAd?$AA?3?$AA?2?$AAc?$AAh?$AAe?$AAl?$AAa?$AAn?$AAr?$AAt?$AAm?$AA2?$AA?2?$AAp?$AAu?$AAb?$AAl?$AAi?$AAc?$AA?2?$AAc?$AAo?$AAm?$AAm?$AAo?$AAn?$AA?2?$AAo?$AAa?$AAk?$AA?2@ 10006270     gpe:swblt.obj
 0001:000052ec       ??_C@_1CK@LKLEEHPJ@?$AAN?$AAe?$AAw?$AA?5?$AAB?$AAl?$AAt?$AA?4?$AA?5?$AAr?$AAo?$AAp?$AA4?$AA?$DN?$AA?$CF?$AA0?$AA4?$AAX?$AA?$AN?$AA?6?$AA?$AA@ 100062ec     gpe:swblt.obj
 0001:00005318       ??_C@_1EM@CBPHKBCP@?$AAR?$AAo?$AAp?$AA4?$AA?5?$AA?$DN?$AA?5?$AA?$CF?$AA0?$AA4?$AAx?$AA?5?$AAb?$AAu?$AAt?$AA?5?$AAm?$AAa?$AAs?$AAk?$AA?4?$AAR?$AAo?$AAw?$AAP?$AAt?$AAr?$AA?5?$AAi?$AAs?$AA?5?$AAN@ 10006318     gpe:swblt.obj
 0001:00005368       ??_C@_1EA@IPGJNIEJ@?$AAR?$AAo?$AAp?$AA4?$AA?5?$AA?$DN?$AA?5?$AA?$CF?$AA0?$AA4?$AAx?$AA?5?$AAb?$AAu?$AAt?$AA?5?$AAp?$AAM?$AAa?$AAs?$AAk?$AA?5?$AAi?$AAs?$AA?5?$AAN?$AAU?$AAL?$AAL?$AA?$AN?$AA?6?$AA?$AA@ 10006368     gpe:swblt.obj
 0001:000053a8       ??_C@_1DK@OGHLJHLF@?$AAD?$AAi?$AAa?$AAg?$AAo?$AAn?$AAa?$AAl?$AA?5?$AAa?$AAc?$AAc?$AAu?$AAm?$AA?$DN?$AA?$CF?$AAd?$AA?5?$AAd?$AAg?$AAs?$AAt?$AAp?$AA?$DN?$AA?$CF?$AAd?$AA?$AN?$AA?6?$AA?$AA@ 100063a8     gpe:swline.obj
 0001:000053e4       ??_C@_1DK@IMLDDPEK@?$AAS?$AAt?$AAr?$AAa?$AAi?$AAg?$AAh?$AAt?$AA?5?$AAa?$AAc?$AAc?$AAu?$AAm?$AA?$DN?$AA?$CF?$AAd?$AA?5?$AAa?$AAx?$AAs?$AAt?$AAp?$AA?$DN?$AA?$CF?$AAd?$AA?$AN?$AA?6?$AA?$AA@ 100063e4     gpe:swline.obj
 0001:00005420       ??_C@_1GA@MHBMBPAI@?$AAR?$AAe?$AAs?$AAu?$AAl?$AAt?$AA?3?$AA?5?$AAP?$AA?5?$AA?$CF?$AA0?$AA8?$AAx?$AA?0?$AA?5?$AAD?$AA?5?$AA?$CF?$AA0?$AA8?$AAx?$AA?0?$AA?5?$AAm?$AAa?$AAs?$AAk?$AA?5?$AA?$CF?$AA0?$AA8@ 10006420     gpe:swline.obj
 0001:00005480       ??_C@_1CG@HGKBKIFB@?$AAI?$AAn?$AAv?$AAa?$AAl?$AAi?$AAd?$AA?5?$AAr?$AAo?$AAp?$AA2?$AA?3?$AA?5?$AA?$CF?$AAd?$AA?$AN?$AA?6?$AA?$AA@ 10006480     gpe:swline.obj
 0001:000054a8       ??_C@_1FE@BNGJJPHG@?$AAR?$AAe?$AAm?$AAa?$AAi?$AAn?$AA?3?$AA?$CF?$AAd?$AA?5?$AAP?$AAt?$AAr?$AA?3?$AA?$CF?$AA0?$AA8?$AAx?$AA?5?$AAS?$AAu?$AAb?$AAP?$AAi?$AAx?$AA?3?$AA?$CF?$AAd?$AA?5?$AAc?$AAa?$AAc@ 100064a8     gpe:swline.obj
 0001:00005500       ??_C@_1FC@EKFELALA@?$AAD?$AAW?$AAo?$AAr?$AAd?$AA?5?$AAP?$AAi?$AAx?$AAe?$AAl?$AA?5?$AA?$CF?$AAd?$AA?5?$AAp?$AAe?$AAn?$AA?3?$AA?5?$AA?$CF?$AA0?$AA8?$AAx?$AA?5?$AAp?$AAe?$AAn?$AAM?$AAa?$AAs?$AAk@ 10006500     gpe:swline.obj
 0001:00005554       ??_C@_1CI@ELKBBDKP@?$AAM?$AAi?$AAx?$AA?3?$AA?5?$AA?$CF?$AA0?$AA4?$AAx?$AA?5?$AAB?$AAp?$AAp?$AA?3?$AA?5?$AA?$CF?$AAd?$AA?$AN?$AA?6?$AA?$AA@ 10006554     gpe:swline.obj
 0001:00005580       ??_C@_1EK@GFGGNHIM@?$AAi?$AAD?$AAi?$AAr?$AA?3?$AA?$CF?$AAd?$AA?5?$AAa?$AAc?$AAc?$AAu?$AAm?$AA?5?$AA?$CF?$AAd?$AA?5?$AAa?$AAx?$AAs?$AAt?$AAp?$AA?5?$AA?$CF?$AAd?$AA?5?$AAd?$AAg?$AAs?$AAt?$AAp?$AA?5@ 10006580     gpe:swline.obj
 0001:000055cc       ??_C@_1CE@NHJNKOGG@?$AAS?$AAt?$AAa?$AAr?$AAt?$AA?5?$AAX?$AA?$DN?$AA?$CF?$AAd?$AA?0?$AAY?$AA?$DN?$AA?$CF?$AAd?$AA?$AN?$AA?6?$AA?$AA@ 100065cc     gpe:swline.obj
 0001:000055f0       ??_C@_1CK@JMKICICF@?$AAS?$AAo?$AAl?$AAi?$AAd?$AA?5?$AAc?$AAo?$AAl?$AAo?$AAr?$AA?5?$AA0?$AAx?$AA?$CF?$AA0?$AA8?$AAx?$AA?$AN?$AA?6?$AA?$AA@ 100065f0     gpe:swline.obj
 0001:0000561c       ??_C@_1CI@JGCGFAPH@?$AAG?$AAP?$AAE?$AA?3?$AA?3?$AAE?$AAm?$AAu?$AAl?$AAa?$AAt?$AAe?$AAd?$AAL?$AAi?$AAn?$AAe?$AA?$AN?$AA?6?$AA?$AA@ 1000661c     gpe:swline.obj
 0001:00005678       ??_C@_1IC@PACPAOAE@?$AAd?$AA?3?$AA?2?$AAc?$AAh?$AAe?$AAl?$AAa?$AAn?$AAr?$AAt?$AAm?$AA2?$AA?2?$AAp?$AAu?$AAb?$AAl?$AAi?$AAc?$AA?2?$AAc?$AAo?$AAm?$AAm?$AAo?$AAn?$AA?2?$AAo?$AAa?$AAk?$AA?2@ 10006678     gpe:swconvrt.obj
 0001:000056fc       ??_C@_1DK@HLNCNPPO@?$AAL?$AAR?$AAU?$AA?3?$AA?3?$AAL?$AAR?$AAU?$AA?$CI?$AA?5?$AAl?$AAi?$AAs?$AAt?$AA?5?$AAs?$AAi?$AAz?$AAe?$AA?5?$AA?$DN?$AA?5?$AA?$CF?$AAd?$AA?5?$AA?$CJ?$AA?$AN?$AA?6?$AA?$AA@ 100066fc     gpe:swconvrt.obj
 0001:00005738       ??_C@_1EK@FEGFCNEO@?$AAL?$AAR?$AAU?$AA?5?$AA0?$AAx?$AA?$CF?$AA0?$AA8?$AAx?$AA?5?$AAF?$AAi?$AAn?$AAd?$AA?5?$AA0?$AAx?$AA?$CF?$AA0?$AA8?$AAx?$AA?3?$AA?5?$AAN?$AAo?$AAt?$AA?5?$AAf?$AAo?$AAu?$AAn@ 10006738     gpe:swconvrt.obj
 0001:00005788       ??_C@_1FO@KFKLLIJI@?$AAL?$AAR?$AAU?$AA?5?$AA0?$AAx?$AA?$CF?$AA0?$AA8?$AAx?$AA?5?$AAF?$AAi?$AAn?$AAd?$AA?5?$AA0?$AAx?$AA?$CF?$AA0?$AA8?$AAx?$AA?3?$AA?5?$AAf?$AAo?$AAu?$AAn?$AAd?$AA?5?$AAa?$AAt@ 10006788     gpe:swconvrt.obj
 0001:000057e8       ??_C@_1DA@JGGIDAGP@?$AAm?$AAa?$AAs?$AAk?$AA?1?$AAr?$AAg?$AAb?$AA?5?$AA?$DM?$AA?9?$AA?$DO?$AA?5?$AAm?$AAa?$AAs?$AAk?$AA?1?$AAr?$AAg?$AAb?$AA?$AN?$AA?6?$AA?$AA@ 100067e8     gpe:swconvrt.obj
 0001:00005818       ??_C@_1CK@COLJNAIA@?$AAU?$AAn?$AAk?$AAn?$AAo?$AAw?$AAn?$AA?5?$AAs?$AAu?$AAr?$AAf?$AAa?$AAc?$AAe?$AA?5?$AAt?$AAy?$AAp?$AAe?$AA?$AA@ 10006818     gpe:swconvrt.obj
 0001:00005844       ??_C@_1CA@IFLBOBIE@?$AA?9?$AA?$DO?$AAP?$AAA?$AAL?$AA_?$AAI?$AAN?$AAD?$AAE?$AAX?$AAE?$AAD?$AA?$AN?$AA?6?$AA?$AA@ 10006844     gpe:swconvrt.obj
 0001:00005864       ??_C@_1CA@MKJFIFEN@?$AAP?$AAA?$AAL?$AA_?$AAI?$AAN?$AAD?$AAE?$AAX?$AAE?$AAD?$AA?9?$AA?$DO?$AA?$AN?$AA?6?$AA?$AA@ 10006864     gpe:swconvrt.obj
 0001:00005884       ??_C@_1BK@JHJDPAGP@?$AAX?$AAO?$AA_?$AAT?$AAO?$AA_?$AAM?$AAO?$AAN?$AAO?$AA?$AN?$AA?6?$AA?$AA@ 10006884     gpe:swconvrt.obj
 0001:000058a0       ??_C@_1BG@IMEEDKKI@?$AAX?$AAO?$AA_?$AAT?$AAA?$AAB?$AAL?$AAE?$AA?$AN?$AA?6?$AA?$AA@ 100068a0     gpe:swconvrt.obj
 0001:000058b8       ??_C@_1BK@HJFOLJIA@?$AAP?$AAA?$AAL?$AA_?$AAF?$AAO?$AAU?$AAR?$AAC?$AAC?$AA?$AN?$AA?6?$AA?$AA@ 100068b8     gpe:swconvrt.obj
 0001:000058d4       ??_C@_1BK@EGBOMKOJ@?$AAX?$AAO?$AA_?$AAT?$AAR?$AAI?$AAV?$AAI?$AAA?$AAL?$AA?$AN?$AA?6?$AA?$AA@ 100068d4     gpe:swconvrt.obj
 0001:000058f0       ??_C@_1BI@IADKPPBE@?$AAM?$AAa?$AAs?$AAk?$AA?5?$AAI?$AAn?$AAi?$AAt?$AA?$AN?$AA?6?$AA?$AA@ 100068f0     gpe:swconvrt.obj
 0001:00005908       ??_C@_1BK@GOEDNDKO@?$AAG?$AAr?$AAo?$AAu?$AAp?$AA?5?$AAI?$AAn?$AAi?$AAt?$AA?$AN?$AA?6?$AA?$AA@ 10006908     gpe:swconvrt.obj
 0001:00005924       ??_C@_1DA@CCGKDIKL@?$AAP?$AAA?$AAL?$AA_?$AAI?$AAN?$AAD?$AAE?$AAX?$AAE?$AAD?$AA?9?$AA?$DO?$AAm?$AAa?$AAs?$AAk?$AA?1?$AAr?$AAg?$AAb?$AA?$AN?$AA?6?$AA?$AA@ 10006924     gpe:swconvrt.obj
 0001:00005954       ??_C@_1DG@NNLJNGCO@?$AAP?$AAA?$AAL?$AA_?$AAI?$AAN?$AAD?$AAE?$AAX?$AAE?$AAD?$AA?9?$AA?$DO?$AAP?$AAA?$AAL?$AA_?$AAI?$AAN?$AAD?$AAE?$AAX?$AAE?$AAD?$AA?$AN?$AA?6?$AA?$AA@ 10006954     gpe:swconvrt.obj
 0001:000059b0       ??_C@_1HG@OPIKMHCE@?$AAX?$AA?0?$AAY?$AA?$DN?$AA?$CF?$AAd?$AA?0?$AA?$CF?$AAd?$AA?5?$AAd?$AAM?$AA?0?$AAd?$AAN?$AA?$DN?$AA?$CF?$AAd?$AA?0?$AA?$CF?$AAd?$AA?5?$AAl?$AAl?$AAG?$AAa?$AAm?$AAm?$AAa?$AA?$DN?$AA?$CF?$AAd@ 100069b0     gpe:drvstrok.obj
 0001:00005a28       ??_C@_1BE@GGDHIBHC@?$AAy?$AA1?$AA?5?$AA?$DN?$AA?5?$AA?$CF?$AAd?$AA?$AN?$AA?6?$AA?$AA@ 10006a28     gpe:drvstrok.obj
 0001:00005a3c       ??_C@_1BM@KIBENLGK@?$AAn?$AAe?$AAw?$AA?5?$AAx?$AA0?$AA?5?$AA?$DN?$AA?5?$AA?$CF?$AAd?$AA?$AN?$AA?6?$AA?$AA@ 10006a3c     gpe:drvstrok.obj
 0001:00005a58       ??_C@_1BM@MNHDOACM@?$AAn?$AAe?$AAw?$AA?5?$AAy?$AA0?$AA?5?$AA?$DN?$AA?5?$AA?$CF?$AAd?$AA?$AN?$AA?6?$AA?$AA@ 10006a58     gpe:drvstrok.obj
 0001:00005a74       ??_C@_1DC@PBLIICNO@?$AAH?$AAo?$AAr?$AAi?$AAz?$AAo?$AAn?$AAt?$AAa?$AAl?$AA?5?$AAo?$AAr?$AA?5?$AAV?$AAe?$AAr?$AAt?$AAi?$AAc?$AAa?$AAl?$AA?$AN?$AA?6?$AA?$AA@ 10006a74     gpe:drvstrok.obj
 0001:00005aa8       ??_C@_1IK@EIAPFKN@?$AAx?$AA0?$AA?0?$AAy?$AA0?$AA?$DN?$AA?$CF?$AAd?$AA?0?$AA?$CF?$AAd?$AA?5?$AAx?$AA1?$AA?$DN?$AA?$CF?$AAd?$AA?4?$AA?5?$AAC?$AAl?$AAi?$AAp?$AA?3?$AA?5?$AA?$CF?$AAd?$AA?0?$AA?$CF?$AAd?$AA?5?$AA?9@ 10006aa8     gpe:drvstrok.obj
 0001:00005b38       ??_C@_1EK@BLKIOAOH@?$AAL?$AAi?$AAn?$AAe?$AA?5?$AAS?$AAe?$AAg?$AA?5?$AA?$CF?$AAd?$AA?4?$AA?$CF?$AAd?$AA?0?$AA?$CF?$AAd?$AA?4?$AA?$CF?$AAd?$AA?5?$AA?9?$AA?5?$AA?$CF?$AAd?$AA?4?$AA?$CF?$AAd?$AA?0?$AA?$CF?$AAd?$AA?4@ 10006b38     gpe:drvstrok.obj
 0001:00005b88       ??_C@_1FC@MJBJPEOD@?$AAD?$AAr?$AAv?$AAS?$AAt?$AAr?$AAo?$AAk?$AAe?$AAP?$AAa?$AAt?$AAh?$AA?3?$AA?5?$AAc?$AAo?$AAm?$AAp?$AAl?$AAe?$AAx?$AA?5?$AAc?$AAl?$AAi?$AAp?$AAp?$AAi?$AAn?$AAg?$AA?5@ 10006b88     gpe:drvstrok.obj
 0001:00005be0       ??_C@_1FG@HACCPIID@?$AAD?$AAr?$AAv?$AAS?$AAt?$AAr?$AAo?$AAk?$AAe?$AAP?$AAa?$AAt?$AAh?$AA?3?$AA?5?$AAs?$AAi?$AAn?$AAg?$AAl?$AAe?$AA?5?$AA?$CI?$AAD?$AAC?$AA_?$AAR?$AAE?$AAC?$AAT?$AA?$CJ?$AA?5@ 10006be0     gpe:drvstrok.obj
 0001:00005c38       ??_C@_1DK@NNIGLIJC@?$AAD?$AAr?$AAv?$AAS?$AAt?$AAr?$AAo?$AAk?$AAe?$AAP?$AAa?$AAt?$AAh?$AA?3?$AA?5?$AAn?$AAo?$AA?5?$AAc?$AAl?$AAi?$AAp?$AAp?$AAi?$AAn?$AAg?$AA?$AN?$AA?6?$AA?$AA@ 10006c38     gpe:drvstrok.obj
 0001:00005c74       ??_C@_1DA@MJEICNOF@?$AAL?$AAe?$AAa?$AAv?$AAi?$AAn?$AAg?$AA?5?$AAD?$AAr?$AAv?$AAS?$AAt?$AAr?$AAo?$AAk?$AAe?$AAP?$AAa?$AAt?$AAh?$AA?$AN?$AA?6?$AA?$AA@ 10006c74     gpe:drvstrok.obj
 0001:00005ca4       ??_C@_1DM@GOMBKNFO@?$AAC?$AAa?$AAl?$AAl?$AAi?$AAn?$AAg?$AA?5?$AAG?$AAP?$AAE?$AA?3?$AA?3?$AAL?$AAi?$AAn?$AAe?$AA?5?$AA?$FL?$AAp?$AAr?$AAe?$AAp?$AAa?$AAr?$AAe?$AA?$FN?$AA?$AN?$AA?6?$AA?$AA@ 10006ca4     gpe:drvstrok.obj
 0001:00005ce0       ??_C@_1DI@EKIJDMNL@?$AAM?$AAi?$AAx?$AA?3?$AA?$CF?$AA0?$AA4?$AAx?$AA?5?$AAL?$AAi?$AAn?$AAe?$AA?5?$AAc?$AAo?$AAl?$AAo?$AAr?$AA?3?$AA?5?$AA?$CF?$AA0?$AA8?$AAx?$AA?$AN?$AA?6?$AA?$AA@ 10006ce0     gpe:drvstrok.obj
 0001:00005d18       ??_C@_1DC@GKEIMHIE@?$AAE?$AAn?$AAt?$AAe?$AAr?$AAi?$AAn?$AAg?$AA?5?$AAD?$AAr?$AAv?$AAS?$AAt?$AAr?$AAo?$AAk?$AAe?$AAP?$AAa?$AAt?$AAh?$AA?$AN?$AA?6?$AA?$AA@ 10006d18     gpe:drvstrok.obj
 0001:00005da8       ??_C@_1CA@MEKIGAL@?$AAA?$AAA?$AAT?$AAe?$AAx?$AAt?$AAB?$AAl?$AAt?$AAD?$AAs?$AAt?$AA8?$AA?$AN?$AA?6?$AA?$AA@ 10006da8     gpe:aablt.obj
 0001:00005dc8       ??_C@_1FM@KBOMGCJC@?$AAD?$AAB?$AAG?$AAC?$AAH?$AAK?$AA_?$AAR?$AAE?$AAT?$AAA?$AAI?$AAL?$AA?5?$AAf?$AAa?$AAi?$AAl?$AAe?$AAd?$AA?5?$AAi?$AAn?$AA?5?$AAf?$AAi?$AAl?$AAe?$AA?5?$AA?$CF?$AAs?$AA?5@ 10006dc8     gpe:aablt.obj
 0001:00005e28       ??_C@_1IA@HGJOOBIK@?$AAd?$AA?3?$AA?2?$AAc?$AAh?$AAe?$AAl?$AAa?$AAn?$AAr?$AAt?$AAm?$AA2?$AA?2?$AAp?$AAu?$AAb?$AAl?$AAi?$AAc?$AA?2?$AAc?$AAo?$AAm?$AAm?$AAo?$AAn?$AA?2?$AAo?$AAa?$AAk?$AA?2@ 10006e28     gpe:aablt.obj
 0001:00005ea8       ??_C@_1CC@LBCFEHKJ@?$AAA?$AAA?$AAT?$AAe?$AAx?$AAt?$AAB?$AAl?$AAt?$AAD?$AAs?$AAt?$AA1?$AA6?$AA?$AN?$AA?6?$AA?$AA@ 10006ea8     gpe:aablt.obj
 0001:00005ecc       ??_C@_1CC@DBJKJJGO@?$AAA?$AAA?$AAT?$AAe?$AAx?$AAt?$AAB?$AAl?$AAt?$AAD?$AAs?$AAt?$AA3?$AA2?$AA?$AN?$AA?6?$AA?$AA@ 10006ecc     gpe:aablt.obj
 0001:00005ef0       ??_C@_1DC@KKGHFHAM@?$AAE?$AAn?$AAt?$AAe?$AAr?$AAi?$AAn?$AAg?$AA?5?$AAD?$AAr?$AAv?$AAA?$AAl?$AAp?$AAh?$AAa?$AAB?$AAl?$AAe?$AAn?$AAd?$AA?$AN?$AA?6?$AA?$AA@ 10006ef0     gpe:drvalphablend.obj
 0001:00005f28       ??_C@_1KK@MMPBPABL@?$AAd?$AA?3?$AA?2?$AAc?$AAh?$AAe?$AAl?$AAa?$AAn?$AAr?$AAt?$AAm?$AA2?$AA?2?$AAp?$AAr?$AAi?$AAv?$AAa?$AAt?$AAe?$AA?2?$AAw?$AAi?$AAn?$AAc?$AAe?$AAo?$AAs?$AA?2?$AAc?$AAo@ 10006f28     gpe:rdrvgradfill.obj
 0001:00005fd8       ??_C@_1IG@KACOKOGP@?$AAd?$AA?3?$AA?2?$AAc?$AAh?$AAe?$AAl?$AAa?$AAn?$AAr?$AAt?$AAm?$AA2?$AA?2?$AAp?$AAr?$AAi?$AAv?$AAa?$AAt?$AAe?$AA?2?$AAw?$AAi?$AAn?$AAc?$AAe?$AAo?$AAs?$AA?2?$AAc?$AAo@ 10006fd8     gpe:rctblt.obj
 0001:00006060       ??_C@_1CI@CIALDMNA@?$AAC?$AAl?$AAe?$AAa?$AAr?$AAT?$AAy?$AAp?$AAe?$AAB?$AAl?$AAt?$AAD?$AAs?$AAt?$AA1?$AA6?$AA?$AN?$AA?6?$AA?$AA@ 10007060     gpe:rctblt.obj
 0001:00006088       ??_C@_1CI@IBBJIAKO@?$AAC?$AAl?$AAe?$AAa?$AAr?$AAT?$AAy?$AAp?$AAe?$AAB?$AAl?$AAt?$AAD?$AAs?$AAt?$AA2?$AA4?$AA?$AN?$AA?6?$AA?$AA@ 10007088     gpe:rctblt.obj
 0001:000060b0       ??_C@_1CI@KILEOCBH@?$AAC?$AAl?$AAe?$AAa?$AAr?$AAT?$AAy?$AAp?$AAe?$AAB?$AAl?$AAt?$AAD?$AAs?$AAt?$AA3?$AA2?$AA?$AN?$AA?6?$AA?$AA@ 100070b0     gpe:rctblt.obj
 0001:000060d8       ??_C@_1CG@CEMICPHK@?$AAC?$AAl?$AAe?$AAa?$AAr?$AAT?$AAy?$AAp?$AAe?$AAB?$AAl?$AAt?$AAD?$AAs?$AAt?$AA8?$AA?$AN?$AA?6?$AA?$AA@ 100070d8     gpe:rctblt.obj
 0001:00006100       ??_C@_1GA@EAMBNKKC@?$AAG?$AAP?$AAE?$AA?3?$AA?5?$AA?$CK?$AA?$CK?$AA?5?$AAW?$AAA?$AAR?$AAN?$AAI?$AAN?$AAG?$AA?5?$AA?$CK?$AA?$CK?$AA?5?$AAS?$AAU?$AAR?$AAF?$AAO?$AAB?$AAJ?$AA?4?$AAf?$AAj?$AAB?$AAi?$AAt@ 10007100     gpe:TmpGPESurf.obj
 0001:00006160       ??_C@_1DG@POALGGHB@?$AAL?$AAe?$AAa?$AAv?$AAe?$AA?5?$AAE?$AAd?$AAg?$AAe?$AAL?$AAi?$AAs?$AAt?$AA?3?$AA?3?$AAE?$AAd?$AAg?$AAe?$AAL?$AAi?$AAs?$AAt?$AA?$AN?$AA?6?$AA?$AA@ 10007160     gpe:swfill.obj
 0001:00006198       ??_C@_1DG@HJGHDMIL@?$AAE?$AAn?$AAt?$AAe?$AAr?$AA?5?$AAE?$AAd?$AAg?$AAe?$AAL?$AAi?$AAs?$AAt?$AA?3?$AA?3?$AAE?$AAd?$AAg?$AAe?$AAL?$AAi?$AAs?$AAt?$AA?$AN?$AA?6?$AA?$AA@ 10007198     gpe:swfill.obj
 0001:000061d0       ??_C@_1DI@OKEGJBNP@?$AAL?$AAe?$AAa?$AAv?$AAe?$AA?5?$AAE?$AAd?$AAg?$AAe?$AAL?$AAi?$AAs?$AAt?$AA?3?$AA?3?$AA?$HO?$AAE?$AAd?$AAg?$AAe?$AAL?$AAi?$AAs?$AAt?$AA?$AN?$AA?6?$AA?$AA@ 100071d0     gpe:swfill.obj
 0001:00006208       ??_C@_1DI@IPKLKHGO@?$AAE?$AAn?$AAt?$AAe?$AAr?$AA?5?$AAE?$AAd?$AAg?$AAe?$AAL?$AAi?$AAs?$AAt?$AA?3?$AA?3?$AA?$HO?$AAE?$AAd?$AAg?$AAe?$AAL?$AAi?$AAs?$AAt?$AA?$AN?$AA?6?$AA?$AA@ 10007208     gpe:swfill.obj
 0001:00006240       ??_C@_1DE@EGJMFFPM@?$AAL?$AAe?$AAa?$AAv?$AAe?$AA?5?$AAE?$AAd?$AAg?$AAe?$AAL?$AAi?$AAs?$AAt?$AA?3?$AA?3?$AAA?$AAd?$AAd?$AAE?$AAd?$AAg?$AAe?$AA?$AN?$AA?6?$AA?$AA@ 10007240     gpe:swfill.obj
 0001:00006274       ??_C@_1DI@BBHJIBNH@?$AAA?$AAb?$AAa?$AAn?$AAd?$AAo?$AAn?$AAi?$AAn?$AAg?$AA?5?$AAe?$AAd?$AAg?$AAe?$AA?5?$AAw?$AAi?$AAt?$AAh?$AA?5?$AAd?$AAY?$AA?$DN?$AA0?$AA?$AN?$AA?6?$AA?$AA@ 10007274     gpe:swfill.obj
 0001:000062b0       ??_C@_1EG@HPNIEEJM@?$AAE?$AAd?$AAg?$AAe?$AAL?$AAi?$AAs?$AAt?$AA?3?$AA?3?$AAA?$AAd?$AAd?$AAE?$AAd?$AAg?$AAe?$AA?5?$AAr?$AAe?$AAa?$AAl?$AAl?$AAo?$AAc?$AA?5?$AAf?$AAa?$AAi?$AAl?$AAe?$AAd@ 100072b0     gpe:swfill.obj
 0001:000062f8       ??_C@_1DE@NEBMAEOF@?$AAE?$AAn?$AAt?$AAe?$AAr?$AA?5?$AAE?$AAd?$AAg?$AAe?$AAL?$AAi?$AAs?$AAt?$AA?3?$AA?3?$AAA?$AAd?$AAd?$AAE?$AAd?$AAg?$AAe?$AA?$AN?$AA?6?$AA?$AA@ 100072f8     gpe:swfill.obj
 0001:0000632c       ??_C@_1CO@JGOEHONL@?$AAL?$AAe?$AAa?$AAv?$AAe?$AA?5?$AAE?$AAd?$AAg?$AAe?$AAL?$AAi?$AAs?$AAt?$AA?3?$AA?3?$AAF?$AAi?$AAl?$AAl?$AA?$AN?$AA?6?$AA?$AA@ 1000732c     gpe:swfill.obj
 0001:0000635c       ??_C@_1CK@MNNLHIFO@?$AAI?$AAn?$AAc?$AAr?$AAe?$AAm?$AAe?$AAn?$AAt?$AAi?$AAn?$AAg?$AA?5?$AAe?$AAd?$AAg?$AAe?$AAs?$AA?$AN?$AA?6?$AA?$AA@ 1000735c     gpe:swfill.obj
 0001:00006388       ??_C@_1CM@MCMADKNN@?$AAx?$AAL?$AAe?$AAf?$AAt?$AA?$DN?$AA?$CF?$AAd?$AA?0?$AA?5?$AAx?$AAR?$AAi?$AAg?$AAh?$AAt?$AA?$DN?$AA?$CF?$AAd?$AA?$AN?$AA?6?$AA?$AA@ 10007388     gpe:swfill.obj
 0001:000063b8       ??_C@_1FE@BKIFFFBC@?$AAU?$AAn?$AAm?$AAa?$AAt?$AAc?$AAh?$AAe?$AAd?$AA?5?$AAl?$AAi?$AAn?$AAe?$AA?5?$AAs?$AAe?$AAg?$AAm?$AAe?$AAn?$AAt?$AA?5?$AAi?$AAn?$AA?5?$AAp?$AAo?$AAl?$AAy?$AAg?$AAo@ 100073b8     gpe:swfill.obj
 0001:0000640c       ??_C@_1CG@CEBNFAFO@?$AAD?$AAr?$AAa?$AAw?$AAi?$AAn?$AAg?$AA?5?$AAr?$AAo?$AAw?$AA?5?$AAy?$AA?$DN?$AA?$CF?$AAd?$AA?$AN?$AA?6?$AA?$AA@ 1000740c     gpe:swfill.obj
 0001:00006434       ??_C@_1DE@IIMGOPAA@?$AAB?$AAu?$AAb?$AAb?$AAl?$AAe?$AA?5?$AAs?$AAo?$AAr?$AAt?$AA?5?$AAa?$AAc?$AAt?$AAi?$AAv?$AAe?$AA?5?$AAl?$AAi?$AAs?$AAt?$AA?$AN?$AA?6?$AA?$AA@ 10007434     gpe:swfill.obj
 0001:00006468       ??_C@_1DO@BIFCGODE@?$AAR?$AAe?$AAm?$AAo?$AAv?$AAe?$AA?5?$AAe?$AAd?$AAg?$AAe?$AA?5?$AAf?$AAr?$AAo?$AAm?$AA?5?$AAa?$AAc?$AAt?$AAi?$AAv?$AAe?$AA?5?$AAl?$AAi?$AAs?$AAt?$AA?$AN?$AA?6?$AA?$AA@ 10007468     gpe:swfill.obj
 0001:000064a8       ??_C@_1DE@IBPEEOBG@?$AAA?$AAd?$AAd?$AA?5?$AAe?$AAd?$AAg?$AAe?$AA?5?$AAt?$AAo?$AA?5?$AAa?$AAc?$AAt?$AAi?$AAv?$AAe?$AA?5?$AAl?$AAi?$AAs?$AAt?$AA?$AN?$AA?6?$AA?$AA@ 100074a8     gpe:swfill.obj
 0001:000064dc       ??_C@_1CG@NKADCMCI@?$AAP?$AAr?$AAo?$AAc?$AAe?$AAs?$AAs?$AA?5?$AAr?$AAo?$AAw?$AA?5?$AAy?$AA?$DN?$AA?$CF?$AAd?$AA?$AN?$AA?6?$AA?$AA@ 100074dc     gpe:swfill.obj
 0001:00006504       ??_C@_1CO@IDCHHKD@?$AAy?$AAM?$AAi?$AAn?$AA?5?$AA?$DN?$AA?5?$AA?$CF?$AAd?$AA?0?$AA?5?$AAy?$AAM?$AAa?$AAx?$AA?5?$AA?$DN?$AA?5?$AA?$CF?$AAd?$AA?$AN?$AA?6?$AA?$AA@ 10007504     gpe:swfill.obj
 0001:00006538       ??_C@_1HM@DHIIKPMK@?$AAI?$AAn?$AAs?$AAe?$AAr?$AAt?$AAi?$AAn?$AAg?$AA?5?$AAe?$AAd?$AAg?$AAe?$AA?5?$AA?$CF?$AAd?$AA?5?$AA?$CI?$AAy?$AAT?$AAo?$AAp?$AA?$DN?$AA?$CF?$AAd?$AA?0?$AAy?$AAB?$AAo?$AAt?$AAt@ 10007538     gpe:swfill.obj
 0001:000065b4       ??_C@_1CO@HDAAPBGJ@?$AAE?$AAn?$AAt?$AAe?$AAr?$AA?5?$AAE?$AAd?$AAg?$AAe?$AAL?$AAi?$AAs?$AAt?$AA?3?$AA?3?$AAF?$AAi?$AAl?$AAl?$AA?$AN?$AA?6?$AA?$AA@ 100075b4     gpe:swfill.obj
 0001:0000f840       ??_C@_1KA@PNMHOICO@?$AAG?$AAe?$AAn?$AAe?$AAr?$AAa?$AAt?$AAe?$AAd?$AAB?$AAl?$AAt?$AA?3?$AA?5?$AAC?$AAl?$AAo?$AAc?$AAk?$AAO?$AAv?$AAe?$AAr?$AAf?$AAl?$AAo?$AAw?$AA?$CI?$AA?$CJ?$AA?5?$AA?9?$AA?5@ 10010840     gpe:genblt.obj
 0001:0000f8e0       ??_C@_1JC@PAKJCNIJ@?$AAd?$AA?3?$AA?2?$AAc?$AAh?$AAe?$AAl?$AAa?$AAn?$AAr?$AAt?$AAm?$AA2?$AA?2?$AAp?$AAu?$AAb?$AAl?$AAi?$AAc?$AA?2?$AAc?$AAo?$AAm?$AAm?$AAo?$AAn?$AA?2?$AAo?$AAa?$AAk?$AA?2@ 100108e0     gpe:genblt.obj
 0001:0000f978       ??_C@_1JI@GBIAEMHL@?$AAd?$AA?3?$AA?2?$AAc?$AAh?$AAe?$AAl?$AAa?$AAn?$AAr?$AAt?$AAm?$AA2?$AA?2?$AAp?$AAu?$AAb?$AAl?$AAi?$AAc?$AA?2?$AAc?$AAo?$AAm?$AAm?$AAo?$AAn?$AA?2?$AAo?$AAa?$AAk?$AA?2@ 10010978     gpe:GenBltGpe.obj
 0001:0000fac4       ??_C@_1CK@BNNKDGEF@?$AAp?$AAD?$AAs?$AAt?$AA?5?$AAd?$AAe?$AAp?$AAt?$AAh?$AA?3?$AA?5?$AA1?$AA6?$AA?5?$AAB?$AAp?$AAp?$AA?$AN?$AA?6?$AA?$AA@ 10010ac4     gpe:FastBlt.obj
 0001:0000faf0       ??_C@_1CK@PCJMFNDP@?$AAp?$AAS?$AAr?$AAc?$AA?5?$AAd?$AAe?$AAp?$AAt?$AAh?$AA?3?$AA?5?$AA3?$AA2?$AA?5?$AAB?$AAp?$AAp?$AA?$AN?$AA?6?$AA?$AA@ 10010af0     gpe:FastBlt.obj
 0001:0000fb1c       ??_C@_1DG@KMEKFPAI@?$AAp?$AAS?$AAr?$AAc?$AA?$DN?$AA0?$AAx?$AA?$CF?$AA0?$AA8?$AAx?$AA?0?$AA?5?$AAp?$AAD?$AAs?$AAt?$AA?$DN?$AA0?$AAx?$AA?$CF?$AA0?$AA8?$AAx?$AA?$AN?$AA?6?$AA?$AA@ 10010b1c     gpe:FastBlt.obj
 0001:0000fb58       ??_C@_1IO@OAJCOEON@?$AAd?$AA?3?$AA?2?$AAc?$AAh?$AAe?$AAl?$AAa?$AAn?$AAr?$AAt?$AAm?$AA2?$AA?2?$AAp?$AAu?$AAb?$AAl?$AAi?$AAc?$AA?2?$AAc?$AAo?$AAm?$AAm?$AAo?$AAn?$AA?2?$AAo?$AAa?$AAk?$AA?2@ 10010b58     gpe:FastBlt.obj
 0001:0000fbe8       ??_C@_1BO@PIEKEHOP@?$AAr?$AAe?$AAs?$AAu?$AAu?$AAl?$AAt?$AA?$DN?$AA?$CF?$AA0?$AA4?$AAx?$AA?$AN?$AA?6?$AA?$AA@ 10010be8     gpe:BltHelpers.obj
 0001:0000fc08       ??_C@_1IM@PPGFIDMG@?$AAP?$AAr?$AAo?$AAc?$AAe?$AAs?$AAs?$AA?5?$AAr?$AAo?$AAp?$AA3?$AA?$DN?$AA?$CF?$AA0?$AA2?$AAx?$AA?0?$AA?5?$AAn?$AAu?$AAm?$AAb?$AAi?$AAt?$AAs?$AA?$DN?$AA?$CF?$AAd?$AA?0?$AA?5?$AAp@ 10010c08     gpe:BltHelpers.obj
 0001:0000fc98       ??_C@_1IG@HPBHFIOF@?$AAd?$AA?3?$AA?2?$AAc?$AAh?$AAe?$AAl?$AAa?$AAn?$AAr?$AAt?$AAm?$AA2?$AA?2?$AAp?$AAu?$AAb?$AAl?$AAi?$AAc?$AA?2?$AAc?$AAo?$AAm?$AAm?$AAo?$AAn?$AA?2?$AAo?$AAa?$AAk?$AA?2@ 10010c98     gpe:BltHelpers.obj
 0001:0000fd20       ??_C@_1JG@IHFEPJJL@?$AAP?$AAi?$AAx?$AAe?$AAl?$AAs?$AAP?$AAe?$AAr?$AAR?$AAo?$AAw?$AA?$DN?$AA?$CF?$AAd?$AA?0?$AA?5?$AAR?$AAo?$AAw?$AAs?$AA?$DN?$AA?$CF?$AAd?$AA?0?$AA?5?$AAR?$AAo?$AAw?$AAI?$AAn?$AAi@ 10010d20     gpe:PixelIterator.obj
 0001:0000fdb8       ??_C@_1FK@JMNMFACP@?$AAB?$AAr?$AAu?$AAs?$AAh?$AAP?$AAi?$AAx?$AAe?$AAl?$AAI?$AAt?$AAe?$AAr?$AAa?$AAt?$AAo?$AAr?$AA?3?$AA?3?$AAI?$AAn?$AAi?$AAt?$AAB?$AAr?$AAu?$AAs?$AAh?$AAP?$AAi?$AAx@ 10010db8     gpe:PixelIterator.obj
 0001:0000fe14       ??_C@_1CA@CJBGECGE@?$AAB?$AAu?$AAf?$AAf?$AAe?$AAr?$AA?$DN?$AA0?$AAx?$AA?$CF?$AA0?$AA8?$AAx?$AA?$AN?$AA?6?$AA?$AA@ 10010e14     gpe:PixelIterator.obj
 0001:0000fe38       ??_C@_1HA@GFGACJLF@?$AAM?$AAa?$AAs?$AAk?$AA?$DN?$AA?$CF?$AA0?$AA8?$AAx?$AA?0?$AA?5?$AAC?$AAa?$AAc?$AAh?$AAe?$AAS?$AAt?$AAa?$AAt?$AAe?$AAN?$AAe?$AAw?$AAD?$AAW?$AAo?$AAr?$AAd?$AA?$DN?$AA?$CF?$AA0@ 10010e38     gpe:PixelIterator.obj
 0001:0000fea8       ??_C@_1IG@OCKIDEGK@?$AAB?$AAy?$AAt?$AAe?$AAs?$AAP?$AAe?$AAr?$AAA?$AAc?$AAc?$AAe?$AAs?$AAs?$AA?$DN?$AA?$CF?$AAd?$AA?0?$AAC?$AAa?$AAc?$AAh?$AAe?$AAS?$AAt?$AAa?$AAt?$AAe?$AAN?$AAe?$AAw?$AAR@ 10010ea8     gpe:PixelIterator.obj
 0001:0000ff30       ??_C@_1IG@PGOKLFFN@?$AAP?$AAi?$AAx?$AAe?$AAl?$AAI?$AAt?$AAe?$AAr?$AAa?$AAt?$AAo?$AAr?$AA?3?$AA?3?$AAP?$AAi?$AAx?$AAe?$AAl?$AAI?$AAt?$AAe?$AAr?$AAa?$AAt?$AAo?$AAr?$AA?0?$AA?5?$AAp?$AAr@ 10010f30     gpe:PixelIterator.obj
 0001:0000ffb8       ??_C@_1IM@PNLKIEIC@?$AAd?$AA?3?$AA?2?$AAc?$AAh?$AAe?$AAl?$AAa?$AAn?$AAr?$AAt?$AAm?$AA2?$AA?2?$AAp?$AAu?$AAb?$AAl?$AAi?$AAc?$AA?2?$AAc?$AAo?$AAm?$AAm?$AAo?$AAn?$AA?2?$AAo?$AAa?$AAk?$AA?2@ 10010fb8     gpe:PixelIterator.obj
 0001:00010048       ??_C@_1IE@FKOBOOFK@?$AAG?$AAe?$AAn?$AAB?$AAl?$AAt?$AA?3?$AA?5?$AAA?$AAt?$AAt?$AAe?$AAm?$AAp?$AAt?$AAi?$AAn?$AAg?$AA?5?$AAt?$AAo?$AA?5?$AAu?$AAs?$AAe?$AA?5?$AAA?$AAR?$AAM?$AA?5?$AAs?$AAp@ 10011048     gpe:genblt_arm.obj
 0001:000100d0       ??_C@_1JA@JJHCOPLG@?$AAd?$AA?3?$AA?2?$AAc?$AAh?$AAe?$AAl?$AAa?$AAn?$AAr?$AAt?$AAm?$AA2?$AA?2?$AAp?$AAu?$AAb?$AAl?$AAi?$AAc?$AA?2?$AAc?$AAo?$AAm?$AAm?$AAo?$AAn?$AA?2?$AAo?$AAa?$AAk?$AA?2@ 100110d0     gpe:parse.obj
 0001:00010160       ??_C@_1JG@CKKGJNCI@?$AAd?$AA?3?$AA?2?$AAc?$AAh?$AAe?$AAl?$AAa?$AAn?$AAr?$AAt?$AAm?$AA2?$AA?2?$AAp?$AAu?$AAb?$AAl?$AAi?$AAc?$AA?2?$AAc?$AAo?$AAm?$AAm?$AAo?$AAn?$AA?2?$AAo?$AAa?$AAk?$AA?2@ 10011160     gpe:InitRegs.obj
 0001:000101f8       ??_C@_1DC@JBNPFEAM@?$AAE?$AAm?$AAu?$AAl?$AAa?$AAt?$AAe?$AAd?$AAB?$AAl?$AAt?$AAA?$AAl?$AAp?$AAh?$AAa?$AAT?$AAe?$AAx?$AAt?$AA0?$AA8?$AA?$AN?$AA?6?$AA?$AA@ 100111f8     gpe:ebalph08.obj
 0001:0001022c       ??_C@_1CI@FNLDAMDN@?$AAE?$AAm?$AAu?$AAl?$AAa?$AAt?$AAe?$AAd?$AAB?$AAl?$AAt?$AAT?$AAe?$AAx?$AAt?$AA0?$AA8?$AA?$AN?$AA?6?$AA?$AA@ 1001122c     gpe:ebtext08.obj
 0001:00010254       ??_C@_1CG@OBEKLLDK@?$AAE?$AAx?$AAp?$AAe?$AAn?$AAs?$AAi?$AAv?$AAe?$AAA?$AAn?$AAt?$AAi?$AAa?$AAl?$AAi?$AAa?$AAs?$AA?$AA@ 10011254     gpe:ebalph16.obj
 0001:0001027c       ??_C@_1BG@FOPGPEPM@?$AAS?$AAy?$AAs?$AAt?$AAe?$AAm?$AA?2?$AAG?$AAD?$AAI?$AA?$AA@ 1001127c     gpe:ebalph16.obj
 0001:00010294       ??_C@_1DC@GLJHCNAA@?$AAE?$AAm?$AAu?$AAl?$AAa?$AAt?$AAe?$AAd?$AAB?$AAl?$AAt?$AAA?$AAl?$AAp?$AAh?$AAa?$AAT?$AAe?$AAx?$AAt?$AA1?$AA6?$AA?$AN?$AA?6?$AA?$AA@ 10011294     gpe:ebalph16.obj
 0001:000102c8       ??_C@_1CI@KHPLHFDB@?$AAE?$AAm?$AAu?$AAl?$AAa?$AAt?$AAe?$AAd?$AAB?$AAl?$AAt?$AAT?$AAe?$AAx?$AAt?$AA1?$AA6?$AA?$AN?$AA?6?$AA?$AA@ 100112c8     gpe:ebtext16.obj
 0001:000102f0       ??_C@_1CI@FOKELJBH@?$AAE?$AAm?$AAu?$AAl?$AAa?$AAt?$AAe?$AAd?$AAB?$AAl?$AAt?$AAF?$AAi?$AAl?$AAl?$AA1?$AA6?$AA?$AN?$AA?6?$AA?$AA@ 100112f0     gpe:ebfill16.obj
 0001:00010318       ??_C@_1CI@NOBLGHNA@?$AAE?$AAm?$AAu?$AAl?$AAa?$AAt?$AAe?$AAd?$AAB?$AAl?$AAt?$AAF?$AAi?$AAl?$AAl?$AA3?$AA2?$AA?$AN?$AA?6?$AA?$AA@ 10011318     gpe:EmulatedBltFill32.obj
 0001:000103f4       ??_C@_1DO@JLNKMIKB@?$AAM?$AAX?$AAD?$AAD?$AAL?$AAc?$AAd?$AAc?$AA?5?$AAb?$AAu?$AAi?$AAl?$AAd?$AAD?$AAD?$AAH?$AAA?$AAL?$AAI?$AAn?$AAf?$AAo?$AA?3?$AA?5?$AA?$DM?$AA?$DN?$AA?$DN?$AA?$AN?$AA?6?$AA?$AA@ 100113f4     lcdc_common_topaz_v1:halcaps.obj
 0001:00010434       ??_C@_1CA@PJINHLOP@?$AAg?$AAp?$AAV?$AAi?$AAd?$AAM?$AAe?$AAm?$AA?$DN?$AA?$CF?$AA0?$AA8?$AAx?$AA?$AN?$AA?6?$AA?$AA@ 10011434     lcdc_common_topaz_v1:halcaps.obj
 0001:00010458       ??_C@_1GM@OHFGMNEL@?$AAG?$AAe?$AAt?$AAP?$AAh?$AAy?$AAs?$AAi?$AAc?$AAa?$AAl?$AAV?$AAi?$AAd?$AAe?$AAo?$AAM?$AAe?$AAm?$AAo?$AAr?$AAy?$AA?5?$AAr?$AAe?$AAt?$AAu?$AAr?$AAn?$AAe?$AAd?$AA?5@ 10011458     lcdc_common_topaz_v1:halcaps.obj
 0001:000104c4       ??_C@_1DO@IOPAIDCN@?$AAM?$AAX?$AAD?$AAD?$AAL?$AAc?$AAd?$AAc?$AA?5?$AAb?$AAu?$AAi?$AAl?$AAd?$AAD?$AAD?$AAH?$AAA?$AAL?$AAI?$AAn?$AAf?$AAo?$AA?3?$AA?5?$AA?$DN?$AA?$DN?$AA?$DO?$AA?$AN?$AA?6?$AA?$AA@ 100114c4     lcdc_common_topaz_v1:halcaps.obj
 0001:000105c0       ??_C@_1EM@BDLCICKK@?$AAH?$AAa?$AAl?$AAC?$AAr?$AAe?$AAa?$AAt?$AAe?$AAS?$AAu?$AAr?$AAf?$AAa?$AAc?$AAe?$AA?3?$AA?5?$AAs?$AAu?$AAr?$AAf?$AAa?$AAc?$AAe?$AA?5?$AAc?$AAr?$AAe?$AAa?$AAt?$AAe@ 100115c0     lcdc_common_topaz_v1:halsurf.obj
 0001:00010610       ??_C@_1FI@CIJNIDAF@?$AAH?$AAa?$AAl?$AAC?$AAr?$AAe?$AAa?$AAt?$AAe?$AAS?$AAu?$AAr?$AAf?$AAa?$AAc?$AAe?$AA?3?$AA?5?$AAN?$AAO?$AA?5?$AAL?$AAO?$AAC?$AAA?$AAL?$AA?5?$AAH?$AAE?$AAA?$AAP?$AA?5@ 10011610     lcdc_common_topaz_v1:halsurf.obj
 0001:00010668       ??_C@_1CC@CAKAKBFN@?$AAH?$AAa?$AAl?$AAC?$AAr?$AAe?$AAa?$AAt?$AAe?$AAS?$AAu?$AAr?$AAf?$AAa?$AAc?$AAe?$AA?$AA@ 10011668     lcdc_common_topaz_v1:halsurf.obj
 0001:00010690       ??_C@_1EG@NFEJGPCN@?$AAH?$AAa?$AAl?$AAC?$AAa?$AAn?$AAC?$AAr?$AAe?$AAa?$AAt?$AAe?$AAS?$AAu?$AAr?$AAf?$AAa?$AAc?$AAe?$AA?3?$AA?5?$AAU?$AAn?$AAs?$AAu?$AAp?$AAp?$AAo?$AAr?$AAt?$AAe?$AAd@ 10011690     lcdc_common_topaz_v1:halsurf.obj
 0001:000106d8       ??_C@_1DE@MIGPICBH@?$AAH?$AAa?$AAl?$AAC?$AAa?$AAn?$AAC?$AAr?$AAe?$AAa?$AAt?$AAe?$AAS?$AAu?$AAr?$AAf?$AAa?$AAc?$AAe?$AA?3?$AA?5?$AAO?$AAK?$AA?$AN?$AA?6?$AA?$AA@ 100116d8     lcdc_common_topaz_v1:halsurf.obj
 0001:00010710       ??_C@_1II@BELLBNIO@?$AAH?$AAa?$AAl?$AAC?$AAa?$AAn?$AAC?$AAr?$AAe?$AAa?$AAt?$AAe?$AAS?$AAu?$AAr?$AAf?$AAa?$AAc?$AAe?$AA?3?$AA?5?$AAt?$AAh?$AAe?$AA?5?$AAr?$AAe?$AAq?$AAu?$AAe?$AAs?$AAt@ 10011710     lcdc_common_topaz_v1:halsurf.obj
 0001:00010798       ??_C@_1CI@JJDELMEE@?$AAH?$AAa?$AAl?$AAC?$AAa?$AAn?$AAC?$AAr?$AAe?$AAa?$AAt?$AAe?$AAS?$AAu?$AAr?$AAf?$AAa?$AAc?$AAe?$AA?$AA@ 10011798     lcdc_common_topaz_v1:halsurf.obj
 0001:000107c0       ??_C@_1CA@DJNNJENL@?$AAH?$AAa?$AAl?$AAG?$AAe?$AAt?$AAB?$AAl?$AAt?$AAS?$AAt?$AAa?$AAt?$AAu?$AAs?$AA?$AA@ 100117c0     lcdc_common_topaz_v1:halsurf.obj
 0001:000107e0       ??_C@_1CC@NIPOBBK@?$AAH?$AAa?$AAl?$AAU?$AAp?$AAd?$AAa?$AAt?$AAe?$AAO?$AAv?$AAe?$AAr?$AAl?$AAa?$AAy?$AA?$AA@ 100117e0     lcdc_common_topaz_v1:halsurf.obj
 0001:00010804       ??_C@_1CM@HBIEIICL@?$AAH?$AAa?$AAl?$AAS?$AAe?$AAt?$AAO?$AAv?$AAe?$AAr?$AAl?$AAa?$AAy?$AAP?$AAo?$AAs?$AAi?$AAt?$AAi?$AAo?$AAn?$AA?$AA@ 10011804     lcdc_common_topaz_v1:halsurf.obj
 0001:000108e4       ??_C@_1DG@JNICDHMN@?$AAG?$AAe?$AAt?$AAD?$AAr?$AAi?$AAv?$AAe?$AAr?$AAI?$AAn?$AAf?$AAo?$AA?5?$AAi?$AAn?$AAv?$AAo?$AAk?$AAe?$AAd?$AA?5?$AA?$CB?$AA?$CB?$AA?$AN?$AA?6?$AA?$AA@ 100118e4     lcdc_common_topaz_v1:haldd.obj
 0001:0001091c       ??_C@_1DA@KJGICEF@?$AAH?$AAa?$AAl?$AAW?$AAa?$AAi?$AAt?$AAF?$AAo?$AAr?$AAV?$AAe?$AAr?$AAt?$AAi?$AAc?$AAa?$AAl?$AAB?$AAl?$AAa?$AAn?$AAk?$AA?$AA@ 1001191c     lcdc_common_topaz_v1:haldd.obj
 0001:00010a04       ??_C@_15JNBOKNOG@?$AA?$AN?$AA?6?$AA?$AA@ 10011a04     ddgpe:ddhsurf.obj
 0001:00010a0c       ??_C@_1CE@LLCIAJPO@?$AAD?$AAD?$AAS?$AAC?$AAA?$AAP?$AAS?$AA_?$AAD?$AAY?$AAN?$AAA?$AAM?$AAI?$AAC?$AA?$DL?$AA?5?$AA?$AA@ 10011a0c     ddgpe:ddhsurf.obj
 0001:00010a30       ??_C@_1DE@BDAPEHOJ@?$AAD?$AAD?$AAS?$AAC?$AAA?$AAP?$AAS?$AA_?$AAN?$AAO?$AAT?$AAU?$AAS?$AAE?$AAR?$AAL?$AAO?$AAC?$AAK?$AAA?$AAB?$AAL?$AAE?$AA?$DL?$AA?5?$AA?$AA@ 10011a30     ddgpe:ddhsurf.obj
 0001:00010a64       ??_C@_1DM@NJCJAIKB@?$AAD?$AAD?$AAS?$AAC?$AAA?$AAP?$AAS?$AA_?$AAH?$AAA?$AAR?$AAD?$AAW?$AAA?$AAR?$AAE?$AAD?$AAE?$AAI?$AAN?$AAT?$AAE?$AAR?$AAL?$AAA?$AAC?$AAE?$AA?$DL?$AA?5?$AA?$AA@ 10011a64     ddgpe:ddhsurf.obj
 0001:00010aa0       ??_C@_1CG@KICDLMMB@?$AAD?$AAD?$AAS?$AAC?$AAA?$AAP?$AAS?$AA_?$AAR?$AAE?$AAA?$AAD?$AAO?$AAN?$AAL?$AAY?$AA?$DL?$AA?5?$AA?$AA@ 10011aa0     ddgpe:ddhsurf.obj
 0001:00010ac8       ??_C@_1CI@LKLFFDLA@?$AAD?$AAD?$AAS?$AAC?$AAA?$AAP?$AAS?$AA_?$AAV?$AAI?$AAD?$AAE?$AAO?$AAP?$AAO?$AAR?$AAT?$AA?$DL?$AA?5?$AA?$AA@ 10011ac8     ddgpe:ddhsurf.obj
 0001:00010af0       ??_C@_1CI@JIKOMBJB@?$AAD?$AAD?$AAS?$AAC?$AAA?$AAP?$AAS?$AA_?$AAW?$AAR?$AAI?$AAT?$AAE?$AAO?$AAN?$AAL?$AAY?$AA?$DL?$AA?5?$AA?$AA@ 10011af0     ddgpe:ddhsurf.obj
 0001:00010b18       ??_C@_1CE@DHHDMFFM@?$AAD?$AAD?$AAS?$AAC?$AAA?$AAP?$AAS?$AA_?$AAP?$AAA?$AAL?$AAE?$AAT?$AAT?$AAE?$AA?$DL?$AA?5?$AA?$AA@ 10011b18     ddgpe:ddhsurf.obj
 0001:00010b3c       ??_C@_1BO@NKFLFJJD@?$AAD?$AAD?$AAS?$AAC?$AAA?$AAP?$AAS?$AA_?$AAF?$AAL?$AAI?$AAP?$AA?$DL?$AA?5?$AA?$AA@ 10011b3c     ddgpe:ddhsurf.obj
 0001:00010b5c       ??_C@_1CA@OEFJNEOI@?$AAD?$AAD?$AAS?$AAC?$AAA?$AAP?$AAS?$AA_?$AAA?$AAL?$AAP?$AAH?$AAA?$AA?$DL?$AA?5?$AA?$AA@ 10011b5c     ddgpe:ddhsurf.obj
 0001:00010b7c       ??_C@_1CO@JLADJEGD@?$AAD?$AAD?$AAS?$AAC?$AAA?$AAP?$AAS?$AA_?$AAS?$AAY?$AAS?$AAT?$AAE?$AAM?$AAM?$AAE?$AAM?$AAO?$AAR?$AAY?$AA?$DL?$AA?5?$AA?$AA@ 10011b7c     ddgpe:ddhsurf.obj
 0001:00010bac       ??_C@_1CM@PFPLMLPK@?$AAD?$AAD?$AAS?$AAC?$AAA?$AAP?$AAS?$AA_?$AAV?$AAI?$AAD?$AAE?$AAO?$AAM?$AAE?$AAM?$AAO?$AAR?$AAY?$AA?$DL?$AA?5?$AA?$AA@ 10011bac     ddgpe:ddhsurf.obj
 0001:00010bd8       ??_C@_1DC@MIDMCGJH@?$AAD?$AAD?$AAS?$AAC?$AAA?$AAP?$AAS?$AA_?$AAP?$AAR?$AAI?$AAM?$AAA?$AAR?$AAY?$AAS?$AAU?$AAR?$AAF?$AAA?$AAC?$AAE?$AA?$DL?$AA?5?$AA?$AA@ 10011bd8     ddgpe:ddhsurf.obj
 0001:00010c0c       ??_C@_1CK@NOBMKHGC@?$AAD?$AAD?$AAS?$AAC?$AAA?$AAP?$AAS?$AA_?$AAB?$AAA?$AAC?$AAK?$AAB?$AAU?$AAF?$AAF?$AAE?$AAR?$AA?$DL?$AA?5?$AA?$AA@ 10011c0c     ddgpe:ddhsurf.obj
 0001:00010c38       ??_C@_1CM@GBMFLCNA@?$AAD?$AAD?$AAS?$AAC?$AAA?$AAP?$AAS?$AA_?$AAF?$AAR?$AAO?$AAN?$AAT?$AAB?$AAU?$AAF?$AAF?$AAE?$AAR?$AA?$DL?$AA?5?$AA?$AA@ 10011c38     ddgpe:ddhsurf.obj
 0001:00010c64       ??_C@_1CE@FKCECFJM@?$AAD?$AAD?$AAS?$AAC?$AAA?$AAP?$AAS?$AA_?$AAO?$AAV?$AAE?$AAR?$AAL?$AAA?$AAY?$AA?$DL?$AA?5?$AA?$AA@ 10011c64     ddgpe:ddhsurf.obj
 0001:00010c88       ??_C@_1CC@DGPFAEKC@?$AAD?$AAD?$AAG?$AAP?$AAE?$AAS?$AAe?$AAt?$AAC?$AAo?$AAl?$AAo?$AAr?$AAK?$AAe?$AAy?$AA?$AA@ 10011c88     ddgpe:ddhsurf.obj
 0001:00010cb0       ??_C@_1IC@IGMONCFG@?$AAD?$AAD?$AAG?$AAP?$AAE?$AAC?$AAa?$AAn?$AAC?$AAr?$AAe?$AAa?$AAt?$AAe?$AAS?$AAu?$AAr?$AAf?$AAa?$AAc?$AAe?$AA?5?$AAE?$AAR?$AAR?$AAO?$AAR?$AA?5?$AA?9?$AA?5?$AAD?$AAD@ 10011cb0     ddgpe:ddhsurf.obj
 0001:00010d34       ??_C@_1CM@IABDLOFC@?$AAD?$AAD?$AAG?$AAP?$AAE?$AAC?$AAa?$AAn?$AAC?$AAr?$AAe?$AAa?$AAt?$AAe?$AAS?$AAu?$AAr?$AAf?$AAa?$AAc?$AAe?$AA?$AA@ 10011d34     ddgpe:ddhsurf.obj
 0001:00010d60       ??_C@_1EM@BDBFKCAB@?$AAF?$AAa?$AAi?$AAl?$AAe?$AAd?$AA?5?$AAt?$AAo?$AA?5?$AAc?$AAr?$AAe?$AAa?$AAt?$AAe?$AA?5?$AAs?$AAu?$AAr?$AAf?$AAa?$AAc?$AAe?$AA?0?$AA?5?$AAs?$AAc?$AA?$DN?$AA0?$AAx?$AA?$CF@ 10011d60     ddgpe:ddhsurf.obj
 0001:00010dac       ??_C@_1CO@DBIDFOEF@?$AAC?$AAr?$AAe?$AAa?$AAt?$AAe?$AA?5?$AAS?$AAu?$AAr?$AAf?$AAa?$AAc?$AAe?$AA?5?$AAf?$AAl?$AAa?$AAg?$AAs?$AA?3?$AA?5?$AA?$AA@ 10011dac     ddgpe:ddhsurf.obj
 0001:00010de0       ??_C@_1EG@FLNAHEAB@?$AAN?$AAu?$AAm?$AAb?$AAe?$AAr?$AA?5?$AAo?$AAf?$AA?5?$AAs?$AAu?$AAr?$AAf?$AAa?$AAc?$AAe?$AAs?$AA?5?$AAt?$AAo?$AA?5?$AAc?$AAr?$AAe?$AAa?$AAt?$AAe?$AA?3?$AA?5?$AA?$CF?$AAd@ 10011de0     ddgpe:ddhsurf.obj
 0001:00010e28       ??_C@_1HM@FIMALGJN@?$AAD?$AAD?$AAG?$AAP?$AAE?$AAC?$AAr?$AAe?$AAa?$AAt?$AAe?$AAS?$AAu?$AAr?$AAf?$AAa?$AAc?$AAe?$AA?5?$AAE?$AAR?$AAR?$AAO?$AAR?$AA?5?$AA?9?$AA?5?$AAD?$AAD?$AAE?$AAR?$AAR@ 10011e28     ddgpe:ddhsurf.obj
 0001:00010ea4       ??_C@_1CG@CBGELKHC@?$AAD?$AAD?$AAG?$AAP?$AAE?$AAC?$AAr?$AAe?$AAa?$AAt?$AAe?$AAS?$AAu?$AAr?$AAf?$AAa?$AAc?$AAe?$AA?$AA@ 10011ea4     ddgpe:ddhsurf.obj
 0001:00010ecc       ??_C@_1BE@IJFMNFGG@?$AAD?$AAD?$AAG?$AAP?$AAE?$AAL?$AAo?$AAc?$AAk?$AA?$AA@ 10011ecc     ddgpe:ddhsurf.obj
 0001:00010ee0       ??_C@_1BI@FDCCKBBK@?$AAD?$AAD?$AAG?$AAP?$AAE?$AAU?$AAn?$AAl?$AAo?$AAc?$AAk?$AA?$AA@ 10011ee0     ddgpe:ddhsurf.obj
 0001:00010ef8       ??_C@_1DG@KHKOAKMM@?$AAD?$AAe?$AAs?$AAt?$AAr?$AAo?$AAy?$AA?5?$AAG?$AAP?$AAE?$AAS?$AAu?$AAr?$AAf?$AA?5?$AA?$CK?$AA?3?$AA0?$AAx?$AA?$CF?$AA0?$AA8?$AAx?$AA?$AN?$AA?6?$AA?$AA@ 10011ef8     ddgpe:ddhsurf.obj
 0001:00010f30       ??_C@_1CI@KAAPPIEG@?$AAD?$AAD?$AAG?$AAP?$AAE?$AAD?$AAe?$AAs?$AAt?$AAr?$AAo?$AAy?$AAS?$AAu?$AAr?$AAf?$AAa?$AAc?$AAe?$AA?$AA@ 10011f30     ddgpe:ddhsurf.obj
 0001:00010f58       ??_C@_1BI@CPLCPBAP@?$AAF?$AAl?$AAi?$AAp?$AA?5?$AAd?$AAo?$AAn?$AAe?$AA?$AN?$AA?6?$AA?$AA@ 10011f58     ddgpe:ddhsurf.obj
 0001:00010f70       ??_C@_1EO@NKBIEOCE@?$AAO?$AAf?$AAf?$AAs?$AAe?$AAt?$AAI?$AAn?$AAV?$AAi?$AAd?$AAe?$AAo?$AAM?$AAe?$AAm?$AAo?$AAr?$AAy?$AA?5?$AAi?$AAs?$AA?5?$AA0?$AAx?$AA?$CF?$AA0?$AA8?$AAx?$AA?5?$AA0?$AAx@ 10011f70     ddgpe:ddhsurf.obj
 0001:00010fc0       ??_C@_1EO@HFBDJLNB@?$AAf?$AAp?$AAV?$AAi?$AAd?$AAm?$AAe?$AAm?$AA?5?$AA?5?$AA?5?$AA?5?$AA?5?$AA?5?$AA?5?$AA?5?$AA?5?$AA?5?$AA?5?$AA?5?$AAi?$AAs?$AA?5?$AA0?$AAx?$AA?$CF?$AA0?$AA8?$AAx?$AA?5?$AA0?$AAx@ 10011fc0     ddgpe:ddhsurf.obj
 0001:00011010       ??_C@_1FC@NHPNFNFP@?$AAF?$AAl?$AAi?$AAp?$AAp?$AAi?$AAn?$AAg?$AA?5?$AAf?$AAr?$AAo?$AAm?$AA?5?$AAG?$AAP?$AAE?$AAS?$AAu?$AAr?$AAf?$AA?5?$AA0?$AAx?$AA?$CF?$AA0?$AA8?$AAx?$AA?5?$AAt?$AAo?$AA?5@ 10012010     ddgpe:ddhsurf.obj
 0001:00011064       ??_C@_1BE@DGHCLBLE@?$AAD?$AAD?$AAG?$AAP?$AAE?$AAF?$AAl?$AAi?$AAp?$AA?$AA@ 10012064     ddgpe:ddhsurf.obj
 0001:00011078       ??_C@_1CG@LFNIEIKO@?$AAD?$AAD?$AAG?$AAP?$AAE?$AAG?$AAe?$AAt?$AAF?$AAl?$AAi?$AAp?$AAS?$AAt?$AAa?$AAt?$AAu?$AAs?$AA?$AA@ 10012078     ddgpe:ddhsurf.obj
 0001:000110a0       ??_C@_1CA@CJJKMALA@?$AAD?$AAD?$AAG?$AAP?$AAE?$AAS?$AAe?$AAt?$AAP?$AAa?$AAl?$AAe?$AAt?$AAt?$AAe?$AA?$AA@ 100120a0     ddgpe:ddhsurf.obj
 0001:00011174       ??_C@_1CG@FDCEDFHK@?$AAD?$AAD?$AAG?$AAP?$AAE?$AAC?$AAr?$AAe?$AAa?$AAt?$AAe?$AAP?$AAa?$AAl?$AAe?$AAt?$AAt?$AAe?$AA?$AA@ 10012174     ddgpe:ddhpalette.obj
 0001:0001119c       ??_C@_1CI@NCEPHHEO@?$AAD?$AAD?$AAG?$AAP?$AAE?$AAD?$AAe?$AAs?$AAt?$AAr?$AAo?$AAy?$AAP?$AAa?$AAl?$AAe?$AAt?$AAt?$AAe?$AA?$AA@ 1001219c     ddgpe:ddhpalette.obj
 0001:000111c4       ??_C@_1CA@HGFAGLNK@?$AAD?$AAD?$AAG?$AAP?$AAE?$AAS?$AAe?$AAt?$AAE?$AAn?$AAt?$AAr?$AAi?$AAe?$AAs?$AA?$AA@ 100121c4     ddgpe:ddhpalette.obj
 0001:0001129c       ??_C@_1DE@FAIEGLLN@?$AAD?$AAD?$AAG?$AAP?$AAE?$AAW?$AAa?$AAi?$AAt?$AAF?$AAo?$AAr?$AAV?$AAe?$AAr?$AAt?$AAi?$AAc?$AAa?$AAl?$AAB?$AAl?$AAa?$AAn?$AAk?$AA?$AA@ 1001229c     ddgpe:ddhdd.obj
 0001:00011388       ??_C@_1IM@ENPJGOLP@?$AAD?$AAD?$AAG?$AAP?$AAE?$AAG?$AAe?$AAt?$AAP?$AAi?$AAx?$AAe?$AAl?$AAF?$AAo?$AAr?$AAm?$AAa?$AAt?$AAF?$AAr?$AAo?$AAm?$AAS?$AAu?$AAr?$AAf?$AAa?$AAc?$AAe?$AAD?$AAe@ 10012388     ddgpe:ddhutil.obj
 0001:00011414       ??_C@_1CK@LMDKNKJD@?$AAg?$AAo?$AAt?$AA?5?$AAp?$AAi?$AAx?$AAe?$AAl?$AAF?$AAo?$AAr?$AAm?$AAa?$AAt?$AA?5?$AA?$CF?$AAd?$AA?$AN?$AA?6?$AA?$AA@ 10012414     ddgpe:ddhutil.obj
 0001:00011440       ??_C@_1IA@FDEHJPLB@?$AAD?$AAD?$AAG?$AAP?$AAE?$AAG?$AAe?$AAt?$AAP?$AAi?$AAx?$AAe?$AAl?$AAF?$AAo?$AAr?$AAm?$AAa?$AAt?$AAF?$AAr?$AAo?$AAm?$AAS?$AAu?$AAr?$AAf?$AAa?$AAc?$AAe?$AAD?$AAe@ 10012440     ddgpe:ddhutil.obj
 0001:000114c0       ??_C@_1EG@JPKJEAHM@?$AAD?$AAD?$AAG?$AAP?$AAE?$AAG?$AAe?$AAt?$AAP?$AAi?$AAx?$AAe?$AAl?$AAF?$AAo?$AAr?$AAm?$AAa?$AAt?$AAF?$AAr?$AAo?$AAm?$AAS?$AAu?$AAr?$AAf?$AAa?$AAc?$AAe?$AAD?$AAe@ 100124c0     ddgpe:ddhutil.obj
 0001:0001152c       ?BSPGetModes@@YAPAUGPEMode@@XZ 1001252c f   bsplcdc.obj
 0001:00011550       ?BSPGetModeNum@@YAKXZ      10012550 f   bsplcdc.obj
 0001:00011568       ?BSPGetModeDescriptor@@YAHHPAULCDC_MODE_DESCRIPTOR@@@Z 10012568 f   bsplcdc.obj
 0001:00011664       ?BSPInitLCDC@@YAHXZ        10012664 f   bsplcdc.obj
 0001:00011dd0       ?BSPDeinitLCDC@@YAHPAULCDC_MODE_DESCRIPTOR@@@Z 10012dd0 f   bsplcdc.obj
 0001:00011df4       ?BSPTurnOnDisplay@@YAXPAULCDC_MODE_DESCRIPTOR@@@Z 10012df4 f   bsplcdc.obj
 0001:00011e0c       ?BSPTurnOffDisplay@@YAXPAULCDC_MODE_DESCRIPTOR@@@Z 10012e0c f   bsplcdc.obj
 0001:00011e24       ?BSPPowerOnDisplay@@YAXPAULCDC_MODE_DESCRIPTOR@@@Z 10012e24 f   bsplcdc.obj
 0001:00011e34       ?BSPPowerOffDisplay@@YAXPAULCDC_MODE_DESCRIPTOR@@@Z 10012e34 f   bsplcdc.obj
 0001:00011e44       ?BSPGetVideoMemorySize@@YAKPAULCDC_MODE_DESCRIPTOR@@@Z 10012e44 f   bsplcdc.obj
 0001:00011ff4       ?BSPGetCacheMode@@YAHXZ    10012ff4 f   bsplcdc.obj
 0001:00012284       ?PowerOnLCD@@YAXPAULCDC_MODE_DESCRIPTOR@@@Z 10013284 f   bsplcdc.obj
 0001:00012294       ?PowerOffLCD@@YAXPAULCDC_MODE_DESCRIPTOR@@@Z 10013294 f   bsplcdc.obj
 0001:000122a4       ?PowerOnTVOut@@YAXPAULCDC_MODE_DESCRIPTOR@@@Z 100132a4 f   bsplcdc.obj
 0001:000122b4       ?PowerOffTVOut@@YAXPAULCDC_MODE_DESCRIPTOR@@@Z 100132b4 f   bsplcdc.obj
 0001:00012440       DrvEnableDriver            10013440 f   lcdc_common_topaz_v1:DDLcdc.obj
 0001:0001247c       DrvGetMasks                1001347c f   lcdc_common_topaz_v1:DDLcdc.obj
 0001:00012544       GetGPE                     10013544 f   lcdc_common_topaz_v1:DDLcdc.obj
 0001:000126b8       ??0MXDDLcdc@@QAA@PAH@Z     100136b8 f   lcdc_common_topaz_v1:DDLcdc.obj
 0001:0001289c       ??1MXDDLcdc@@UAA@XZ        1001389c f   lcdc_common_topaz_v1:DDLcdc.obj
 0001:000128cc       ?SetMode@MXDDLcdc@@UAAJHPAPAUHPALETTE__@@@Z 100138cc f   lcdc_common_topaz_v1:DDLcdc.obj
 0001:00013438       ?GetModeInfo@MXDDLcdc@@UAAJPAUGPEMode@@H@Z 10014438 f   lcdc_common_topaz_v1:DDLcdc.obj
 0001:000134f8       ?GetModeInfoEx@MXDDLcdc@@UAAJPAUGPEModeEx@@H@Z 100144f8 f   lcdc_common_topaz_v1:DDLcdc.obj
 0001:000135a8       ?NumModes@MXDDLcdc@@UAAHXZ 100145a8 f   lcdc_common_topaz_v1:DDLcdc.obj
 0001:000135d4       ?GetPhysicalVideoMemory@MXDDLcdc@@UAAXPAK0@Z 100145d4 f   lcdc_common_topaz_v1:DDLcdc.obj
 0001:0001360c       ?GetBpp@MXDDLcdc@@QAAHXZ   1001460c f   lcdc_common_topaz_v1:DDLcdc.obj
 0001:00013638       ?Init@MXDDLcdc@@AAAHXZ     10014638 f   lcdc_common_topaz_v1:DDLcdc.obj
 0001:000138d0       ?ReInit@MXDDLcdc@@AAAHXZ   100148d0 f   lcdc_common_topaz_v1:DDLcdc.obj
 0001:00013ae4       ?InitHardware@MXDDLcdc@@AAAHXZ 10014ae4 f   lcdc_common_topaz_v1:DDLcdc.obj
 0001:00013e94       ?AllocVideoMemory@MXDDLcdc@@AAAHXZ 10014e94 f   lcdc_common_topaz_v1:DDLcdc.obj
 0001:0001430c       ?FreeVideoMemory@MXDDLcdc@@AAAHXZ 1001530c f   lcdc_common_topaz_v1:DDLcdc.obj
 0001:00014418       ?SetRGBQuadPalette@MXDDLcdc@@QAAJPBUtagRGBQUAD@@GG@Z 10015418 f   lcdc_common_topaz_v1:DDLcdc.obj
 0001:0001454c       ?SetPalette@MXDDLcdc@@UAAJPBUtagPALETTEENTRY@@GG@Z 1001554c f   lcdc_common_topaz_v1:DDLcdc.obj
 0001:00014680       ?SetModeHardware@MXDDLcdc@@AAAHH@Z 10015680 f   lcdc_common_topaz_v1:DDLcdc.obj
 0001:00014cc8       ?Cleanup@MXDDLcdc@@AAAXXZ  10015cc8 f   lcdc_common_topaz_v1:DDLcdc.obj
 0001:00014f88       ?IntrProc@MXDDLcdc@@AAAKXZ 10015f88 f   lcdc_common_topaz_v1:DDLcdc.obj
 0001:000150bc       ?MXDDLcdcIntr@@YAKPAVMXDDLcdc@@@Z 100160bc f   lcdc_common_topaz_v1:DDLcdc.obj
 0001:000150e8       ?GetPhysicalModeId@DDGPE@@UAAKXZ 100160e8 f i lcdc_common_topaz_v1:DDLcdc.obj
 0001:00015114       ?GetDriverData@DDGPE@@UAAPAUDDGPEDriverData@@XZ 10016114 f i lcdc_common_topaz_v1:DDLcdc.obj
 0001:00015140       ?SetDriverData@DDGPE@@UAAXPAUDDGPEDriverData@@@Z 10016140 f i lcdc_common_topaz_v1:DDLcdc.obj
 0001:00015160       ?GetGraphicsCaps@MXDDLcdc@@UAAKXZ 10016160 f i lcdc_common_topaz_v1:DDLcdc.obj
 0001:00015188       ??_EMXDDLcdc@@UAAPAXI@Z    10016188 f i lcdc_common_topaz_v1:DDLcdc.obj
 0001:00015188       ??_GMXDDLcdc@@UAAPAXI@Z    10016188 f i lcdc_common_topaz_v1:DDLcdc.obj
 0001:000151c8       ?OffsetInVideoMemory@GPESurf@@QAAKXZ 100161c8 f i lcdc_common_topaz_v1:DDLcdc.obj
 0001:000151f4       SetEvent                   100161f4 f i lcdc_common_topaz_v1:DDLcdc.obj
 0001:00015230       ?AdvertisePowerInterface@MXDDLcdc@@AAAHPAUHINSTANCE__@@@Z 10016230 f   lcdc_common_topaz_v1:DDLcdcPower.obj
 0001:000154d0       ?SetDisplayPower@MXDDLcdc@@AAAXW4_CEDEVICE_POWER_STATE@@@Z 100164d0 f   lcdc_common_topaz_v1:DDLcdcPower.obj
 0001:000156ec       ?PmToVideoPowerState@MXDDLcdc@@AAA?AW4_VIDEO_POWER_STATE@@W4_CEDEVICE_POWER_STATE@@@Z 100166ec f   lcdc_common_topaz_v1:DDLcdcPower.obj
 0001:00015798       ?VideoToPmPowerState@MXDDLcdc@@AAA?AW4_CEDEVICE_POWER_STATE@@W4_VIDEO_POWER_STATE@@@Z 10016798 f   lcdc_common_topaz_v1:DDLcdcPower.obj
 0001:00015850       ?ConvertStringToGuid@MXDDLcdc@@AAAHPBGPAU_GUID@@@Z 10016850 f   lcdc_common_topaz_v1:DDLcdcPower.obj
 0001:00015a24       ?BltPrepare@MXDDLcdc@@UAAJPAUGPEBltParms@@@Z 10016a24 f   lcdc_common_topaz_v1:DDLcdcBlt.obj
 0001:00015ac8       ?BltComplete@MXDDLcdc@@UAAJPAUGPEBltParms@@@Z 10016ac8 f   lcdc_common_topaz_v1:DDLcdcBlt.obj
 0001:00015b18       ?Line@MXDDLcdc@@UAAJPAUGPELineParms@@W4EGPEPhase@@@Z 10016b18 f   lcdc_common_topaz_v1:DDLcdcLine.obj
 0001:00015b64       ?WrappedEmulatedLine@MXDDLcdc@@QAAJPAUGPELineParms@@@Z 10016b64 f   lcdc_common_topaz_v1:DDLcdcLine.obj
 0001:00016038       ?SetVisibleSurface@MXDDLcdc@@UAAXPAVGPESurf@@H@Z 10017038 f   lcdc_common_topaz_v1:DDLcdcSurf.obj
 0001:000160a4       ?AllocSurface@MXDDLcdc@@UAAJPAPAVGPESurf@@HHW4EGPEFormat@@H@Z 100170a4 f   lcdc_common_topaz_v1:DDLcdcSurf.obj
 0001:00016120       ?AllocSurface@MXDDLcdc@@UAAJPAPAVDDGPESurf@@HHW4EGPEFormat@@W4EDDGPEPixelFormat@@H@Z 10017120 f   lcdc_common_topaz_v1:DDLcdcSurf.obj
 0001:00016548       ?Flip@MXDDLcdc@@QAAKPAU_DDHAL_FLIPDATA@@@Z 10017548 f   lcdc_common_topaz_v1:DDLcdcSurf.obj
 0001:000166f8       ??0MXDDLcdcSurf@@QAA@HHKPAXHW4EGPEFormat@@W4EDDGPEPixelFormat@@PAVSurfaceHeap@@@Z 100176f8 f   lcdc_common_topaz_v1:DDLcdcSurf.obj
 0001:0001678c       ??1MXDDLcdcSurf@@UAA@XZ    1001778c f   lcdc_common_topaz_v1:DDLcdcSurf.obj
 0001:000167c4       ?Buffer@GPESurf@@QAAPAXXZ  100177c4 f i lcdc_common_topaz_v1:DDLcdcSurf.obj
 0001:000167f0       ?Address@SurfaceHeap@@QAAKXZ 100177f0 f i lcdc_common_topaz_v1:DDLcdcSurf.obj
 0001:0001681c       ?GetDriverData@DDGPESurf@@UAAPAUDDGPEDriverData@@XZ 1001781c f i lcdc_common_topaz_v1:DDLcdcSurf.obj
 0001:00016848       ?SetDriverData@DDGPESurf@@UAAXPAUDDGPEDriverData@@@Z 10017848 f i lcdc_common_topaz_v1:DDLcdcSurf.obj
 0001:00016868       ?SurfaceSize@DDGPESurf@@UAAHXZ 10017868 f i lcdc_common_topaz_v1:DDLcdcSurf.obj
 0001:00016894       ??_GMXDDLcdcSurf@@UAAPAXI@Z 10017894 f i lcdc_common_topaz_v1:DDLcdcSurf.obj
 0001:00016894       ??_EMXDDLcdcSurf@@UAAPAXI@Z 10017894 f i lcdc_common_topaz_v1:DDLcdcSurf.obj
 0001:000168d4       ?SetPointerShape@MXDDLcdc@@UAAJPAVGPESurf@@0HHHH@Z 100178d4 f   lcdc_common_topaz_v1:DDLcdcCursor.obj
 0001:00016b98       ?MovePointer@MXDDLcdc@@UAAJHH@Z 10017b98 f   lcdc_common_topaz_v1:DDLcdcCursor.obj
 0001:00016c74       ?CursorOn@MXDDLcdc@@QAAXXZ 10017c74 f   lcdc_common_topaz_v1:DDLcdcCursor.obj
 0001:000174f8       ?CursorOff@MXDDLcdc@@QAAXXZ 100184f8 f   lcdc_common_topaz_v1:DDLcdcCursor.obj
 0001:0001787c       ?PointerBltPrepare@MXDDLcdc@@QAAXPAUGPEBltParms@@@Z 1001887c f   lcdc_common_topaz_v1:DDLcdcCursor.obj
 0001:00017a9c       ?MouseNotificationsThread@MXDDLcdc@@CAKPAX@Z 10018a9c f   lcdc_common_topaz_v1:DDLcdcCursor.obj
 0001:00017b7c       ?StartMouseNotificationsThread@MXDDLcdc@@QAAHXZ 10018b7c f   lcdc_common_topaz_v1:DDLcdcCursor.obj
 0001:00017cb8       ?StopMouseNotificationsThread@MXDDLcdc@@QAAXXZ 10018cb8 f   lcdc_common_topaz_v1:DDLcdcCursor.obj
 0001:00017da8       ?Stride@GPESurf@@QAAHXZ    10018da8 f i lcdc_common_topaz_v1:DDLcdcCursor.obj
 0001:00017dd4       ResetEvent                 10018dd4 f i lcdc_common_topaz_v1:DDLcdcCursor.obj
 0001:00017e08       ?DrvEscapeGAPI@MXDDLcdc@@QAAKKKPAXK0@Z 10018e08 f   lcdc_common_topaz_v1:DDLcdcMisc.obj
 0001:00017e2c       ?DrvEscape@MXDDLcdc@@UAAKPAU_SURFOBJ@@KKPAXK1@Z 10018e2c f   lcdc_common_topaz_v1:DDLcdcMisc.obj
 0001:00018900       ?IsBusy@MXDDLcdc@@UAAHXZ   10019900 f   lcdc_common_topaz_v1:DDLcdcMisc.obj
 0001:000189b0       ?InVBlank@MXDDLcdc@@UAAHXZ 100199b0 f   lcdc_common_topaz_v1:DDLcdcMisc.obj
 0001:00018a10       ?WaitForNotBusy@MXDDLcdc@@UAAXXZ 10019a10 f   lcdc_common_topaz_v1:DDLcdcMisc.obj
 0001:00018a80       ?WaitForVerticalBlank@MXDDLcdc@@QAAKPAU_DDHAL_WAITFORVERTICALBLANKDATA@@@Z 10019a80 f   lcdc_common_topaz_v1:DDLcdcMisc.obj
 0001:00018b98       ?GetRotateModeFromReg@MXDDLcdc@@QAAHXZ 10019b98 f   lcdc_common_topaz_v1:DDLcdcRotate.obj
 0001:00018cdc       ?SetRotateParams@MXDDLcdc@@QAAXXZ 10019cdc f   lcdc_common_topaz_v1:DDLcdcRotate.obj
 0001:00018da4       ?DynRotate@MXDDLcdc@@QAAJH@Z 10019da4 f   lcdc_common_topaz_v1:DDLcdcRotate.obj
 0001:00018e80       ?UpdateOverlay@MXDDLcdc@@QAAKPAU_DDHAL_UPDATEOVERLAYDATA@@@Z 10019e80 f   lcdc_common_topaz_v1:DDLcdcOverlay.obj
 0001:00019b98       ?SetOverlayPosition@MXDDLcdc@@QAAKPAU_DDHAL_SETOVERLAYPOSITIONDATA@@@Z 1001ab98 f   lcdc_common_topaz_v1:DDLcdcOverlay.obj
 0001:0001a2c4       ?SetVisibleSurfaceOverlay@MXDDLcdc@@QAAXPAVDDGPESurf@@@Z 1001b2c4 f   lcdc_common_topaz_v1:DDLcdcOverlay.obj
 0001:0001a408       ?EnableOverlay@MXDDLcdc@@QAAJXZ 1001b408 f   lcdc_common_topaz_v1:DDLcdcOverlay.obj
 0001:0001a924       ?DisableOverlay@MXDDLcdc@@QAAJXZ 1001b924 f   lcdc_common_topaz_v1:DDLcdcOverlay.obj
 0001:0001a9e0       ?GetOverlayAlphaValue@MXDDLcdc@@QAAJXZ 1001b9e0 f   lcdc_common_topaz_v1:DDLcdcOverlay.obj
 0001:0001aa40       ?SetOverlayAlphaValue@MXDDLcdc@@QAAJXZ 1001ba40 f   lcdc_common_topaz_v1:DDLcdcOverlay.obj
 0001:0001ab08       ?WaitForNotBusyOverlay@MXDDLcdc@@QAAXXZ 1001bb08 f   lcdc_common_topaz_v1:DDLcdcOverlay.obj
 0001:0001ab18       ?IsOverlaySurfEqual@@YAHPAUoverlaySurf@@0@Z 1001bb18 f   lcdc_common_topaz_v1:DDLcdcOverlay.obj
 0001:0001accc       ?LcdcVMSetAttributeEx@@YAHPAULcdcVMSetAttributeExDataStruct@@@Z 1001bccc f   lcdc_common_topaz_v1:DDLcdcEscape.obj
 0001:0001ae04       ?LCDCGetBaseRegAddr@@YAIXZ 1001be04 f   lcdc_mx25_topaz_v1:lcdc_base.obj
 0001:0001ae20       ?LCDCGetIRQ@@YAKXZ         1001be20 f   lcdc_mx25_topaz_v1:lcdc_base.obj
 0001:0001ae38       ?LCDCEnableClock@@YAHH@Z   1001be38 f   lcdc_mx25_topaz_v1:lcdc_base.obj
 0001:0001af8c       ?LCDCGetRefClk@@YAKPAULCDC_MODE_DESCRIPTOR@@@Z 1001bf8c f   lcdc_mx25_topaz_v1:lcdc_base.obj
 0001:0001afc4       HALInit                    1001bfc4 f   ddgpe:ddhinit.obj
 0001:0001b210       UpdateHALInit              1001c210 f   ddgpe:ddhinit.obj
 0001:0001b2f8       ?GetDDGPE@@YAPAVDDGPE@@XZ  1001c2f8 f   ddgpe:ddgpe.obj
 0001:0001b31c       ??0DDGPE@@QAA@XZ           1001c31c f   ddgpe:ddgpe.obj
 0001:0001b38c       ??1DDGPE@@UAA@XZ           1001c38c f   ddgpe:ddgpe.obj
 0001:0001b3b4       ?AllocSurface@DDGPE@@UAAJPAPAVDDGPESurf@@HHW4EGPEFormat@@W4EDDGPEPixelFormat@@H@Z 1001c3b4 f   ddgpe:ddgpe.obj
 0001:0001b444       ?AllocSurface@DDGPE@@UAAJPAPAVDDGPESurf@@PAUDDGPEAllocSurfaceData@@@Z 1001c444 f   ddgpe:ddgpe.obj
 0001:0001b520       ?AllocVideoSurface@DDGPE@@UAAJPAPAVDDGPESurf@@HHW4EGPEFormat@@W4EDDGPEPixelFormat@@PAK@Z 1001c520 f   ddgpe:ddgpe.obj
 0001:0001b618       ?AllocVideoSurface@DDGPE@@UAAJPAU_DDRAWI_DDRAWSURFACE_LCL@@HHW4EGPEFormat@@W4EDDGPEPixelFormat@@PAK@Z 1001c618 f   ddgpe:ddgpe.obj
 0001:0001b6cc       ?AllocVideoSurface@DDGPE@@UAAJPAPAVDDGPESurf@@PAUDDGPEAllocSurfaceData@@PAK@Z 1001c6cc f   ddgpe:ddgpe.obj
 0001:0001b7f8       ?AllocVideoSurface@DDGPE@@UAAJPAU_DDRAWI_DDRAWSURFACE_LCL@@PAUDDGPEAllocSurfaceData@@PAK@Z 1001c7f8 f   ddgpe:ddgpe.obj
 0001:0001b894       ?AllocBackBuffer@DDGPE@@UAAJPAU_DDRAWI_DDRAWSURFACE_LCL@@@Z 1001c894 f   ddgpe:ddgpe.obj
 0001:0001b9cc       ?WrapSurface@DDGPE@@UAAJPAU_DDRAWI_DDRAWSURFACE_LCL@@HHW4EGPEFormat@@W4EDDGPEPixelFormat@@HH@Z 1001c9cc f   ddgpe:ddgpe.obj
 0001:0001ba9c       ?WrapSurface@DDGPE@@UAAJPAPAVDDGPESurf@@HHW4EGPEFormat@@W4EDDGPEPixelFormat@@PAEH@Z 1001ca9c f   ddgpe:ddgpe.obj
 0001:0001bb98       ?WrapSurface@DDGPE@@UAAJPAU_DDRAWI_DDRAWSURFACE_LCL@@HHW4EGPEFormat@@W4EDDGPEPixelFormat@@PAEH@Z 1001cb98 f   ddgpe:ddgpe.obj
 0001:0001bc54       ?WrapSurface@DDGPE@@UAAJPAPAVDDGPESurf@@PAUDDGPEAllocSurfaceData@@@Z 1001cc54 f   ddgpe:ddgpe.obj
 0001:0001bda4       ?WrapSurface@DDGPE@@UAAJPAU_DDRAWI_DDRAWSURFACE_LCL@@PAUDDGPEAllocSurfaceData@@@Z 1001cda4 f   ddgpe:ddgpe.obj
 0001:0001be3c       ?BltPrepare@DDGPE@@UAAJPAUDDGPEBltParms@@@Z 1001ce3c f   ddgpe:ddgpe.obj
 0001:0001bf3c       ?PerformBlt@DDGPE@@UAAJPAUDDGPEBltParms@@@Z 1001cf3c f   ddgpe:ddgpe.obj
 0001:0001c01c       ?BltExpanded@DDGPE@@UAAJPAVDDGPESurf@@000PAU_CLIPOBJ@@PAU_XLATEOBJ@@PBUtagRECT@@3KKK@Z 1001d01c f   ddgpe:ddgpe.obj
 0001:0001c274       ?BltExpanded@DDGPE@@UAAJPAVDDGPESurf@@00PBUtagRECT@@1KKK@Z 1001d274 f   ddgpe:ddgpe.obj
 0001:0001c310       ?SetVisibleSurface@DDGPE@@UAAXPAVGPESurf@@KH@Z 1001d310 f   ddgpe:ddgpe.obj
 0001:0001c340       ?SetVisibleSurface@DDGPE@@UAAXPAVGPESurf@@H@Z 1001d340 f   ddgpe:ddgpe.obj
 0001:0001c3c8       ?DetectPixelFormat@DDGPE@@UAAJKPAU_DDPIXELFORMAT@@PAW4EGPEFormat@@PAW4EDDGPEPixelFormat@@@Z 1001d3c8 f   ddgpe:ddgpe.obj
 0001:0001c9d4       ?DetectMode@DDGPE@@UAAJPAKKKW4EGPEFormat@@W4EDDGPEPixelFormat@@PAU_DDPIXELFORMAT@@@Z 1001d9d4 f   ddgpe:ddgpe.obj
 0001:0001ce20       ?InDisplay@DDGPE@@UAAHXZ   1001de20 f   ddgpe:ddgpe.obj
 0001:0001ce44       ?GetModeInfoEx@DDGPE@@UAAJPAUGPEModeEx@@H@Z 1001de44 f   ddgpe:ddgpe.obj
 0001:0001cea0       ?SetMode@DDGPE@@UAAJHPAPAUHPALETTE__@@H@Z 1001dea0 f   ddgpe:ddgpe.obj
 0001:0001cefc       ?RegisterDDHALAPI@@YAXXZ   1001defc f   ddgpe:ddgpe.obj
 0001:0001cf00       ??_GDDGPE@@UAAPAXI@Z       1001df00 f i ddgpe:ddgpe.obj
 0001:0001cf00       ??_EDDGPE@@UAAPAXI@Z       1001df00 f i ddgpe:ddgpe.obj
 0001:0001cf40       ?Format@GPESurf@@QAA?AW4EGPEFormat@@XZ 1001df40 f i ddgpe:ddgpe.obj
 0001:0001cf6c       ?Width@GPESurf@@QAAHXZ     1001df6c f i ddgpe:ddgpe.obj
 0001:0001cf98       ?Height@GPESurf@@QAAHXZ    1001df98 f i ddgpe:ddgpe.obj
 0001:0001cfc4       ?Rotate@GPESurf@@QAAHXZ    1001dfc4 f i ddgpe:ddgpe.obj
 0001:0001cff0       ?ScreenWidth@GPESurf@@QAAHXZ 1001dff0 f i ddgpe:ddgpe.obj
 0001:0001d01c       ?ScreenHeight@GPESurf@@QAAHXZ 1001e01c f i ddgpe:ddgpe.obj
 0001:0001d048       ?DDGPEPrimarySurface@DDGPE@@QAAPAVDDGPESurf@@XZ 1001e048 f i ddgpe:ddgpe.obj
 0001:0001d078       ?PrimarySurface@GPE@@QAAPAVGPESurf@@XZ 1001e078 f i ddgpe:ddgpe.obj
 0001:0001d0a4       ?FourCCLookup@@YAPBU_FourCCDescription@@K@Z 1001e0a4 f i ddgpe:ddgpe.obj
 0001:0001d134       ?Available@SurfaceHeap@@QAAKXZ 1001e134 f   ddgpe:surfheap.obj
 0001:0001d1b4       ??0SurfaceHeap@@QAA@KKPAV0@0@Z 1001e1b4 f   ddgpe:surfheap.obj
 0001:0001d2a4       ??1SurfaceHeap@@QAA@XZ     1001e2a4 f   ddgpe:surfheap.obj
 0001:0001d47c       ?Alloc@SurfaceHeap@@QAAPAV1@K@Z 1001e47c f   ddgpe:surfheap.obj
 0001:0001d690       ?Free@SurfaceHeap@@QAAXXZ  1001e690 f   ddgpe:surfheap.obj
 0001:0001d830       ?Size@SurfaceHeap@@QAAKXZ  1001e830 f   ddgpe:surfheap.obj
 0001:0001d89c       ??_GSurfaceHeap@@QAAPAXI@Z 1001e89c f i ddgpe:surfheap.obj
 0001:0001d8dc       ??0DDGPESurf@@QAA@HHPAXHW4EGPEFormat@@@Z 1001e8dc f   ddgpe:ddgpesurf.obj
 0001:0001d9c8       ??0DDGPESurf@@QAA@HHPAXHW4EGPEFormat@@W4EDDGPEPixelFormat@@@Z 1001e9c8 f   ddgpe:ddgpesurf.obj
 0001:0001daac       ??0DDGPESurf@@QAA@HHHW4EGPEFormat@@W4EDDGPEPixelFormat@@@Z 1001eaac f   ddgpe:ddgpesurf.obj
 0001:0001dc40       ??0DDGPESurf@@QAA@HHW4EGPEFormat@@@Z 1001ec40 f   ddgpe:ddgpesurf.obj
 0001:0001ddec       ??0DDGPESurf@@QAA@XZ       1001edec f   ddgpe:ddgpesurf.obj
 0001:0001deac       ??1DDGPESurf@@UAA@XZ       1001eeac f   ddgpe:ddgpesurf.obj
 0001:0001df68       ?Init@DDGPESurf@@UAAXHHPAXHW4EGPEFormat@@W4EDDGPEPixelFormat@@@Z 1001ef68 f   ddgpe:ddgpesurf.obj
 0001:0001dfcc       ?Bpp@DDGPESurf@@UAAKXZ     1001efcc f   ddgpe:ddgpesurf.obj
 0001:0001e014       ?AlignedWidth@DDGPESurf@@UAAKXZ 1001f014 f   ddgpe:ddgpesurf.obj
 0001:0001e07c       ?SetColorKey@DDGPESurf@@UAAXK@Z 1001f07c f   ddgpe:ddgpesurf.obj
 0001:0001e0c4       ?ColorKey@DDGPESurf@@UAAKXZ 1001f0c4 f   ddgpe:ddgpesurf.obj
 0001:0001e104       ?SetColorKeyMask@DDGPESurf@@UAAXK@Z 1001f104 f   ddgpe:ddgpesurf.obj
 0001:0001e124       ?ColorKeyMask@DDGPESurf@@UAAKXZ 1001f124 f   ddgpe:ddgpesurf.obj
 0001:0001e150       ?SetColorKeyLow@DDGPESurf@@UAAXK@Z 1001f150 f   ddgpe:ddgpesurf.obj
 0001:0001e170       ?ColorKeyLow@DDGPESurf@@UAAKXZ 1001f170 f   ddgpe:ddgpesurf.obj
 0001:0001e19c       ?SetColorKeyHigh@DDGPESurf@@UAAXK@Z 1001f19c f   ddgpe:ddgpesurf.obj
 0001:0001e1bc       ?ColorKeyHigh@DDGPESurf@@UAAKXZ 1001f1bc f   ddgpe:ddgpesurf.obj
 0001:0001e1e8       ?PixelFormat@DDGPESurf@@UAA?AW4EDDGPEPixelFormat@@XZ 1001f1e8 f   ddgpe:ddgpesurf.obj
 0001:0001e214       ?HasAlpha@DDGPESurf@@UAAHXZ 1001f214 f   ddgpe:ddgpesurf.obj
 0001:0001e288       ?SetDDGPESurf@DDGPESurf@@UAAXPAU_DDRAWI_DDRAWSURFACE_LCL@@@Z 1001f288 f   ddgpe:ddgpesurf.obj
 0001:0001e2b8       ?DeleteSurface@DDGPESurf@@SAXPAU_DDRAWI_DDRAWSURFACE_LCL@@@Z 1001f2b8 f   ddgpe:ddgpesurf.obj
 0001:0001e348       ?GetDDGPESurf@DDGPESurf@@SAPAV1@PAU_DDRAWI_DDRAWSURFACE_LCL@@@Z 1001f348 f   ddgpe:ddgpesurf.obj
 0001:0001e38c       ?SetRotation@DDGPESurf@@QAAXHHH@Z 1001f38c f   ddgpe:ddgpesurf.obj
 0001:0001e3fc       ??0GPESurf@@QAA@HHPAXHW4EGPEFormat@@@Z 1001f3fc f i ddgpe:ddgpesurf.obj
 0001:0001e464       ??0GPEFormat@@QAA@XZ       1001f464 f i ddgpe:ddgpesurf.obj
 0001:0001e4c4       ??_EGPESurf@@UAAPAXI@Z     1001f4c4 f i ddgpe:ddgpesurf.obj
 0001:0001e4c4       ??_GGPESurf@@UAAPAXI@Z     1001f4c4 f i ddgpe:ddgpesurf.obj
 0001:0001e504       ??_GDDGPESurf@@UAAPAXI@Z   1001f504 f i ddgpe:ddgpesurf.obj
 0001:0001e504       ??_EDDGPESurf@@UAAPAXI@Z   1001f504 f i ddgpe:ddgpesurf.obj
 0001:0001e544       ??0GPESurf@@QAA@XZ         1001f544 f i ddgpe:ddgpesurf.obj
 0001:0001e5a8       DllMain                    1001f5a8 f   gpe:ddi_if.obj
 0001:0001e610       ?SafeGetGPE@@YAPAVGPE@@PAX@Z 1001f610 f   gpe:ddi_if.obj
 0001:0001e6ac       ?SetSurfaceFormat@@YAXPAVGPESurf@@PAU_XLATEOBJ@@KPAK@Z 1001f6ac f   gpe:ddi_if.obj
 0001:0001e9d4       ?GPEEnableDriver@@YAHKKPAUtagDrvEnableData@@PAU_ENGCALLBACKS@@@Z 1001f9d4 f   gpe:ddi_if.obj
 0001:0001ecbc       DrvContrastControl         1001fcbc f   gpe:ddi_if.obj
 0001:0001ed1c       DrvPowerHandler            1001fd1c f   gpe:ddi_if.obj
 0001:0001ed6c       DrvEscape                  1001fd6c f   gpe:ddi_if.obj
 0001:0001ef94       DrvDisableDriver           1001ff94 f   gpe:ddi_if.obj
 0001:0001f064       DrvDisablePDEV             10020064 f   gpe:ddi_if.obj
 0001:0001f158       DrvDisableSurface          10020158 f   gpe:ddi_if.obj
 0001:0001f1f4       DrvEnableSurface           100201f4 f   gpe:ddi_if.obj
 0001:0001f390       DrvCreateDeviceBitmap      10020390 f   gpe:ddi_if.obj
 0001:0001f504       DrvDeleteDeviceBitmap      10020504 f   gpe:ddi_if.obj
 0001:0001f5f8       DrvMovePointer             100205f8 f   gpe:ddi_if.obj
 0001:0001f6a8       DrvSetPointerShape         100206a8 f   gpe:ddi_if.obj
 0001:0001f950       DrvSetPalette              10020950 f   gpe:ddi_if.obj
 0001:0001fab4       DrvFillPath                10020ab4 f   gpe:ddi_if.obj
 0001:00020390       DrvRealizeBrush            10021390 f   gpe:ddi_if.obj
 0001:0002088c       DrvGetModes                1002188c f   gpe:ddi_if.obj
 0001:00020b20       DrvEnablePDEV              10021b20 f   gpe:ddi_if.obj
 0001:000211e8       DrvPaint                   100221e8 f   gpe:ddi_if.obj
 0001:0002133c       DrvCopyBits                1002233c f   gpe:ddi_if.obj
 0001:000213d0       DrvAnyBlt                  100223d0 f   gpe:ddi_if.obj
 0001:000214a4       DrvTransparentBlt          100224a4 f   gpe:ddi_if.obj
 0001:00021584       DrvBitBlt                  10022584 f   gpe:ddi_if.obj
 0001:000216e0       AnyBlt                     100226e0 f   gpe:ddi_if.obj
 0001:00022810       ?ClipBlt@@YAJPAVGPE@@PAUGPEBltParms@@@Z 10023810 f   gpe:ddi_if.obj
 0001:00022bc4       ?AAGetMaskBits@@YAXPAK00@Z 10023bc4 f   gpe:ddi_if.obj
 0001:00022c40       ?FormatPtr@GPESurf@@QAAPAVGPEFormat@@XZ 10023c40 f i gpe:ddi_if.obj
 0001:00022c68       DispPerfQueryEsc           10023c68 f i gpe:ddi_if.obj
 0001:00022c8c       ?SetHSurf@GPE@@QAAXK@Z     10023c8c f i gpe:ddi_if.obj
 0001:00022cac       ?GetHSurf@GPE@@QAAKXZ      10023cac f i gpe:ddi_if.obj
 0001:00022cd8       ?ScreenHeight@GPE@@QAAHXZ  10023cd8 f i gpe:ddi_if.obj
 0001:00022d04       ?ScreenWidth@GPE@@QAAHXZ   10023d04 f i gpe:ddi_if.obj
 0001:00022d30       ?SurfobjToGPE@@YAPAVGPE@@PAU_SURFOBJ@@@Z 10023d30 f i gpe:ddi_if.obj
 0001:00022d5c       ??BTmpGPESurf@@QAAPAVGPESurf@@XZ 10023d5c f i gpe:ddi_if.obj
 0001:00022d84       ??1TmpGPESurf@@QAA@XZ      10023d84 f i gpe:ddi_if.obj
 0001:00022da0       ?GetModeId@GPE@@QAAHXZ     10023da0 f i gpe:ddi_if.obj
 0001:00022dd0       ?SourceMatters@@YA_NK@Z    10023dd0 f i gpe:ddi_if.obj
 0001:00022e28       ?BrushMatters@@YA_NK@Z     10023e28 f i gpe:ddi_if.obj
 0001:00022e80       ?MaskMatters@@YA_NK@Z      10023e80 f i gpe:ddi_if.obj
 0001:00022ed0       ??0GPE@@QAA@XZ             10023ed0 f   gpe:gpe.obj
 0001:00022f88       ??1GPE@@UAA@XZ             10023f88 f   gpe:gpe.obj
 0001:00022fa8       ?ContrastControl@GPE@@UAAHKPAK@Z 10023fa8 f   gpe:gpe.obj
 0001:00022fcc       ?PowerHandler@GPE@@UAAXH@Z 10023fcc f   gpe:gpe.obj
 0001:00022fdc       ?GetPalette@GPE@@UAAJPAPAUtagPALETTEENTRY@@PAG@Z 10023fdc f   gpe:gpe.obj
 0001:00023084       ?DrvEscape@GPE@@UAAKPAU_SURFOBJ@@KKPAXK1@Z 10024084 f   gpe:gpe.obj
 0001:000230a8       ?GetGraphicsCaps@GPE@@UAAKXZ 100240a8 f   gpe:gpe.obj
 0001:000230cc       ?GetPhysicalVideoMemory@GPE@@UAAXPAK0@Z 100240cc f   gpe:gpe.obj
 0001:000230dc       ?GetVirtualVideoMemory@GPE@@UAAXPAK0@Z 100240dc f   gpe:gpe.obj
 0001:000230ec       ?SetVisibleSurface@GPE@@UAAXPAVGPESurf@@@Z 100240ec f   gpe:gpe.obj
 0001:000230fc       ?FlipInProgress@GPE@@UAAHXZ 100240fc f   gpe:gpe.obj
 0001:00023120       ?WaitForVBlank@GPE@@UAAXXZ 10024120 f   gpe:gpe.obj
 0001:00023130       ?SurfaceBusyFlipping@GPE@@UAAHPAVGPESurf@@@Z 10024130 f   gpe:gpe.obj
 0001:00023154       ?IsBusy@GPE@@UAAHXZ        10024154 f   gpe:gpe.obj
 0001:00023178       ?WaitForNotBusy@GPE@@UAAXXZ 10024178 f   gpe:gpe.obj
 0001:00023188       ?AvailableVideoMemory@GPE@@UAAKXZ 10024188 f   gpe:gpe.obj
 0001:000231ac       ?ScanLine@GPE@@UAAHXZ      100241ac f   gpe:gpe.obj
 0001:000231d0       ?ProcessCommandBlock@GPE@@UAAJPAE@Z 100241d0 f   gpe:gpe.obj
 0001:000231f8       ?GetScreenDimensions@GPE@@UAAHPAUGPEScreenProps@@@Z 100241f8 f   gpe:gpe.obj
 0001:000235cc       ?IsPaletteSettable@GPE@@UAAHXZ 100245cc f   gpe:gpe.obj
 0001:00023620       ?RotateRectl@GPE@@QAAXPAU_RECTL@@@Z 10024620 f   gpe:gpe.obj
 0001:000237bc       ?RotateRectlBack@GPE@@QAAXPAU_RECTL@@@Z 100247bc f   gpe:gpe.obj
 0001:00023958       ?GetClearTypeRGBMasks@GPE@@UAAPAKXZ 10024958 f   gpe:gpe.obj
 0001:00023988       ?DisablePrimary@GPE@@UAAHXZ 10024988 f   gpe:gpe.obj
 0001:00023a20       ??0GPESurf@@QAA@HHW4EGPEFormat@@@Z 10024a20 f   gpe:gpe.obj
 0001:00023d44       ?Init@GPESurf@@QAAXHHPAXHW4EGPEFormat@@@Z 10024d44 f   gpe:gpe.obj
 0001:00023e48       ??1GPESurf@@UAA@XZ         10024e48 f   gpe:gpe.obj
 0001:00023ebc       ?RotateLineParms@GPESurf@@QAAXPAUGPELineParms@@@Z 10024ebc f   gpe:gpe.obj
 0001:000240f4       ?SetRotation@GPESurf@@QAAXHHH@Z 100250f4 f   gpe:gpe.obj
 0001:000241c4       ?RotatePathdata@GPESurf@@QAAXPAU_PATHDATA@@@Z 100251c4 f   gpe:gpe.obj
 0001:000243ec       ?RotatePathdataBack@GPESurf@@QAAXPAU_PATHDATA@@@Z 100253ec f   gpe:gpe.obj
 0001:00024614       ?RotateRectl@GPESurf@@QAAXPAU_RECTL@@@Z 10025614 f   gpe:gpe.obj
 0001:000247b0       ?RotateRectlBack@GPESurf@@QAAXPAU_RECTL@@@Z 100257b0 f   gpe:gpe.obj
 0001:0002494c       ?GetPtr@GPESurf@@QAAPAEHH@Z 1002594c f   gpe:gpe.obj
 0001:00024b30       ??1GPEFormat@@QAA@XZ       10025b30 f   gpe:gpe.obj
 0001:00024b84       ??_GGPE@@UAAPAXI@Z         10025b84 f i gpe:gpe.obj
 0001:00024b84       ??_EGPE@@UAAPAXI@Z         10025b84 f i gpe:gpe.obj
 0001:00024bc4       ?IntToULong@@YAJHPAK@Z     10025bc4 f i gpe:gpe.obj
 0001:00024c20       ?ULongMult@@YAJKKPAK@Z     10025c20 f i gpe:gpe.obj
 0001:00024c7c       ?ULongLongToULong@@YAJ_KPAK@Z 10025c7c f i gpe:gpe.obj
 0001:00024d00       ?SelectBlt@GPE@@IAAJPAUGPEBltParms@@P81@AAJ0@Z@Z 10025d00 f   gpe:swblt.obj
 0001:00025950       ?EmulatedBlt@GPE@@QAAJPAUGPEBltParms@@@Z 10026950 f   gpe:swblt.obj
 0001:0002598c       ?EmulatedBltRotate@GPE@@QAAJPAUGPEBltParms@@@Z 1002698c f   gpe:swblt.obj
 0001:000259c8       ?EmulatedBlt_Internal@GPE@@QAAJPAUGPEBltParms@@@Z 100269c8 f   gpe:swblt.obj
 0001:00028b80       ?EmulatedBlt_Bilinear@GPE@@QAAJPAUGPEBltParms@@@Z 10029b80 f   gpe:swblt.obj
 0001:000299e8       ?EmulatedBlt_Halftone@GPE@@QAAJPAUGPEBltParms@@@Z 1002a9e8 f   gpe:swblt.obj
 0001:0002a964       ?EmulatedBltRotate_Internal@GPE@@QAAJPAUGPEBltParms@@@Z 1002b964 f   gpe:swblt.obj
 0001:0002dfb8       ?EmulatedBltRotate_Bilinear@GPE@@QAAJPAUGPEBltParms@@@Z 1002efb8 f   gpe:swblt.obj
 0001:0002f324       ?EmulatedBltRotate_Halftone@GPE@@QAAJPAUGPEBltParms@@@Z 10030324 f   gpe:swblt.obj
 0001:0003080c       ?InVideoMemory@GPESurf@@QAAHXZ 1003180c f i gpe:swblt.obj
 0001:00030838       ?IsRotate@GPESurf@@QAAHXZ  10031838 f i gpe:swblt.obj
 0001:00030884       ?DestMatters@@YA_NK@Z      10031884 f i gpe:swblt.obj
 0001:000308dc       ?InitPixelIterator@PixelIterator@@QAAXXZ 100318dc f i gpe:swblt.obj
 0001:00030908       ?InitPixelIterator@PixelIteratorRotate@@QAAXXZ 10031908 f i gpe:swblt.obj
 0001:00030944       ?EmulatedLine@GPE@@QAAJPAUGPELineParms@@@Z 10031944 f   gpe:swline.obj
 0001:00031dd8       ??_H@YAXPAXIHP6APAX0@Z@Z   10032dd8 f i gpe:swconvrt.obj
 0001:00031e20       ?AllocConverters@@YAHXZ    10032e20 f   gpe:swconvrt.obj
 0001:00031f28       ?FreeConverters@@YAXXZ     10032f28 f   gpe:swconvrt.obj
 0001:00031fac       ?InitLRU@GroupColorConverter@@QAAHXZ 10032fac f   gpe:swconvrt.obj
 0001:00031fe4       ?FreeLRU@GroupColorConverter@@QAAXXZ 10032fe4 f   gpe:swconvrt.obj
 0001:00032000       ??0LRU@@QAA@XZ             10033000 f   gpe:swconvrt.obj
 0001:00032060       ?Init@LRU@@QAAHG@Z         10033060 f   gpe:swconvrt.obj
 0001:00032308       ?Find@LRU@@QAAFK@Z         10033308 f   gpe:swconvrt.obj
 0001:00032644       ?Add@LRU@@QAAFK@Z          10033644 f   gpe:swconvrt.obj
 0001:00032770       ?Fill@LRU@@QAAXK@Z         10033770 f   gpe:swconvrt.obj
 0001:000327f8       ?Free@LRU@@QAAXXZ          100337f8 f   gpe:swconvrt.obj
 0001:000328cc       ?SwapRedBlue@@YAKK@Z       100338cc f   gpe:swconvrt.obj
 0001:00032908       ?InitMaskInfo@MaskInfo@@QAAXPAU_XLATEOBJ@@KG@Z 10033908 f   gpe:swconvrt.obj
 0001:00032b04       ?RGBToGroup@@YAFK@Z        10033b04 f   gpe:swconvrt.obj
 0001:00032b58       ?InitConverter@ColorConverter@@SAXPAU_XLATEOBJ@@PAPAV1@PAP81@AAKK@ZPAPAK@Z 10033b58 f   gpe:swconvrt.obj
 0001:00033198       ?Init@MaskColorConverter@@QAAXPAU_XLATEOBJ@@@Z 10034198 f   gpe:swconvrt.obj
 0001:00033220       ?Init@GroupColorConverter@@QAAXPAU_XLATEOBJ@@@Z 10034220 f   gpe:swconvrt.obj
 0001:0003367c       ?Init@LookupColorConverter@@QAAXPAU_XLATEOBJ@@@Z 1003467c f   gpe:swconvrt.obj
 0001:000339d4       ?MaskedSrcToPaletteDst@GroupColorConverter@@QAAKK@Z 100349d4 f   gpe:swconvrt.obj
 0001:00033df0       ?RGBToFromBGR@MaskColorConverter@@QAAKK@Z 10034df0 f   gpe:swconvrt.obj
 0001:00033e20       ?RGBToFromBGR@GroupColorConverter@@QAAKK@Z 10034e20 f   gpe:swconvrt.obj
 0001:00033e50       ?MaskedSrcToRGB@MaskColorConverter@@QAAKK@Z 10034e50 f   gpe:swconvrt.obj
 0001:00033f70       ?MaskedSrcToRGB@GroupColorConverter@@QAAKK@Z 10034f70 f   gpe:swconvrt.obj
 0001:000340b4       ?MaskedSrcToBGR@MaskColorConverter@@QAAKK@Z 100350b4 f   gpe:swconvrt.obj
 0001:000341d4       ?RGBSrcToMaskedDst@MaskColorConverter@@QAAKK@Z 100351d4 f   gpe:swconvrt.obj
 0001:00034274       ?RGBSrcToMaskedDst@LookupColorConverter@@QAAKK@Z 10035274 f   gpe:swconvrt.obj
 0001:00034314       ?BGRSrcToMaskedDst@MaskColorConverter@@QAAKK@Z 10035314 f   gpe:swconvrt.obj
 0001:000343b4       ?MaskedSrcToMaskedDst@MaskColorConverter@@QAAKK@Z 100353b4 f   gpe:swconvrt.obj
 0001:000344c4       ?AnyToMono@MonoColorConverter@@QAAKK@Z 100354c4 f   gpe:swconvrt.obj
 0001:00034510       DrvRealizeColor            10035510 f   gpe:swconvrt.obj
 0001:00034844       DrvUnrealizeColor          10035844 f   gpe:swconvrt.obj
 0001:00034a84       ?Init@MonoColorConverter@@QAAXK@Z 10035a84 f i gpe:swconvrt.obj
 0001:00034aa0       ?LookupTable@LookupColorConverter@@QAAPAKXZ 10035aa0 f i gpe:swconvrt.obj
 0001:00034ac8       ??0GroupColorConverter@@QAA@XZ 10035ac8 f i gpe:swconvrt.obj
 0001:00034af8       DrvStrokePath              10035af8 f   gpe:drvstrok.obj
 0001:00035f94       ?SafeCallLine@@YAJPAVGPE@@PAUGPELineParms@@@Z 10036f94 f   gpe:drvstrok.obj
 0001:00036008       ?AATextBltInit@@YAHP6AXPAK00@Z@Z 10037008 f   gpe:aablt.obj
 0001:0003603c       ?AATextBltSelect@@YAJPAUGPEBltParms@@@Z 1003703c f   gpe:aablt.obj
 0001:0003616c       ?AATextBltDst8@AATextBlt@@QAAJPAUGPEBltParms@@@Z 1003716c f   gpe:aablt.obj
 0001:000364c8       ?BlendPixelAA@AAMASKINFO@@QAAKKE@Z 100374c8 f   gpe:aablt.obj
 0001:000367bc       ?SetAAGammaValue@@YAHKH@Z  100377bc f   gpe:aablt.obj
 0001:0003694c       ?AATextBltDst16@AATextBlt@@QAAJPAUGPEBltParms@@@Z 1003794c f   gpe:aablt.obj
 0001:00037070       ?AATextBltDst24@AATextBlt@@QAAJPAUGPEBltParms@@@Z 10038070 f   gpe:aablt.obj
 0001:000374bc       ?AATextBltDst32@AATextBlt@@QAAJPAUGPEBltParms@@@Z 100384bc f   gpe:aablt.obj
 0001:000378b0       ?SetGamma@AAMASKINFO@@QAAXM@Z 100388b0 f i gpe:aablt.obj
 0001:00037afc       ?SetUF@AAMASKINFO@@QAAXK@Z 10038afc f i gpe:aablt.obj
 0001:00037bc8       DrvAlphaBlend              10038bc8 f   gpe:drvalphablend.obj
 0001:00037ca0       ?drvRectFill32@@YAXPAVGPESurf@@PAU_DRVGRADIENTRECTDATA@@@Z 10038ca0 f   gpe:rdrvgradfill.obj
 0001:00038870       ?drvRectFill24@@YAXPAVGPESurf@@PAU_DRVGRADIENTRECTDATA@@@Z 10039870 f   gpe:rdrvgradfill.obj
 0001:000392bc       ?drvRectFill16@@YAXPAVGPESurf@@PAU_DRVGRADIENTRECTDATA@@H@Z 1003a2bc f   gpe:rdrvgradfill.obj
 0001:00039b1c       ?drvRectFill16_565@@YAXPAVGPESurf@@PAU_DRVGRADIENTRECTDATA@@@Z 1003ab1c f   gpe:rdrvgradfill.obj
 0001:00039b3c       ?drvRectFill16_555@@YAXPAVGPESurf@@PAU_DRVGRADIENTRECTDATA@@@Z 1003ab3c f   gpe:rdrvgradfill.obj
 0001:00039bec       ?drvRectFill16Bitfields@@YAXPAVGPESurf@@PAU_DRVGRADIENTRECTDATA@@@Z 1003abec f   gpe:rdrvgradfill.obj
 0001:00039c0c       ?drvRectFillPalIndex@@YAXPAVGPESurf@@PAU_DRVGRADIENTRECTDATA@@H@Z 1003ac0c f   gpe:rdrvgradfill.obj
 0001:0003a3e0       ?drvRectFill8@@YAXPAVGPESurf@@PAU_DRVGRADIENTRECTDATA@@@Z 1003b3e0 f   gpe:rdrvgradfill.obj
 0001:0003a400       ?drvRectFill4@@YAXPAVGPESurf@@PAU_DRVGRADIENTRECTDATA@@@Z 1003b400 f   gpe:rdrvgradfill.obj
 0001:0003a420       ?drvRectFill1@@YAXPAVGPESurf@@PAU_DRVGRADIENTRECTDATA@@@Z 1003b420 f   gpe:rdrvgradfill.obj
 0001:0003ac58       DrvGradientFill            1003bc58 f   gpe:rdrvgradfill.obj
 0001:0003c190       ?IntToUInt@@YAJHPAI@Z      1003d190 f i gpe:rdrvgradfill.obj
 0001:0003c1ec       ?UIntMult@@YAJIIPAI@Z      1003d1ec f i gpe:rdrvgradfill.obj
 0001:0003c248       ?ULongLongToUInt@@YAJ_KPAI@Z 1003d248 f i gpe:rdrvgradfill.obj
 0001:0003c2cc       ?vClearTypeLookupTableLoop@@YAXKPAU_BLENDINFO@@KK@Z 1003d2cc f   gpe:rctblt.obj
 0001:0003cc9c       ?pvFillOpaqTableCT@@YAPAXKKKPAU_BLENDINFO@@@Z 1003dc9c f   gpe:rctblt.obj
 0001:0003cd88       ?ulBlendPixelCT@@YAKPAU_BLENDINFO@@KPAU_F_RGB@@@Z 1003dd88 f   gpe:rctblt.obj
 0001:0003d0a8       ?ulBlendPixelCT8bpp@@YAKPAU_BLENDINFO@@KPAU_F_RGB@@@Z 1003e0a8 f   gpe:rctblt.obj
 0001:0003d2e4       ?ClearTypeBltInit@@YAHPAUGPEMode@@PAKPAUtagPALETTEENTRY@@I@Z 1003e2e4 f   gpe:rctblt.obj
 0001:0003d41c       ?ClearTypeBltSelect@@YAJPAUGPEBltParms@@@Z 1003e41c f   gpe:rctblt.obj
 0001:0003d748       ?ClearTypeBltDst16@ClearTypeBlt@@QAAJPAUGPEBltParms@@@Z 1003e748 f   gpe:rctblt.obj
 0001:0003db1c       ?ClearTypeBltDst24@ClearTypeBlt@@QAAJPAUGPEBltParms@@@Z 1003eb1c f   gpe:rctblt.obj
 0001:0003dfa4       ?ClearTypeBltDst32@ClearTypeBlt@@QAAJPAUGPEBltParms@@@Z 1003efa4 f   gpe:rctblt.obj
 0001:0003e360       ?ClearTypeBltDst8@ClearTypeBlt@@QAAJPAUGPEBltParms@@@Z 1003f360 f   gpe:rctblt.obj
 0001:0003e714       ?SetClearTypeBltMasks@@YAXKKK@Z 1003f714 f   gpe:rctblt.obj
 0001:0003e8e4       ?SetClearTypeBltPalette@@YAXPAUtagPALETTEENTRY@@H@Z 1003f8e4 f   gpe:rctblt.obj
 0001:0003e914       ?SetClearTypeBltGamma@@YAXK@Z 1003f914 f   gpe:rctblt.obj
 0001:0003ebec       ?GetGammaValue@@YAHPAK@Z   1003fbec f   gpe:rctblt.obj
 0001:0003ec24       ?SetGammaValue@@YAHKH@Z    1003fc24 f   gpe:rctblt.obj
 0001:0003ed0c       ??0TmpGPESurf@@QAA@PAU_SURFOBJ@@0PAV0@K@Z 1003fd0c f   gpe:TmpGPESurf.obj
 0001:0003ef60       ?InUserMemory@GPESurf@@QAAXH@Z 1003ff60 f i gpe:TmpGPESurf.obj
 0001:0003ef80       ??0EdgeList@@QAA@H@Z       1003ff80 f   gpe:swfill.obj
 0001:0003f0d4       ??1EdgeList@@QAA@XZ        100400d4 f   gpe:swfill.obj
 0001:0003f16c       ?AddEdge@EdgeList@@QAAJJJJJ@Z 1004016c f   gpe:swfill.obj
 0001:0003f6e0       ?Fill@EdgeList@@QAAJPAUGPEBltParms@@PAU_RECTL@@PAVGPE@@@Z 100406e0 f   gpe:swfill.obj
 0001:000402d0       GenBltInitialize           100412d0 f   gpe:genblt.obj
 0001:00040760       GenBltSetMode              10041760 f   gpe:genblt.obj
 0001:00040ad4       ?ClockOverflow@@YAXXZ      10041ad4 f   gpe:genblt.obj
 0001:00040c14       ?FunctionCacheLookup@@YAPAUGenBltFunction@@PAUGenBltSignature@@@Z 10041c14 f   gpe:genblt.obj
 0001:00040d60       ?GetFnCacheMem@@YAPAUGenBltFunction@@PAUGenBltSignature@@@Z 10041d60 f   gpe:genblt.obj
 0001:00040f5c       ?InvalidateFnCacheItem@@YAHPAX@Z 10041f5c f   gpe:genblt.obj
 0001:000410b8       ?GetBltFunction@@YAPAUGenBltFunction@@PAUGenBltSignature@@@Z 100420b8 f   gpe:genblt.obj
 0001:00041218       ?GenerateSignature@@YAHPAUGPEBltParms@@PAUGenBltSignature@@@Z 10042218 f   gpe:genblt.obj
 0001:00041c68       ?GPEFormatToGenBltFormat@@YA?AW4GenBltFormat@@PAVGPEFormat@@W4EGPEFormat@@@Z 10042c68 f   gpe:genblt.obj
 0001:00041f3c       GeneratedBltSelect         10042f3c f   gpe:GenBltGpe.obj
 0001:00041fc8       ?WrappedGeneratedBlt@GPE@@QAAJPAUGPEBltParms@@@Z 10042fc8 f   gpe:GenBltGpe.obj
 0001:000421d0       ?GetGenBltCpuFuncs@@YAPAUGenBltCpuFuncs@@XZ 100431d0 f i gpe:GenBltGpe.obj
 0001:000421ec       ?ClockIncrement@@YAXXZ     100431ec f i gpe:GenBltGpe.obj
 0001:00042220       ?BltClock@@YAKXZ           10043220 f i gpe:GenBltGpe.obj
 0001:00042240       ?Blt_Stretch_Alpha_32To16at565@Emulator@@QAAJPAUGPEBltParms@@@Z 10043240 f   gpe:FastBlt.obj
 0001:00042e00       ?Blt_NoStretch_Alpha_32To16at565@Emulator@@QAAJPAUGPEBltParms@@@Z 10043e00 f   gpe:FastBlt.obj
 0001:000431a0       ?Blt_NoStretch_Alpha_24To24_Aligned@@YAJPAKH0HHHK@Z 100441a0 f   gpe:FastBlt.obj
 0001:000432e0       ?Blt_NoStretch_Alpha_24To24@Emulator@@QAAJPAUGPEBltParms@@@Z 100442e0 f   gpe:FastBlt.obj
 0001:00043680       ?Blt_NoStretch_Alpha_16To16@Emulator@@QAAJPAUGPEBltParms@@@Z 10044680 f   gpe:FastBlt.obj
 0001:0004397c       ?Blt_NoStretch_Trans_16To16@Emulator@@QAAJPAUGPEBltParms@@@Z 1004497c f   gpe:FastBlt.obj
 0001:00043c4c       ?Blt_Stretch_Trans_16To16@Emulator@@QAAJPAUGPEBltParms@@@Z 10044c4c f   gpe:FastBlt.obj
 0001:00044a1c       ?Blt_NoStretch_NoTrans_32To16at565@Emulator@@QAAJPAUGPEBltParms@@@Z 10045a1c f   gpe:FastBlt.obj
 0001:00044cfc       ?Blt_NoStretch_NoTrans_16at565To32@Emulator@@QAAJPAUGPEBltParms@@@Z 10045cfc f   gpe:FastBlt.obj
 0001:00044fcc       ?Blt_NoStretch_NoTrans_24To24@Emulator@@QAAJPAUGPEBltParms@@@Z 10045fcc f   gpe:FastBlt.obj
 0001:00045228       ?Blt_NoStretch_NoTrans_16To16@Emulator@@QAAJPAUGPEBltParms@@@Z 10046228 f   gpe:FastBlt.obj
 0001:000454d0       ?Blt_Text_32@Emulator@@QAAJPAUGPEBltParms@@@Z 100464d0 f   gpe:FastBlt.obj
 0001:000457b0       ?Blt_Fill_32@Emulator@@QAAJPAUGPEBltParms@@@Z 100467b0 f   gpe:FastBlt.obj
 0001:000459b0       ?Blt_Fill_24@Emulator@@QAAJPAUGPEBltParms@@@Z 100469b0 f   gpe:FastBlt.obj
 0001:00045bdc       FastBltSelect              10046bdc f   gpe:FastBlt.obj
 0001:00045f28       ?AlphaBlendPixel_32to16at565@@YAKHKKKK@Z 10046f28 f i gpe:FastBlt.obj
 0001:00046144       ?CanUse_Blt_Stretch_Alpha_32To16at565@@YAHPAUGPEBltParms@@@Z 10047144 f i gpe:FastBlt.obj
 0001:000462d0       ?IsAlphaBlend@@YAHPAUGPEBltParms@@@Z 100472d0 f i gpe:FastBlt.obj
 0001:0004634c       ?IsSurface_R5_G6_B5@@YAHPAVGPESurf@@@Z 1004734c f i gpe:FastBlt.obj
 0001:00046424       ?IsSurface_A8_R8_G8_B8@@YAHPAVGPESurf@@@Z 10047424 f i gpe:FastBlt.obj
 0001:00046514       ?CanUse_Blt_NoStretch_Alpha_32To16at565@@YAHPAUGPEBltParms@@@Z 10047514 f i gpe:FastBlt.obj
 0001:00046580       ?AlphaBlendPixel_32to32@@YAKKKK@Z 10047580 f i gpe:FastBlt.obj
 0001:00046608       ?CanUse_Blt_NoStretch_Alpha_24To24@@YAHPAUGPEBltParms@@@Z 10047608 f i gpe:FastBlt.obj
 0001:00046750       ?AlphaBlendPixel_16to16at565@@YAKKKKK@Z 10047750 f i gpe:FastBlt.obj
 0001:00046960       ?CanUse_Blt_NoStretch_Alpha_16To16@@YAHPAUGPEBltParms@@@Z 10047960 f i gpe:FastBlt.obj
 0001:00046aa8       ?CanUse_Blt_NoStretch_Trans_16To16@@YAHPAUGPEBltParms@@@Z 10047aa8 f i gpe:FastBlt.obj
 0001:00046bf0       ?CanUse_Blt_Stretch_Trans_16To16@@YAHPAUGPEBltParms@@@Z 10047bf0 f i gpe:FastBlt.obj
 0001:00046d48       ?CanUse_Blt_NoStretch_NoTrans_32To16at565@@YAHPAUGPEBltParms@@@Z 10047d48 f i gpe:FastBlt.obj
 0001:00046e4c       ?CanUse_Blt_NoStretch_NoTrans_16at565To32@@YAHPAUGPEBltParms@@@Z 10047e4c f i gpe:FastBlt.obj
 0001:00046f64       ?CanUse_Blt_NoStretch_NoTrans_24To24@@YAHPAUGPEBltParms@@@Z 10047f64 f i gpe:FastBlt.obj
 0001:000470a8       ?CanUse_Blt_NoStretch_NoTrans_16To16@@YAHPAUGPEBltParms@@@Z 100480a8 f i gpe:FastBlt.obj
 0001:000471ec       ?CanUse_Blt_Text_32@@YAHPAUGPEBltParms@@@Z 100481ec f i gpe:FastBlt.obj
 0001:00047304       ?CanUse_Blt_Fill_32@@YAHPAUGPEBltParms@@@Z 10048304 f i gpe:FastBlt.obj
 0001:000473c0       ?CanUse_Blt_Fill_24@@YAHPAUGPEBltParms@@@Z 100483c0 f i gpe:FastBlt.obj
 0001:0004747c       ??$swap@J@std@@YAXAAJ0@Z   1004847c f i gpe:FastBlt.obj
 0001:000474bc       EmulatedBltSelect02        100484bc f   gpe:ebbltsel.obj
 0001:000474e0       EmulatedBltSelect08        100484e0 f   gpe:ebbltsel.obj
 0001:0004796c       EmulatedBltSelect16        1004896c f   gpe:ebbltsel.obj
 0001:00047d54       EmulatedBltSelect32        10048d54 f   gpe:ebbltsel.obj
 0001:00047fd0       ?ProcessROP3@@YAKKKKEE@Z   10048fd0 f   gpe:BltHelpers.obj
 0001:000481ac       ?RGBError@@YAKKK@Z         100491ac f   gpe:BltHelpers.obj
 0001:000482b4       ?FillMasksAndShifts@@YAXPAVGPESurf@@PAK1@Z 100492b4 f   gpe:BltHelpers.obj
 0001:00048484       ?ClipRect@@YA_NPAU_RECTL@@PBU1@1@Z 10049484 f   gpe:BltHelpers.obj
 0001:00048630       ?AveragePixels@@YAKKKHHPAK0@Z 10049630 f   gpe:BltHelpers.obj
 0001:00048890       ?AverageAndClampPixels@@YAKKKHHPAK0@Z 10049890 f   gpe:BltHelpers.obj
 0001:00048ba8       ?HalftoneBlend16Bpp@@YAXPAEKHHPAK1@Z 10049ba8 f   gpe:BltHelpers.obj
 0001:00048c08       ?HalftoneBlend24Bpp@@YAXPAEKHHPAK1@Z 10049c08 f   gpe:BltHelpers.obj
 0001:00048cd4       ?HalftoneBlend32Bpp@@YAXPAEKHHPAK1@Z 10049cd4 f   gpe:BltHelpers.obj
 0001:00048d2c       ?InitBrushPixelIterator@BrushPixelIterator@@QAAXPAVGPESurf@@HHPAU_RECTL@@@Z 10049d2c f   gpe:PixelIterator.obj
 0001:00049000       ?InitPixelIterator@PixelIterator@@QAAXPAVGPESurf@@HHPAU_RECTL@@HH@Z 1004a000 f   gpe:PixelIterator.obj
 0001:0004956c       ?InitPixelIterator@PixelIteratorRotate@@QAAXPAVGPESurf@@HHPAU_RECTL@@HH@Z 1004a56c f   gpe:PixelIterator.obj
 0001:000499d8       ?GetPtr@PixelIteratorRotate@@QAAPAEXZ 1004a9d8 f   gpe:PixelIterator.obj
 0001:00049c20       GenBltCpuInitialize        1004ac20 f   gpe:genblt_arm.obj
 0001:00049cd4       ?InvariantInitialize@@YAHPBK@Z 1004acd4 f   gpe:parse.obj
 0001:0004a17c       ?InvariantRecurse@@YAFPBKKKHF@Z 1004b17c f   gpe:parse.obj
 0001:0004a958       ?RopRecurse@@YAFPBKF@Z     1004b958 f   gpe:parse.obj
 0001:0004aba4       ?ConvertRecurse@@YAFPBKKF@Z 1004bba4 f   gpe:parse.obj
 0001:0004af58       ?GenBltInvariantParser@@YA_NPBKPAKPAUGenBltSignature@@@Z 1004bf58 f   gpe:parse.obj
 0001:0004b72c       ?InstructionFetchAndDecode@@YAKPBKPAUPCodeInstruction_t@@@Z 1004c72c f i gpe:parse.obj
 0001:0004b7d8       ?BRegFromBltSig@@YAKPAUGenBltSignature@@@Z 1004c7d8 f   gpe:InitRegs.obj
 0001:0004bc74       ?InitPCodeRegs@@YAXPAUGPEBltParms@@PAUPCodeRegisters_t@@@Z 1004cc74 f   gpe:InitRegs.obj
 0001:0004decc       ?EmulatedBltSrcInvert0808@Emulator@@QAAJPAUGPEBltParms@@@Z 1004eecc f   gpe:ebsinv08.obj
 0001:0004e77c       ?EmulatedBltSrcPaint0808@Emulator@@QAAJPAUGPEBltParms@@@Z 1004f77c f   gpe:ebspnt08.obj
 0001:0004f02c       ?EmulatedBltSrcAnd0808@Emulator@@QAAJPAUGPEBltParms@@@Z 1005002c f   gpe:ebsand08.obj
 0001:0004f8dc       ?EmulatedBltSrcCopy0108@Emulator@@QAAJPAUGPEBltParms@@@Z 100508dc f   gpe:ebcp0108.obj
 0001:000503e4       ?EmulatedBltSrcCopy0408@Emulator@@QAAJPAUGPEBltParms@@@Z 100513e4 f   gpe:ebcp0408.obj
 0001:00050798       ?EmulatedBltSrcCopy0808@Emulator@@QAAJPAUGPEBltParms@@@Z 10051798 f   gpe:ebcopy08.obj
 0001:00050ed0       ?EmulatedBltDstInvert08@Emulator@@QAAJPAUGPEBltParms@@@Z 10051ed0 f   gpe:ebdinv08.obj
 0001:000511d0       ?EmulatedBltPatInvert08@Emulator@@QAAJPAUGPEBltParms@@@Z 100521d0 f   gpe:ebpinv08.obj
 0001:000514e4       ?EmulatedBltPatternInvert08@Emulator@@QAAJPAUGPEBltParms@@@Z 100524e4 f   gpe:ebp08.obj
 0001:00051888       ?EmulatedBltPatternCopy08@Emulator@@QAAJPAUGPEBltParms@@@Z 10052888 f   gpe:ebpcpy08.obj
 0001:00051e94       ?EmulatedBltAlphaText08@Emulator@@QAAJPAUGPEBltParms@@@Z 10052e94 f   gpe:ebalph08.obj
 0001:00051f14       ?EmulatedBltText08@Emulator@@QAAJPAUGPEBltParms@@@Z 10052f14 f   gpe:ebtext08.obj
 0001:00052210       ?EmulatedBltFill08@Emulator@@QAAJPAUGPEBltParms@@@Z 10053210 f   gpe:ebfill08.obj
 0001:000523a8       ?EmulatedBltSrcInvert1616@Emulator@@QAAJPAUGPEBltParms@@@Z 100533a8 f   gpe:EBSINV16.obj
 0001:00052d38       ?EmulatedBltSrcPaint1616@Emulator@@QAAJPAUGPEBltParms@@@Z 10053d38 f   gpe:EBSPNT16.obj
 0001:000536c8       ?EmulatedBltSrcAnd1616@Emulator@@QAAJPAUGPEBltParms@@@Z 100546c8 f   gpe:ebsand16.obj
 0001:00054058       ?EmulatedBltSrcCopy0116@Emulator@@QAAJPAUGPEBltParms@@@Z 10055058 f   gpe:ebcp0116.obj
 0001:00054c08       ?EmulatedBltSrcCopy0416@Emulator@@QAAJPAUGPEBltParms@@@Z 10055c08 f   gpe:ebcp0416.obj
 0001:00054fec       ?EmulatedBltSrcCopy1616@Emulator@@QAAJPAUGPEBltParms@@@Z 10055fec f   gpe:EBCOPY16.obj
 0001:000557d0       ?EmulatedBltAlphaText16@Emulator@@QAAJPAUGPEBltParms@@@Z 100567d0 f   gpe:ebalph16.obj
 0001:00055e90       ?EmulatedBltText16@Emulator@@QAAJPAUGPEBltParms@@@Z 10056e90 f   gpe:ebtext16.obj
 0001:00056188       ?EmulatedBltFill16@Emulator@@QAAJPAUGPEBltParms@@@Z 10057188 f   gpe:ebfill16.obj
 0001:0005640c       ?EmulatedBltSrcCopy0132@Emulator@@QAAJPAUGPEBltParms@@@Z 1005740c f   gpe:EmulatedBltSrcCopy0132.obj
 0001:00056eb4       ?EmulatedBltSrcCopy32@Emulator@@QAAJPAUGPEBltParms@@@Z 10057eb4 f   gpe:EmulatedBltSrcCopy32.obj
 0001:00057698       ?EmulatedBltText32@Emulator@@QAAJPAUGPEBltParms@@@Z 10058698 f   gpe:EmulatedBltText32.obj
 0001:00057988       ?EmulatedBltFill32@Emulator@@QAAJPAUGPEBltParms@@@Z 10058988 f   gpe:EmulatedBltFill32.obj
 0001:00057c60       DDKIomuxSetPadConfig       10058c60 f   cspddk:CSPDDK.dll
 0001:00057c70       DDKIomuxSetPinMux          10058c70 f   cspddk:CSPDDK.dll
 0001:00057c80       DDKGpioWriteDataPin        10058c80 f   cspddk:CSPDDK.dll
 0001:00057c90       DDKGpioSetConfig           10058c90 f   cspddk:CSPDDK.dll
 0001:00057ca0       DDKClockSetGatingMode      10058ca0 f   cspddk:CSPDDK.dll
 0001:00057cb0       DDKClockGetFreq            10058cb0 f   cspddk:CSPDDK.dll
 0001:00057cc0       MmMapIoSpace               10058cc0 f   ceddk:CEDDK.dll
 0001:00057cd0       MmUnmapIoSpace             10058cd0 f   ceddk:CEDDK.dll
 0001:00057ce0       NKDbgPrintfW               10058ce0 f   coredll:COREDLL.dll
 0001:00057cf0       RegCloseKey                10058cf0 f   coredll:COREDLL.dll
 0001:00057d00       RegQueryValueExW           10058d00 f   coredll:COREDLL.dll
 0001:00057d10       RegOpenKeyExW              10058d10 f   coredll:COREDLL.dll
 0001:00057d20       RegSetValueExW             10058d20 f   coredll:COREDLL.dll
 0001:00057d30       GetLastError               10058d30 f   coredll:COREDLL.dll
 0001:00057d40       SystemParametersInfoW      10058d40 f   coredll:COREDLL.dll
 0001:00057d50       ChangeDisplaySettingsEx    10058d50 f   coredll:COREDLL.dll
 0001:00057d60       InitializeCriticalSection  10058d60 f   coredll:COREDLL.dll
 0001:00057d70       CreateThread               10058d70 f   coredll:COREDLL.dll
 0001:00057d80       InterruptInitialize        10058d80 f   coredll:COREDLL.dll
 0001:00057d90       KernelIoControl            10058d90 f   coredll:COREDLL.dll
 0001:00057da0       CreateEventW               10058da0 f   coredll:COREDLL.dll
 0001:00057db0       VirtualSetAttributes       10058db0 f   coredll:COREDLL.dll
 0001:00057dc0       VirtualCopy                10058dc0 f   coredll:COREDLL.dll
 0001:00057dd0       VirtualAlloc               10058dd0 f   coredll:COREDLL.dll
 0001:00057de0       AllocPhysMem               10058de0 f   coredll:COREDLL.dll
 0001:00057df0       FreePhysMem                10058df0 f   coredll:COREDLL.dll
 0001:00057e00       VirtualFree                10058e00 f   coredll:COREDLL.dll
 0001:00057e10       Sleep                      10058e10 f   coredll:COREDLL.dll
 0001:00057e20       DeleteCriticalSection      10058e20 f   coredll:COREDLL.dll
 0001:00057e30       WaitForSingleObject        10058e30 f   coredll:COREDLL.dll
 0001:00057e40       CloseHandle                10058e40 f   coredll:COREDLL.dll
 0001:00057e50       InterruptDisable           10058e50 f   coredll:COREDLL.dll
 0001:00057e60       EventModify                10058e60 f   coredll:COREDLL.dll
 0001:00057e70       InterruptDone              10058e70 f   coredll:COREDLL.dll
 0001:00057e80       LeaveCriticalSection       10058e80 f   coredll:COREDLL.dll
 0001:00057e90       EnterCriticalSection       10058e90 f   coredll:COREDLL.dll
 0001:00057ea0       ExitThread                 10058ea0 f   coredll:COREDLL.dll
 0001:00057eb0       AdvertiseInterface         10058eb0 f   coredll:COREDLL.dll
 0001:00057ec0       GetModuleFileNameW         10058ec0 f   coredll:COREDLL.dll
 0001:00057ed0       WaitForMultipleObjects     10058ed0 f   coredll:COREDLL.dll
 0001:00057ee0       TerminateThread            10058ee0 f   coredll:COREDLL.dll
 0001:00057ef0       SetSystemPowerState        10058ef0 f   coredll:COREDLL.dll
 0001:00057f00       SetLastError               10058f00 f   coredll:COREDLL.dll
 0001:00057f10       GetCallerVMProcessId       10058f10 f   coredll:COREDLL.dll
 0001:00057f20       LocalAlloc                 10058f20 f   coredll:COREDLL.dll
 0001:00057f30       MulDiv                     10058f30 f   coredll:COREDLL.dll
 0001:00057f40       LocalFree                  10058f40 f   coredll:COREDLL.dll
 0001:00057f50       DisableThreadLibraryCalls  10058f50 f   coredll:COREDLL.dll
 0001:00057f60       RegisterDbgZones           10058f60 f   coredll:COREDLL.dll
 0001:00057f70       RegCreateKeyExW            10058f70 f   coredll:COREDLL.dll
 0001:00057f80       LocalReAlloc               10058f80 f   coredll:COREDLL.dll
 0001:00057f90       CeSetExtendedPdata         10058f90 f   coredll:COREDLL.dll
 0001:00057fa0       CacheRangeFlush            10058fa0 f   coredll:COREDLL.dll
 0001:00057fb0       _DllMainCRTStartup         10058fb0 f   corelib0:pegdmain.obj
 0001:00058148       __security_init_cookie     10059148 f   corelib0:seccinit.obj
 0001:000581e0       __GSHandlerCheck           100591e0 f   corelib0:gshandler.obj
 0001:00058224       __GSHandlerCheckCommon     10059224 f   corelib0:gshandler.obj
 0001:000582c8       __security_check_cookie    100592c8 f   corelib0:armsecgs.obj
 0001:000582d8       __gsfailure                100592d8     corelib0:armsecgs.obj
 0001:0005831c       exit                       1005931c f   corelib0:cexit.obj
 0001:00058440       _exit                      10059440 f   corelib0:cexit.obj
 0001:00058460       _cexit                     10059460 f   corelib0:cexit.obj
 0001:00058478       _c_exit                    10059478 f   corelib0:cexit.obj
 0001:00058490       _initterm                  10059490 f   corelib0:crt0dat.obj
 0001:000584dc       _cinit                     100594dc f   corelib0:crt0dat.obj
 0001:0005850c       __crt_ExitProcess          1005950c f   corelib0:exitproc_proxy.obj
 0001:00058538       GetCurrentProcess          10059538 f i corelib0:exitproc_proxy.obj
 0001:00058550       _onexit                    10059550 f   corelib0:onexit.obj
 0001:0005872c       atexit                     1005972c f   corelib0:onexit.obj
 0001:0005877c       memcpy                     1005977c f   corelib1:COREDLL.dll
 0001:0005878c       mbstowcs                   1005978c f   corelib1:COREDLL.dll
 0001:0005879c       wcslen                     1005979c f   corelib1:COREDLL.dll
 0001:000587ac       __rt_sdiv                  100597ac f   corelib1:COREDLL.dll
 0001:000587bc       ??2@YAPAXI@Z               100597bc f   corelib1:COREDLL.dll
 0001:000587cc       memset                     100597cc f   corelib1:COREDLL.dll
 0001:000587dc       malloc                     100597dc f   corelib1:COREDLL.dll
 0001:000587ec       ??3@YAXPAX@Z               100597ec f   corelib1:COREDLL.dll
 0001:000587fc       __itos                     100597fc f   corelib1:COREDLL.dll
 0001:0005880c       __divs                     1005980c f   corelib1:COREDLL.dll
 0001:0005881c       __muls                     1005981c f   corelib1:COREDLL.dll
 0001:0005882c       __adds                     1005982c f   corelib1:COREDLL.dll
 0001:0005883c       __stou                     1005983c f   corelib1:COREDLL.dll
 0001:0005884c       __utos                     1005984c f   corelib1:COREDLL.dll
 0001:0005885c       __rt_udiv                  1005985c f   corelib1:COREDLL.dll
 0001:0005886c       free                       1005986c f   corelib1:COREDLL.dll
 0001:0005887c       wcscpy                     1005987c f   corelib1:COREDLL.dll
 0001:0005888c       swscanf                    1005988c f   corelib1:COREDLL.dll
 0001:0005889c       __C_specific_handler       1005989c f   corelib1:COREDLL.dll
 0001:000588ac       _purecall                  100598ac f   corelib1:COREDLL.dll
 0001:000588bc       memmove                    100598bc f   corelib1:COREDLL.dll
 0001:000588cc       _XcptFilter                100598cc f   corelib1:COREDLL.dll
 0001:000588dc       __security_gen_cookie2     100598dc f   corelib1:COREDLL.dll
 0001:000588ec       __report_gsfailure         100598ec f   corelib1:COREDLL.dll
 0001:000588fc       realloc                    100598fc f   corelib1:COREDLL.dll
 0001:0005890c       _msize                     1005990c f   corelib1:COREDLL.dll
 0001:0005891c       buildDDHALInfo             1005991c f   lcdc_common_topaz_v1:halcaps.obj
 0001:00058ce0       ?HalCreateSurface@@YAKPAU_DDHAL_CREATESURFACEDATA@@@Z 10059ce0 f   lcdc_common_topaz_v1:halsurf.obj
 0001:00058fc0       ?HalCanCreateSurface@@YAKPAU_DDHAL_CANCREATESURFACEDATA@@@Z 10059fc0 f   lcdc_common_topaz_v1:halsurf.obj
 0001:000590fc       ?HalFlip@@YAKPAU_DDHAL_FLIPDATA@@@Z 1005a0fc f   lcdc_common_topaz_v1:halsurf.obj
 0001:00059138       ?HalGetBltStatus@@YAKPAU_DDHAL_GETBLTSTATUSDATA@@@Z 1005a138 f   lcdc_common_topaz_v1:halsurf.obj
 0001:00059268       ?HalUpdateOverlay@@YAKPAU_DDHAL_UPDATEOVERLAYDATA@@@Z 1005a268 f   lcdc_common_topaz_v1:halsurf.obj
 0001:000592e0       ?HalSetOverlayPosition@@YAKPAU_DDHAL_SETOVERLAYPOSITIONDATA@@@Z 1005a2e0 f   lcdc_common_topaz_v1:halsurf.obj
 0001:00059358       ?HalSetColorKey@@YAKPAU_DDHAL_SETCOLORKEYDATA@@@Z 1005a358 f   lcdc_common_topaz_v1:halsurf.obj
 0001:00059414       ?HalGetDriverInfo@@YAKPAU_DDHAL_GETDRIVERINFODATA@@@Z 1005a414 f   lcdc_common_topaz_v1:haldd.obj
 0001:00059480       ?HalWaitForVerticalBlank@@YAKPAU_DDHAL_WAITFORVERTICALBLANKDATA@@@Z 1005a480 f   lcdc_common_topaz_v1:haldd.obj
 0001:000594f8       ?DumpDDSCAPS@@YAXU_DDSCAPS@@@Z 1005a4f8 f   ddgpe:ddhsurf.obj
 0001:000598c8       DDGPESetColorKey           1005a8c8 f   ddgpe:ddhsurf.obj
 0001:00059a20       DDGPECanCreateSurface      1005aa20 f   ddgpe:ddhsurf.obj
 0001:00059b50       DDGPECreateSurface         1005ab50 f   ddgpe:ddhsurf.obj
 0001:0005a58c       DDGPELock                  1005b58c f   ddgpe:ddhsurf.obj
 0001:0005a834       DDGPEUnlock                1005b834 f   ddgpe:ddhsurf.obj
 0001:0005a8d8       DDGPEDestroySurface        1005b8d8 f   ddgpe:ddhsurf.obj
 0001:0005aa0c       DDGPEFlip                  1005ba0c f   ddgpe:ddhsurf.obj
 0001:0005ac64       DDGPEGetFlipStatus         1005bc64 f   ddgpe:ddhsurf.obj
 0001:0005ada4       DDGPESetPalette            1005bda4 f   ddgpe:ddhsurf.obj
 0001:0005ae48       ?BytesPerPixel@GPESurf@@QAAHXZ 1005be48 f i ddgpe:ddhsurf.obj
 0001:0005ae74       ?SetOverlay@DDGPESurf@@QAAXXZ 1005be74 f i ddgpe:ddhsurf.obj
 0001:0005ae94       DDGPECreatePalette         1005be94 f   ddgpe:ddhpalette.obj
 0001:0005af38       DDGPEDestroyPalette        1005bf38 f   ddgpe:ddhpalette.obj
 0001:0005afdc       DDGPESetEntries            1005bfdc f   ddgpe:ddhpalette.obj
 0001:0005b080       DDGPEWaitForVerticalBlank  1005c080 f   ddgpe:ddhdd.obj
 0001:0005b308       DDGPEGetPixelFormatFromSurfaceDesc 1005c308 f   ddgpe:ddhutil.obj
 0001:0005b690       TerminateProcess           1005c690 f   coredll:COREDLL.dll
 0001:0005b7e4       __IMPORT_DESCRIPTOR_CSPDDK 1005c7e4     cspddk:CSPDDK.dll
 0001:0005b7f8       __IMPORT_DESCRIPTOR_CEDDK  1005c7f8     ceddk:CEDDK.dll
 0001:0005b80c       __IMPORT_DESCRIPTOR_COREDLL 1005c80c     coredll:COREDLL.dll
 0001:0005b820       __NULL_IMPORT_DESCRIPTOR   1005c820     cspddk:CSPDDK.dll
 0002:00000000       __imp_MmMapIoSpace         1005d000     ceddk:CEDDK.dll
 0002:00000004       __imp_MmUnmapIoSpace       1005d004     ceddk:CEDDK.dll
 0002:00000008       \177CEDDK_NULL_THUNK_DATA  1005d008     ceddk:CEDDK.dll
 0002:0000000c       __imp_realloc              1005d00c     corelib1:COREDLL.dll
 0002:00000010       __imp__XcptFilter          1005d010     corelib1:COREDLL.dll
 0002:00000014       __imp_memmove              1005d014     corelib1:COREDLL.dll
 0002:00000018       __imp__msize               1005d018     corelib1:COREDLL.dll
 0002:0000001c       __imp___security_gen_cookie2 1005d01c     corelib1:COREDLL.dll
 0002:00000020       __imp___report_gsfailure   1005d020     corelib1:COREDLL.dll
 0002:00000024       __imp_SetLastError         1005d024     coredll:COREDLL.dll
 0002:00000028       __imp_NKDbgPrintfW         1005d028     coredll:COREDLL.dll
 0002:0000002c       __imp_RegCloseKey          1005d02c     coredll:COREDLL.dll
 0002:00000030       __imp_RegQueryValueExW     1005d030     coredll:COREDLL.dll
 0002:00000034       __imp_RegOpenKeyExW        1005d034     coredll:COREDLL.dll
 0002:00000038       __imp_RegSetValueExW       1005d038     coredll:COREDLL.dll
 0002:0000003c       __imp_GetLastError         1005d03c     coredll:COREDLL.dll
 0002:00000040       __imp_SystemParametersInfoW 1005d040     coredll:COREDLL.dll
 0002:00000044       __imp_ChangeDisplaySettingsEx 1005d044     coredll:COREDLL.dll
 0002:00000048       __imp_InitializeCriticalSection 1005d048     coredll:COREDLL.dll
 0002:0000004c       __imp_CreateThread         1005d04c     coredll:COREDLL.dll
 0002:00000050       __imp_InterruptInitialize  1005d050     coredll:COREDLL.dll
 0002:00000054       __imp_KernelIoControl      1005d054     coredll:COREDLL.dll
 0002:00000058       __imp_CreateEventW         1005d058     coredll:COREDLL.dll
 0002:0000005c       __imp_VirtualSetAttributes 1005d05c     coredll:COREDLL.dll
 0002:00000060       __imp_VirtualCopy          1005d060     coredll:COREDLL.dll
 0002:00000064       __imp_VirtualAlloc         1005d064     coredll:COREDLL.dll
 0002:00000068       __imp_AllocPhysMem         1005d068     coredll:COREDLL.dll
 0002:0000006c       __imp_FreePhysMem          1005d06c     coredll:COREDLL.dll
 0002:00000070       __imp_VirtualFree          1005d070     coredll:COREDLL.dll
 0002:00000074       __imp_Sleep                1005d074     coredll:COREDLL.dll
 0002:00000078       __imp_DeleteCriticalSection 1005d078     coredll:COREDLL.dll
 0002:0000007c       __imp_WaitForSingleObject  1005d07c     coredll:COREDLL.dll
 0002:00000080       __imp_CloseHandle          1005d080     coredll:COREDLL.dll
 0002:00000084       __imp_InterruptDisable     1005d084     coredll:COREDLL.dll
 0002:00000088       __imp_EventModify          1005d088     coredll:COREDLL.dll
 0002:0000008c       __imp_InterruptDone        1005d08c     coredll:COREDLL.dll
 0002:00000090       __imp_LeaveCriticalSection 1005d090     coredll:COREDLL.dll
 0002:00000094       __imp_EnterCriticalSection 1005d094     coredll:COREDLL.dll
 0002:00000098       __imp_ExitThread           1005d098     coredll:COREDLL.dll
 0002:0000009c       __imp_AdvertiseInterface   1005d09c     coredll:COREDLL.dll
 0002:000000a0       __imp_GetModuleFileNameW   1005d0a0     coredll:COREDLL.dll
 0002:000000a4       __imp_WaitForMultipleObjects 1005d0a4     coredll:COREDLL.dll
 0002:000000a8       __imp_TerminateThread      1005d0a8     coredll:COREDLL.dll
 0002:000000ac       __imp_SetSystemPowerState  1005d0ac     coredll:COREDLL.dll
 0002:000000b0       __imp_TerminateProcess     1005d0b0     coredll:COREDLL.dll
 0002:000000b4       __imp_GetCallerVMProcessId 1005d0b4     coredll:COREDLL.dll
 0002:000000b8       __imp_LocalAlloc           1005d0b8     coredll:COREDLL.dll
 0002:000000bc       __imp_MulDiv               1005d0bc     coredll:COREDLL.dll
 0002:000000c0       __imp_LocalFree            1005d0c0     coredll:COREDLL.dll
 0002:000000c4       __imp_DisableThreadLibraryCalls 1005d0c4     coredll:COREDLL.dll
 0002:000000c8       __imp_RegisterDbgZones     1005d0c8     coredll:COREDLL.dll
 0002:000000cc       __imp_RegCreateKeyExW      1005d0cc     coredll:COREDLL.dll
 0002:000000d0       __imp_LocalReAlloc         1005d0d0     coredll:COREDLL.dll
 0002:000000d4       __imp_CeSetExtendedPdata   1005d0d4     coredll:COREDLL.dll
 0002:000000d8       __imp_CacheRangeFlush      1005d0d8     coredll:COREDLL.dll
 0002:000000dc       __imp_memcpy               1005d0dc     corelib1:COREDLL.dll
 0002:000000e0       __imp_mbstowcs             1005d0e0     corelib1:COREDLL.dll
 0002:000000e4       __imp_wcslen               1005d0e4     corelib1:COREDLL.dll
 0002:000000e8       __imp___rt_sdiv            1005d0e8     corelib1:COREDLL.dll
 0002:000000ec       __imp_??2@YAPAXI@Z         1005d0ec     corelib1:COREDLL.dll
 0002:000000f0       __imp_memset               1005d0f0     corelib1:COREDLL.dll
 0002:000000f4       __imp_malloc               1005d0f4     corelib1:COREDLL.dll
 0002:000000f8       __imp_??3@YAXPAX@Z         1005d0f8     corelib1:COREDLL.dll
 0002:000000fc       __imp___itos               1005d0fc     corelib1:COREDLL.dll
 0002:00000100       __imp___divs               1005d100     corelib1:COREDLL.dll
 0002:00000104       __imp___muls               1005d104     corelib1:COREDLL.dll
 0002:00000108       __imp___adds               1005d108     corelib1:COREDLL.dll
 0002:0000010c       __imp___stou               1005d10c     corelib1:COREDLL.dll
 0002:00000110       __imp___utos               1005d110     corelib1:COREDLL.dll
 0002:00000114       __imp___rt_udiv            1005d114     corelib1:COREDLL.dll
 0002:00000118       __imp_free                 1005d118     corelib1:COREDLL.dll
 0002:0000011c       __imp_wcscpy               1005d11c     corelib1:COREDLL.dll
 0002:00000120       __imp_swscanf              1005d120     corelib1:COREDLL.dll
 0002:00000124       __imp___C_specific_handler 1005d124     corelib1:COREDLL.dll
 0002:00000128       __imp__purecall            1005d128     corelib1:COREDLL.dll
 0002:0000012c       __imp___stod               1005d12c     corelib1:COREDLL.dll
 0002:00000130       __imp_pow                  1005d130     corelib1:COREDLL.dll
 0002:00000134       __imp___dtos               1005d134     corelib1:COREDLL.dll
 0002:00000138       __imp___subs               1005d138     corelib1:COREDLL.dll
 0002:0000013c       __imp___rt_sdiv64by64      1005d13c     corelib1:COREDLL.dll
 0002:00000140       \177COREDLL_NULL_THUNK_DATA 1005d140     coredll:COREDLL.dll
 0002:00000144       __imp_DDKClockGetFreq      1005d144     cspddk:CSPDDK.dll
 0002:00000148       __imp_DDKClockSetGatingMode 1005d148     cspddk:CSPDDK.dll
 0002:0000014c       __imp_DDKGpioSetConfig     1005d14c     cspddk:CSPDDK.dll
 0002:00000150       __imp_DDKGpioWriteDataPin  1005d150     cspddk:CSPDDK.dll
 0002:00000154       __imp_DDKIomuxSetPinMux    1005d154     cspddk:CSPDDK.dll
 0002:00000158       __imp_DDKIomuxSetPadConfig 1005d158     cspddk:CSPDDK.dll
 0002:0000015c       \177CSPDDK_NULL_THUNK_DATA 1005d15c     cspddk:CSPDDK.dll
 0002:000001e8       ?_rgbIdentity@@3PAUtagPALETTEENTRY@@A 1005d1e8     lcdc_common_topaz_v1:DDLcdc.obj
 0002:000005e8       ?_rgb2bpp@@3PAUtagRGBQUAD@@A 1005d5e8     lcdc_common_topaz_v1:DDLcdc.obj
 0002:000005f8       ?_rgb4bpp@@3PAUtagRGBQUAD@@A 1005d5f8     lcdc_common_topaz_v1:DDLcdc.obj
 0002:00000688       dpCurSettings              1005d688     lcdc_common_topaz_v1:DDLcdc.obj
 0002:00000aec       ?gaMix@@3PAEA              1005daec     gpe:ddi_if.obj
 0002:00000f38       ?pfnDrvAlphaBlend@@3P6AHPAU_SURFOBJ@@0PAU_CLIPOBJ@@PAU_XLATEOBJ@@PAU_RECTL@@3PAUtagBLENDOBJ@@K@ZA 1005df38     gpe:drvalphablend.obj
 0002:00000f40       ?pfnDrvGradientFill@@3P6AHPAU_SURFOBJ@@PAU_CLIPOBJ@@PAU_XLATEOBJ@@PAU_TRIVERTEX@@KPAXKPAU_RECTL@@PAU_POINTL@@K@ZA 1005df40     gpe:rdrvgradfill.obj
 0002:00000f48       ?gulDither32@@3PAKA        1005df48     gpe:rdrvgradfill.obj
 0002:00000f88       ?gDitherMatrix16x16Halftone@@3PAEA 1005df88     gpe:rdrvgradfill.obj
 0002:00001088       ?gDitherMatrix16x16Default@@3PAEA 1005e088     gpe:rdrvgradfill.obj
 0002:00001188       ?vTranslateIdentity@@3PAEA 1005e188     gpe:rdrvgradfill.obj
 0002:00001288       ?DefaultSaturationTable@@3PAEA 1005e288     gpe:rdrvgradfill.obj
 0002:00001408       ?Saturation16_5@@3PAEA     1005e408     gpe:rdrvgradfill.obj
 0002:00001448       ?Saturation16_6@@3PAEA     1005e448     gpe:rdrvgradfill.obj
 0002:000014c8       ?gulGamma@@3KA             1005e4c8     gpe:rctblt.obj
 0002:000014cc       ?szGamma@@3PAGA            1005e4cc     gpe:rctblt.obj
 0002:000014f0       ?szGammaValue@@3PAGA       1005e4f0     gpe:rctblt.obj
 0002:00001508       ?alAlpha@@3PAJA            1005e508     gpe:rctblt.obj
 0002:00001528       ?ajGammaCT_10@@3PAEA       1005e528     gpe:rctblt.obj
 0002:00001628       ?ajGammaCT_11@@3PAEA       1005e628     gpe:rctblt.obj
 0002:00001728       ?ajGammaInvCT_11@@3PAEA    1005e728     gpe:rctblt.obj
 0002:00001828       ?ajGammaCT_12@@3PAEA       1005e828     gpe:rctblt.obj
 0002:00001928       ?ajGammaInvCT_12@@3PAEA    1005e928     gpe:rctblt.obj
 0002:00001a28       ?ajGammaCT_13@@3PAEA       1005ea28     gpe:rctblt.obj
 0002:00001b28       ?ajGammaInvCT_13@@3PAEA    1005eb28     gpe:rctblt.obj
 0002:00001c28       ?ajGammaCT_14@@3PAEA       1005ec28     gpe:rctblt.obj
 0002:00001d28       ?ajGammaInvCT_14@@3PAEA    1005ed28     gpe:rctblt.obj
 0002:00001e28       ?ajGammaCT_15@@3PAEA       1005ee28     gpe:rctblt.obj
 0002:00001f28       ?ajGammaInvCT_15@@3PAEA    1005ef28     gpe:rctblt.obj
 0002:00002028       ?ajGammaCT_16@@3PAEA       1005f028     gpe:rctblt.obj
 0002:00002128       ?ajGammaInvCT_16@@3PAEA    1005f128     gpe:rctblt.obj
 0002:00002228       ?ajGammaCT_17@@3PAEA       1005f228     gpe:rctblt.obj
 0002:00002328       ?ajGammaInvCT_17@@3PAEA    1005f328     gpe:rctblt.obj
 0002:00002428       ?ajGammaCT_18@@3PAEA       1005f428     gpe:rctblt.obj
 0002:00002528       ?ajGammaInvCT_18@@3PAEA    1005f528     gpe:rctblt.obj
 0002:00002628       ?ajGammaCT_19@@3PAEA       1005f628     gpe:rctblt.obj
 0002:00002728       ?ajGammaInvCT_19@@3PAEA    1005f728     gpe:rctblt.obj
 0002:00002828       ?ajGammaCT_20@@3PAEA       1005f828     gpe:rctblt.obj
 0002:00002928       ?ajGammaInvCT_20@@3PAEA    1005f928     gpe:rctblt.obj
 0002:00002a28       ?ajGammaCT_21@@3PAEA       1005fa28     gpe:rctblt.obj
 0002:00002b28       ?ajGammaInvCT_21@@3PAEA    1005fb28     gpe:rctblt.obj
 0002:00002c28       ?ajGammaCT_22@@3PAEA       1005fc28     gpe:rctblt.obj
 0002:00002d28       ?ajGammaInvCT_22@@3PAEA    1005fd28     gpe:rctblt.obj
 0002:00002e28       ?gaOutTable@@3PAU_F_RGB@@A 1005fe28     gpe:rctblt.obj
 0002:00002ff8       ?uAlas@@3PAIA              1005fff8     gpe:ebalph16.obj
 0002:000033f8       __security_cookie          100603f8     corelib0:seccinit.obj
 0002:000033fc       __security_cookie_complement 100603fc     corelib0:seccinit.obj
 0002:00003400       ?FSLFourCC@@3PAKA          10060400     lcdc_common_topaz_v1:halcaps.obj
 0002:00003408       ?cbDDCallbacks@@3U_DDHAL_DDCALLBACKS@@A 10060408     lcdc_common_topaz_v1:halcaps.obj
 0002:00003424       ?MiscellaneousCallbacks@@3U_DDHAL_DDMISCELLANEOUSCALLBACKS@@A 10060424     lcdc_common_topaz_v1:halcaps.obj
 0002:00003434       ?cbDDPaletteCallbacks@@3U_DDHAL_DDPALETTECALLBACKS@@A 10060434     lcdc_common_topaz_v1:halcaps.obj
 0002:00003444       ?cbDDSurfaceCallbacks@@3U_DDHAL_DDSURFACECALLBACKS@@A 10060444     lcdc_common_topaz_v1:halcaps.obj
 0002:00003478       ?VideoPortCallbacks@@3U_DDHAL_DDVIDEOPORTCALLBACKS@@A 10060478     lcdc_common_topaz_v1:halcaps.obj
 0002:000034cc       PATHOBJ_vGetBounds         100604cc     gpe:ddi_if.obj
 0002:000034d0       PATHOBJ_bEnum              100604d0     gpe:ddi_if.obj
 0002:000034d4       PALOBJ_cGetColors          100604d4     gpe:ddi_if.obj
 0002:000034d8       CLIPOBJ_bEnum              100604d8     gpe:ddi_if.obj
 0002:000034dc       EngGetPaletteFromPool      100604dc     gpe:ddi_if.obj
 0002:000034e0       EngAddPaletteToPool        100604e0     gpe:ddi_if.obj
 0002:000034e4       BRUSHOBJ_pvAllocRbrush     100604e4     gpe:ddi_if.obj
 0002:000034e8       BRUSHOBJ_pvGetRbrush       100604e8     gpe:ddi_if.obj
 0002:000034ec       CLIPOBJ_cEnumStart         100604ec     gpe:ddi_if.obj
 0002:000034f0       XLATEOBJ_cGetPalette       100604f0     gpe:ddi_if.obj
 0002:000034f4       PATHOBJ_vEnumStart         100604f4     gpe:ddi_if.obj
 0002:000034f8       EngCreatePalette           100604f8     gpe:ddi_if.obj
 0002:000034fc       EngCreateDeviceSurface     100604fc     gpe:ddi_if.obj
 0002:00003500       EngDeleteSurface           10060500     gpe:ddi_if.obj
 0002:00003504       EngCreateDeviceBitmap      10060504     gpe:ddi_if.obj
 0002:00003508       EngReleasePooledPalette    10060508     gpe:ddi_if.obj
 0002:0000350c       pfnGetGPEPerCard           1006050c     gpe:ddi_if.obj
 0002:00003510       g_hmodDisplayDll           10060510     gpe:ddi_if.obj
 0002:00003514       ?g_pxlo@@3PAU_XLATEOBJ@@A  10060514     gpe:ddi_if.obj
 0002:00003528       ?gMaskedConverter@@3PAVMaskColorConverter@@A 10060528     gpe:swconvrt.obj
 0002:000037a8       ?gLookupConverter@@3PAVLookupColorConverter@@A 100607a8     gpe:swconvrt.obj
 0002:00004828       ?gMonoConverter@@3PAVMonoColorConverter@@A 10061828     gpe:swconvrt.obj
 0002:00004850       ?gMaskedLRU@@3VLRU@@A      10061850     gpe:swconvrt.obj
 0002:00004868       ?gLookupLRU@@3VLRU@@A      10061868     gpe:swconvrt.obj
 0002:00004880       ?gMonoLRU@@3VLRU@@A        10061880     gpe:swconvrt.obj
 0002:00004898       ?gGroupLRU@@3VLRU@@A       10061898     gpe:swconvrt.obj
 0002:000048b0       ?gGroupConverter@@3PAVGroupColorConverter@@A 100618b0     gpe:swconvrt.obj
 0002:00005740       ?pfnGetAAMaskBits@@3P6AXPAK00@ZA 10062740     gpe:aablt.obj
 0002:00005748       ?uBCacheCT@@3KA            10062748     gpe:rctblt.obj
 0002:0000574c       ?uFCacheCT@@3KA            1006274c     gpe:rctblt.obj
 0002:00005750       ?aulCacheCT@@3PAKA         10062750     gpe:rctblt.obj
 0002:0000591c       ?sizeCacheCT@@3KA          1006291c     gpe:rctblt.obj
 0002:00005920       ?uGammaCacheCT@@3KA        10062920     gpe:rctblt.obj
 0002:0000595c       ?gbHateMmx@@3HA            1006295c     gpe:rctblt.obj
 0002:00005be8       ?g_BltFnPData@@3U_xpdata@@A 10062be8     gpe:genblt.obj
 0002:00005c70       ?g_CpuFuncs@@3UGenBltCpuFuncs@@A 10062c70     gpe:genblt.obj
 0002:00005c8c       ?g_pPCodeRegisters@@3PAUPCodeRegisters_t@@A 10062c8c     gpe:genblt.obj
 0002:00005c90       ?g_BltClock@@3KA           10062c90     gpe:genblt.obj
 0002:00005c94       ?g_fUseFastBlt@@3HA        10062c94     gpe:FastBlt.obj
 0002:000074b8       _exitflag                  100644b8     corelib0:cexit.obj
 0002:000074bc       ?g_nVideoMemorySize@@3KA   100644bc     lcdc_common_topaz_v1:halcaps.obj
 0002:000074c0       ?g_pVideoMemory@@3PAEA     100644c0     lcdc_common_topaz_v1:halcaps.obj
 0002:000074c4       __onexitend                100644c4     <common>
 0002:000074c8       __onexitbegin              100644c8     <common>
 0002:000074cc       _pRawDllMain               100644cc     <common>

 entry point at        0001:00057fb0

 Static symbols

 0001:00011cb4       ?GetModeFromRegistry@@YAPAULCD_MODE_INFO@@XZ 10012cb4 f   bsplcdc.obj
 0001:0001200c       ?TurnOnLCD@@YAHPAULCDC_MODE_DESCRIPTOR@@@Z 1001300c f   bsplcdc.obj
 0001:00012148       ?TurnOffLCD@@YAHPAULCDC_MODE_DESCRIPTOR@@@Z 10013148 f   bsplcdc.obj
 0001:000122c4       ?SetWallpaper@@YAXPBG@Z    100132c4 f   bsplcdc.obj
 0001:0001b070       ?FillHelCaps@@YAXPAU_DDCAPS@@@Z 1001c070 f   ddgpe:ddhinit.obj
 0001:00036d50       ?GetAAMaskInfo@@YAXKKK@Z   10037d50 f   gpe:aablt.obj
 0001:00036f34       ?InitGamma@@YAXXZ          10037f34 f   gpe:aablt.obj
 0001:0003ba90       ?MDiv64@@YA_J_J00@Z        1003ca90 f   gpe:rdrvgradfill.obj
 0001:0003bc70       ?RectFillBlt@@YAHPAU_SURFOBJ@@PAU_DRVGRADIENTRECTDATA@@P6AXPAVGPESurf@@1@Z@Z 1003cc70 f   gpe:rdrvgradfill.obj
 0001:0003c0d4       ?GFGetShift@@YAXKPAK0@Z    1003d0d4 f   gpe:rdrvgradfill.obj
 0001:0003cab8       ?GetNearestIndex@@YAKK@Z   1003dab8 f   gpe:rctblt.obj
 0001:00055908       ?EmulatedBltAlphaText16Venus@@YAJPAUGPEBltParms@@@Z 10056908 f   gpe:ebalph16.obj
 0001:00058000       _DllMainCRTStartupHelper   10059000 f   corelib0:pegdmain.obj
 0001:0005833c       doexit                     1005933c f   corelib0:cexit.obj
 0001:0005a554       ?ComputeStride@@YAJII@Z    1005b554 f   ddgpe:ddhsurf.obj
 0001:0005b6a0       ??__EdpCurSettings@@YAXXZ  1005c6a0 f   lcdc_common_topaz_v1:DDLcdc.obj
 0001:0005b6dc       ??__EgMaskedLRU@@YAXXZ     1005c6dc f   gpe:swconvrt.obj
 0001:0005b6f0       ??__EgGroupLRU@@YAXXZ      1005c6f0 f   gpe:swconvrt.obj
 0001:0005b704       ??__EgMonoLRU@@YAXXZ       1005c704 f   gpe:swconvrt.obj
 0001:0005b718       ??__EgLookupLRU@@YAXXZ     1005c718 f   gpe:swconvrt.obj
 0001:0005b72c       ??__EgGroupConverter@@YAXXZ 1005c72c f   gpe:swconvrt.obj
